:020000040800F2
:1000000000000110D1320408E1820308A1D80008E1
:10001000D5330408D5330408D533040800000000A4
:10002000000000000000000000000000218903081B
:100030001F890308000000001D8903084DD4000833
:10004000D5330408D5330408D5330408D533040860
:10005000D5330408D53304085D7A0108897B01088B
:100060004D7B0108117B0108D57A010801AB00081E
:10007000F1AA0008E1AA0008D1AA0008C1AA000854
:10008000ADAA000899AA0008D5330408D53304089E
:10009000D5330408D5330408D5330408997A010808
:1000A000D533040829CB0008C9CA000839CB000899
:1000B00019CB000809CB0008F9CA0008D533040899
:1000C000D5330408D5330408D5330408D5330408E0
:1000D000D5330408B9D60008D533040819D600086A
:1000E000237A0108D5330408DD920308D5330408C8
:1000F000D9CA0008D5330408E9CA000885AA00084F
:10010000D5330408D5330408D5330408D53304089F
:1001100079D50008D5330408F93A0308DD3A030815
:1001200071AA00085DAA000849AA000835AA0008BB
:1001300021AA0008D5330408D5330408D5330408B0
:10014000D5330408D5330408D5330408E382030803
:100150000DAA0008F9A90008E5A90008D9D40008EB
:10016000D5330408D5330408D5330408D53304083F
:10017000D5330408D5330408D5330408D53304082F
:08018000D5330408D53304084F
:08018800682E040001000000D4
:1001900016000800502900206429002000000000FB
:1001A0005406000827000400EC2E0020542F0020E5
:1001B000000000005C060008031233003733002003
:1001C00004330020000000006006000825005A00EB
:1001D00050320020AA320020000000000000000081
:1001E000F6110C009830002044320020000000007E
:1001F000940600081500700064310020D4310020FE
:1002000000000000000000002A006000A430002070
:100210000431002000000000CD1A02080101040092
:10022000F0330020F4460020000000000000000031
:1002300008020900B0460020F84600200000000037
:10024000A96C0108FF010100DC46002004470020E2
:1002500000000000A006000802000C00BC460020C0
:10026000084700200000000000000000F701060021
:10027000A44600201447002000000000A206000849
:1002800001200800944D00209C4D0020000000003B
:10029000A80600081A0008007C4D0020A44D00208C
:1002A00000000000B0060008030001001448002010
:1002B000AC4D002000000000000000002C001000E9
:1002C0004051002030510020000000008D600208E5
:1002D0002B00240074510020505100200000000029
:1002E0005D600208290050005C50002098510020F9
:1002F0000000000000000000090201005654002028
:100300008C54002000000000B8060008010205001F
:10031000005400209054002000000000A581020835
:1003200000020500E8510020985400200000000061
:10033000000000000C00240022560020AC570020D2
:1003400000000000110102080E20EA0016550020EE
:10035000D057002000000000391B020813000400E1
:100360006C560020BC58002000000000BC060008AD
:100370000201030001550020C058002000000000C9
:100380003901020814000200A45A0020E45D002094
:1003900000000000C00600081B00F400D85E00202A
:1003A000A86D002000000000B10503080E02020045
:1003B000A66000209C6E002000000000C20600081D
:1003C0002F0011005A6D0020A06E002000000000D8
:1003D000C406000805100600806D0020B46E0020E1
:1003E00000000000D6060008F5216C004C5E0020DD
:1003F000BC6E00200000000041E302081E00040063
:10040000646F0020D472002000000000DC060008A9
:1004100022000C0004720020D872002000000000AE
:10042000E00600080A020A0014730020247300206A
:1004300000000000EC060008FD012100A48100205E
:10044000C881002000000000D1BD00080600160091
:10045000247E0020EC81002000000000591B0208CF
:10046000FB010100607D00200482002000000000EC
:1004700019BA0008FC0109002C7C00200882002029
:1004800000000000E5B900080A101200007C0020FE
:100490001482002000000000F6060008340010005E
:1004A000507300202882002000000000F51A020886
:1004B00012200C0040730020388200200000000051
:1004C0000807000803010A007882002084820020C7
:1004D00000000000140700081F000E00E483002045
:1004E000B8850020000000001E070008050201007A
:1004F000CC830020C8850020000000002C070008E5
:1005000011000C0084950020E8A0002000000000ED
:100510007901020818102C0024950020F4A0002076
:1005200000000000496302080D00340050950020CF
:1005300020A1002000000000B1010408FA0102001F
:10054000088E002054A100200000000075BA0008A9
:1005500002020300F08D002058A1002000000000DE
:10056000000000000C020100E08D00205CA10020D2
:10057000000000002E07000826000E0090A70020B3
:1005800080A700200000000019D203080B201000F3
:1005900064A50020A0A7002000000000300700088C
:1005A0001000030018A8002024A80020000000006C
:1005B000400700082800100008A8002028A80020F4
:1005C00000000000B1B1020823001000F8A70020CD
:1005D00038A800200000000085AF030819000500BE
:1005E000F0A7002048A800200000000044070008F1
:1005F000F8110100ECA7002050A800200000000026
:100600004A07000800010400E8A7002054A80020C1
:10061000000000004C070008FE0109000CAA0020A1
:1006200060AA00200000000055BA00080400800005
:10063000B8CA0020D0D30020000000000000000055
:10064000F901040034AD002050D400200000000067
:0406500041BE00089F
:10065400C40900001901282820030000000000003C
:100664000000000000000000000000000000000086
:100674000000000000000000000000000000000076
:100684000000000000000000000000000000010065
:100694000000000000000000000000000000240131
:1006A4000000D80EE8036400040A00017E05EA0590
:1006B400B405320029000000080004000300000013
:1006C4000000000000000000000000000000000026
:1006D400000020000201000000000100C800141EF8
:1006E400010064002C01280000004A01B400D60176
:1006F400290000300100005A0000000090012C0184
:10070400C8006400000000010005434C523400009E
:10071400040101006C16000000000000000000004D
:100724000100000000050000000001002B21231E31
:1007340064010100000001000A0129000001050014
:0C0744000000280100000400FA00000082
:10075000010000005001000007000000020000003E
:100760000000000000000000010203040607080961
:1007700001010000007F040884BB040800000000A1
:1007800000000000107F0408187F0408000000002B
:10079000012000001C7F0408247F040800000000E2
:1007A00001400000287F0408A09504080000000014
:1007B00001200000347F0408407F0408000000008E
:1007C00004000000447F040864BA0408000000002C
:1007D00004000000507F04083CAA04080000000048
:1007E000010000000201FF000000803F0000803F88
:1007F000FFFFFFFF986804080508040000000000E0
:10080000B06B0408707104089C6B040800000000C1
:10081000C468040805080A0000000000B06B040862
:1008200070710408C86B0408000000000000803FDD
:100830000000000000000000000000000000803FF9
:1008400000000000000000000000000000000000A8
:100850000000000000000000000000000000000098
:10086000000000000000803F0000000000000000C9
:1008700000000000E001010101000000698302089E
:1008800000000000A0020020DCAF0408000000000F
:1008900000000000000000000000000084BB04080D
:1008A0000000000000000000E4060020040000003A
:1008B00088AF04080D000000399E0208CC06002015
:1008C0000000000010B304080D000000119E020893
:1008D000C006002000000000FCAF04080800000073
:1008E00000000000B406002004000000ECAF040883
:1008F0000D00000041970208A8060020000000003B
:1009000098AE04080300000075A002089C060020B1
:1009100000000000F4AF04080300000075A0020806
:1009200090060020000000009CAE040801000000BA
:1009300000000000000000000000000000000000B7
:100940000E00000000000000000000000000000099
:10095000DCAF040800000000000000000000000000
:100960000000000084BB040800000000000000003C
:10097000E40600200400000020AF0408030000008B
:100980003D8B02088406002008000000ECAF04083C
:100990000D00000041970208A8060020000000009A
:1009A00098AE04080300000075A002089C06002011
:1009B00000000000F4AF04080300000075A0020866
:1009C00090060020000000009CAE0408010000001A
:1009D0000000000000000000000000000000000017
:1009E0000E000000000000000000000000000000F9
:1009F00004B0040800000000000000000000000037
:100A00000000000084BB040800000000000000009B
:100A1000E40600200400000028AF040803000000E2
:100A200075A00208D8060020000000009CAE040853
:100A300001000000000000000000000000000000B5
:100A4000000000000E000000000000000000000098
:100A500000000000080000008454002088136F1775
:100A6000010000008654002088136F17000000006A
:100A700070AE04080000000000000000000000004C
:100A80000000000080AE0408080000000000000024
:100A900014030020040000008CAE040808000000CD
:100AA00000000000080300200000000098AE0408C9
:100AB000040000004D9C020800000000000000003F
:100AC0009CAE0408010000000000000000000000CF
:100AD00000000000000000000E0000000000000008
:100AE0000000000000000000FC53002088136F1776
:100AF00001000000C483002088136F17000000006D
:100B000019970208000000002003002088540020EC
:100B100001000000706B0408C68300200100000083
:100B20007C6B0408BC83002002000000846B040876
:100B30008ECB002000000000000000008CCB0020C5
:100B400000000000000000008ACB00200000000030
:100B50000000000088CB0020000000000000000022
:100B600086CB0020000000000000000084CB0020A5
:100B70000000000000000000981D002000000000A0
:100B800000000000FB53002002000000906B0408EE
:100B9000D8AE0408000000000000000000000000C3
:100BA0000000000080AE0408080000000000000003
:100BB000A4030020040000008CAE0408080000001C
:100BC00000000000980300200000000098AE040818
:100BD00004000000A18302080000000000000000E3
:100BE0009CAE0408010000000000000000000000AE
:100BF00000000000000000000E00000000000000E7
:100C00000000000000000000E8AE04080000000042
:100C1000000000000000000000000000F8AE040822
:100C20000D000000B99D0208D4030020040000005C
:100C300004AF04080D000000959D0208C8030020C1
:100C40000400000010AF04080D000000699C0208B9
:100C5000BC030020000000001CAF040803000000DB
:100C60002D9C0208B00300200800000028AF0408F3
:100C70000300000075A00208D80600200000000054
:100C80009CAE04080100000000000000000000000D
:100C900000000000000000000E0000000000000046
:100CA000000000000000000030AF04080000000059
:100CB00000000000000000000000000038AF040841
:100CC000040000009D9C02080000000000000000DD
:100CD0009CAE0408010000000000000000000000BD
:100CE00000000000000000000E00000000000000F6
:100CF000000000000000000090AF040800000000A9
:100D00000000000000000000000000006CA30408C8
:100D10000D0000000000000034040020040000006A
:100D2000A0AF040808000000000000002804002014
:100D300004000000ACAF0408080000000000000040
:100D40001C04002004000000B4AF040808000000E8
:100D5000000000001004002004000000BCAF0408E4
:100D6000080000000000000004040020040000004F
:100D7000C4AF04080800000000000000F8030020D1
:100D800004000000CCAF04080800000000000000D0
:100D9000EC03002004000000D4AF040808000000A9
:100DA00000000000E0030020040000009CAE0408E6
:100DB0000100000000000000000000000000000032
:100DC000000000000E000000000000000000000015
:100DD00000000000B9830208000000004004002069
:100DE0000000000000000000B80400200000000027
:100DF0000000000058050020C2830020040000000D
:100E00009C6B0408C0830020E0150C170000000054
:100E1000BF8300200800000070710408BE8300201A
:100E200005000000B06B0408000000000000000096
:100E3000A80500202D202D2D202D2D2D2D202D2DF0
:100E40002D00000000000000000000000000000075
:100E50000000000020700020702D720000000000D3
:100E600000000000441A0020FFFFFFFFFA0000000E
:100E7000010000000100000070B0040878B0040810
:100E800030AF040800000000000000000000000077
:100E9000000000005CB0040804000000B18A0208F1
:100EA00000000000000000009CAE040801000000EB
:100EB0000000000000000000000000000000000032
:100EC0000E00000000000000000000000000000014
:100ED000826000200100C409000000008060002042
:100EE0000100C409000000007E6000200100C40968
:100EF000000000007C6000200100C4090000000028
:100F0000786000200100C409000000007A60002021
:100F10000100C40900000000766000200100C4093F
:100F200000000000746000200100C40900000000FF
:100F3000AC5400200100C80001000000AA540020A9
:100F40003200307532000000A9540020055A050017
:100F5000A454002000FF0100A8540020010000005C
:100F600028070020A6540020020000009C6E040800
:100F7000A354002000FF0100A7540020010000003E
:100F800028070020A5540020020000009C6E0408E1
:100F900000000000000000003007002088830020CF
:100FA0009CFF2C0100000000260100200A00000028
:100FB000C86B0408F8530020E0150C17000000006F
:100FC000280100200800000070710408270100209B
:100FD00005000000B06B0408FA5300200200000076
:100FE000E06B04085A5600200100FF7F010000005A
:100FF0005956002002000000EC6B04080A5500203E
:1010000003000000FC6B04080955002003000000E9
:10101000FC6B0408085600200000F40101000000E9
:10102000065600200000F4010100000004560020D4
:101030000000F40101000000025600200000F4014D
:10104000010000000056002000FF01002056002093
:10105000E803D0070A0000001E56002000640100CB
:101060000A0000001A5600200064010019560020F2
:10107000006401001F560020006401000A00000007
:1010800018560020006401000A0000001D560020D0
:10109000006401000A0000001C56002000640100EA
:1010A0000A0000001B560020006401000A00000036
:1010B0001756002000FF01000A000000165600200D
:1010C00000FF01000A000000125500200000F4019A
:1010D00001000000105500200000F4010100000094
:1010E0000E5500200000F401010000000C55002006
:1010F0000000F40101000000125600201400E80373
:101100000100000010560020E803307501000000C7
:101110000F56002000C801000E56002000C8010034
:101120000D56002000C801000C560020006401008C
:101130000A0000000B56002000FF01000A0000001A
:101140004F56002000C801004E56002000C8010084
:101150004D56002000C801004C56002000C8010078
:101160004B56002000C801004A56002000C801006C
:101170004956002000C801004856002000C8010060
:101180004756002000C80100A4B004080000000079
:10119000000000000000000000000000B4B00408DF
:1011A0000900000000000000D40700200400000037
:1011B000BCB004080900000000000000C8070020BF
:1011C000040000004CB60408090000000000000004
:1011D000BC07002004000000308004080900000063
:1011E00000000000B007002004000000C4B00408A4
:1011F0000900000000000000A40700200400000017
:10120000CCB004080900000000000000980700208E
:1012100004000000D4B00408090000000000000031
:101220008C07002004000000DCB004080900000066
:101230000000000080070020040000009CAE0408AD
:10124000010000000000000000000000000000009D
:10125000000000000E000000000000000000000080
:1012600000000000F0B104080000000000000000D1
:10127000000000000000000090A00408070000002B
:1012800000000000F80700200000000000B2040881
:101290000800000000000000EC0700200000000033
:1012A0000CB204080800000000000000E007002065
:1012B000000000009CAE04080100000000000000D7
:1012C0000000000000000000000000000E00000010
:1012D00000000000000000000000000014B204083C
:1012E00000000000000000000000000000000000FE
:1012F00024B204080D0000000000000034080020A3
:10130000000000002CB204080D00000000000000E6
:10131000280800200000000034B204080700000084
:101320000000000020080020000000003CB204087B
:101330000D00000000000000140800200000000064
:1013400044B204080D00000000000000080800205E
:10135000000000004CB2040807000000000000007C
:1013600000080020000000009CAE040801000000FE
:10137000000000000000000000000000000000006D
:101380000E0000000000000000000000000000004F
:1013900054B204080000000000000000000000003B
:1013A0000000000090A004080C00000000000000F5
:1013B000AE5400200000000068B204080C000000D9
:1013C00000000000B05400200000000078B20408C3
:1013D0000C00000000000000E654002000000000A7
:1013E00088B204080C00000000000000DA5400205D
:1013F000000000009CB204080C0000000000000087
:10140000B254002000000000A8B204080C00000044
:1014100000000000B454002000000000B0B2040836
:101420000C00000000000000B65400200000000086
:10143000C4B204080C00000000000000B8540020F2
:1014400000000000CCB204080C0000000000000006
:10145000BA54002000000000D4B204080C000000C0
:1014600000000000F854002000000000ECB2040866
:101470000C00000000000000BC5400200000000030
:10148000F8B204080C00000000000000BE54002068
:101490000000000000B304080C0000000000000081
:1014A000C0540020000000000CB304080C00000031
:1014B00000000000C25400200000000018B304081F
:1014C0000C00000000000000C454002000000000D8
:1014D00024B304080C00000000000000C6540020E3
:1014E0000000000030B304080C0000000000000001
:1014F000C8540020000000003CB304080C000000A9
:1015000000000000CA5400200000000048B3040896
:101510000C00000000000000DE540020000000006D
:1015200050B304080C00000000000000DC54002050
:101530000000000058B304080C0000000000000088
:10154000EA5400200000000064B304080C0000000E
:1015500000000000EC5400200000000070B30408FC
:101560000C00000000000000F25400200000000009
:1015700088B104080C00000000000000CC540020DA
:1015800000000000ECAF04080C00000000000000A8
:10159000D4540020000000007CB304080C000000BC
:1015A00000000000CE5400200000000088B30408B2
:1015B0000C00000000000000D054002000000000DB
:1015C00094B304080C00000000000000D254002076
:1015D000000000009CB304080C00000000000000A4
:1015E000D654002000000000B0A004080C00000049
:1015F00000000000E054002000000000A8B3040830
:101600000C00000000000000D85400200000000082
:10161000B4B304080C00000000000000E8540020EF
:1016200000000000C0B304080C000000000000002F
:10163000E254002000000000C8B304080C000000C1
:1016400000000000E454002000000000D0B30408B3
:101650000C00000000000000EE540020000000001C
:10166000D8B304080C00000000000000F054002073
:10167000000000009CAE0408010000000000000013
:101680000000000000000000000000000E0000004C
:10169000000000000000000000000000E0B30408AB
:1016A000000000000000000000000000000000003A
:1016B000F0B30408050000000000000008550020F9
:1016C000000000009CAE04080100000000000000C3
:1016D0000000000000000000000000000E000000FC
:1016E000000000000000000000000000F8B3040843
:1016F00000000000000000000000000000000000EA
:1017000084BB040800000000000000005F1D0020F2
:101710000400000004B404080D000000158B02084A
:10172000880800200000000088AF04080D000000B9
:101730004D8302087C0800200000000010B304085C
:101740000D00000031830208700800200000000036
:10175000FCAF04080800000000000000640800203E
:1017600004000000ECAF04080D00000079820208BC
:10177000580800200000000008B404080900000018
:10178000000000004C0800200400000098AE04088F
:101790000300000075A002084008002000000000BF
:1017A0009CAE0408010000000000000000000000E2
:1017B00000000000000000000E000000000000001B
:1017C000000000000000000010B404080000000049
:1017D00000000000000000000000000020B4040829
:1017E0000D00000000000000A00800200000000024
:1017F00028B404080A00000000000000C8560020B9
:101800000000000034B404080A00000000000000DA
:10181000D0560020000000003CB404080A0000007C
:1018200000000000D85600200000000044B4040866
:1018300008000000000000009408002000000000E4
:101840004CB404080400000031A2020800000000AB
:10185000000000009CAE0408010000000000000031
:101860000000000000000000000000000E0000006A
:1018700000000000000000000000000058B4040850
:101880000000000000000000000000000000000058
:101890006CB404080D00000000000000B80800202F
:1018A000000000007CB4040804000000B59E02089B
:1018B000000000000000000084B404080D000000D7
:1018C00000000000AC0800200000000098B40408EC
:1018D00004000000919E02080000000000000000CB
:1018E0009CAE0408010000000000000000000000A1
:1018F00000000000000000000E00000000000000DA
:101900000000000000000000A0B404080000000077
:10191000000000000000000000000000B4B4040853
:101920000700000000000000F40800200000000094
:10193000C0B404080800000000000000E80800200F
:1019400000000000CCB40408080000000000000003
:10195000DC08002000000000D8B4040808000000E3
:1019600000000000D008002000000000E4B40408DB
:101970000800000000000000C40800200000000073
:101980009CAE040801000000000000000000000000
:1019900000000000000000000E0000000000000039
:1019A0000000000000000000F0B404080000000087
:1019B0000000000007070020000000005C7F040812
:1019C0000B000000000000006C0900200000000077
:1019D000FCB404080B0000000000000060090020B7
:1019E0000000000008B504080B0000000000000023
:1019F000540900200000000014B504080B0000008A
:101A000000000000480900200000000020B5040884
:101A10000B000000000000003C0900200000000056
:101A2000647F04080B000000000000003009002063
:101A3000000000002CB504080B00000000000000AE
:101A4000240900200000000038B504080700000049
:101A5000000000001C0900200000000040B5040840
:101A60000700000000000000140900200000000032
:101A70004CB504080B00000000000000080900201D
:101A80000000000058B50408080000000000000035
:101A9000FC080020000000009CAE040801000000CB
:101AA0000000000000000000000000000000000036
:101AB0000E00000000000000000000000000000018
:101AC00064B50408000000000000000000000000F1
:101AD0000000000078B504080800000000000000C5
:101AE0009C0900200000000084B5040808000000E4
:101AF00000000000900900200000000090B50408DC
:101B00000800000000000000840900200000000020
:101B10009CB50408080000000000000078090020BF
:101B2000000000009CAE040801000000000000005E
:101B30000000000000000000000000000E00000097
:101B4000000000000000000000000000A4B5040830
:101B5000000000000000000004070020000000005A
:101B6000B4B504080B00000000000000E4090020E8
:101B700000000000C0B504080B00000000000000D9
:101B8000D809002000000000CCB5040807000000C0
:101B900000000000D009002000000000D8B50408B3
:101BA0000700000000000000C8090020000000003D
:101BB000E4B504080700000000000000C009002090
:101BC00000000000F0B5040808000000000000005C
:101BD000B409002000000000F8B504080800000067
:101BE00000000000A8090020000000009CAE0408CE
:101BF00001000000000000000000000000000000E4
:101C0000000000000E0000000000000000000000C6
:101C10000000000000B60408000000000000000002
:101C200004070020000000000CB6040807000000B4
:101C300000000000300A00200000000014B6040874
:101C40000700000000000000280A0020000000003B
:101C50001CB604080700000000000000200A002055
:101C600000000000F87F04080700000000000000EA
:101C7000180A00200000000000800408070000008F
:101C800000000000100A0020000000000880040886
:101C90000700000000000000080A0020000000000B
:101CA00024B604080700000000000000000A00201D
:101CB000000000002CB6040807000000000000002F
:101CC000F80900200000000034B6040807000000F6
:101CD00000000000F0090020000000009CAE040895
:101CE00001000000000000000000000000000000F3
:101CF000000000000E0000000000000000000000D6
:101D0000000000000000000015990208380A0020B9
:101D1000065500201B0000000C6C0408055500202F
:101D20000A3201000455002001FA0100005500208C
:101D300000C80100FE540020E803D00701000000A5
:101D4000434C524143494E4746340000A2540020C0
:101D500000030100A154002000030100399802088B
:101D600015980208140B0020DD9702089D970208C1
:101D70008C0B0020759802085D980208400C00202A
:101D80002B990208619E02084C0F0020B9820208BC
:101D9000000000009C0F00200DA20208919B020889
:101DA0007810002051990208000000002C1100203A
:101DB000F5990208C5990208B8110020819A020815
:101DC000C59A020858120020145600200103010091
:101DD000919902086599020870130020259A02085B
:101DE000D99E0208FC130020F19A0208359F0208D0
:101DF000C41400200A560020010301003CB6040868
:101E000000000000000000000000000000000000D2
:101E100048B604080800000000000000E415002097
:101E20000000000050B60408070000000000000099
:101E3000DC1500200000000060B604080700000068
:101E400000000000D4150020000000006CB604085B
:101E50000700000000000000CC150020000000007A
:101E600078B604080D00000000000000C015002036
:101E70000000000084B604080300000075A00208FA
:101E8000B4150020000000009CAE04080100000012
:101E90000000000000000000000000000000000042
:101EA0000E00000000000000000000000000000024
:101EB0008CB60408000000000000000000000000D4
:101EC000000000009CB604080A00000000000000AA
:101ED000987E040800000000A4B604080A00000070
:101EE00000000000E07E040800000000ACB604081A
:101EF0000A00000000000000505600200000000012
:101F0000B4B604080A00000000000000F01500202C
:101F1000000000009CAE040801000000000000006A
:101F20000000000000000000000000000E000000A3
:101F3000000000000000000000000000BCB6040823
:101F40000000000000000000000000000000000091
:101F5000C8B604080300000075A00208241600207B
:101F600000000000D4B604080300000075A00208B9
:101F70001816002000000000DCB604080300000072
:101F800075A002080C16002000000000E4B604084A
:101F90000500000000000000A05400200000000028
:101FA000ECB6040807000000000000000416002042
:101FB00000000000F8B60408070000000000000060
:101FC000FC150020000000009CAE04080100000089
:101FD0000000000000000000000000000000000001
:101FE0000E000000000000000000000000000000E3
:101FF00004B704080000000000000000000000001A
:102000000000000018B704080300000075A00208D3
:10201000481600200000000024B704080300000058
:1020200075A002082C010020000000002CB7040855
:102030000300000075A002083C160020000000000C
:1020400034B704080300000075A002083016002011
:10205000000000009CAE0408010000000000000029
:102060000000000000000000000000000E00000062
:1020700000000000000000000000000040B704085D
:102080000000000000000000000000000000000050
:102090004CB7040807000000819F0208A416002026
:1020A0000000000098B304080300000075A00208B7
:1020B000981600200000000058B704080300000034
:1020C00075A002088C1600200000000060B704080C
:1020D0000300000075A00208801600200000000028
:1020E00068B7040807000000659F02087816002002
:1020F000000000008C7F04080300000075A00208A7
:102100006C1600200000000074B7040803000000F3
:1021100075A00208601600200000000080B70408C7
:102120000300000075A00208541600200000000003
:102130009CAE040801000000000000000000000048
:1021400000000000000000000E0000000000000081
:102150000000000000000000D19802088D980208DD
:10216000AC1600205D9B02080000000060170020F4
:102170008197020865970208EC1700200000000014
:1021800000000000A0180020359B02089D9F020857
:102190002C1900208CB7040800000000000000008B
:1021A000000000000000000098B7040803000000D1
:1021B00075A00208381A002000000000A0B704082B
:1021C0000300000075A002082C1A00200000000087
:1021D000A8A104080300000075A00208201A00202E
:1021E00000000000ACB704080300000075A002085E
:1021F000141A002000000000B8B704080300000013
:1022000075A00208081A002000000000C0B70408EA
:1022100002000000E1A2020800000000000000002F
:10222000C8B7040802000000E1A202080100000093
:1022300000000000D4B7040802000000E1A2020878
:102240000200000000000000000000000E0000007E
:10225000000000000000000000000000000101017B
:102260000100000009024300020100C0320904001D
:1022700000010202010005240010010524010001F3
:10228000042402020524060001070582030800FF5A
:1022900009040100020A00000007050102400000D5
:1022A0000705810240000000FF000000010100005E
:1022B000FFFFFFFF000001FFFF0000000000803F64
:1022C000000000000000000000000000010000000D
:1022D000006002401060024000000000000B00009F
:1022E000000020000000000000000000006002402C
:1022F0002860024000000000060C000000002000E2
:102300000000000000000000006002404060024049
:1023100000000000100D0000000020000000000080
:102320000000000000600240586002400000000011
:10233000160E000000002000000000000000000059
:10234000006002407060024000000000200F0000AA
:1023500000002000000000000000000000600240BB
:1023600088600240000000002610000000002000ED
:10237000000000000000000000600240A060024079
:1023800000000000301100000000200000000000EC
:102390000000000000600240B86002400000000041
:1023A000362F0000000020000000000000000000A8
:1023B0000064024010640240000000000038000089
:1023C0000000400000000000000000000064024027
:1023D00028640240000000000639000000004000B0
:1023E0000000000000000000006402404064024061
:1023F00000000000103A0000000040000000000053
:102400000000000000640240586402400000000028
:10241000163B00000000400000000000000000002B
:10242000006402407064024000000000203C000094
:1024300000004000000000000000000000640240B6
:1024400088640240000000002644000000004000B4
:10245000000000000000000000640240A064024090
:1024600000000000304500000000400000000000B7
:102470000000000000640240B86402400000000058
:102480003646000000004000000000000000000090
:10249000000000000102030401020304060708090A
:1024A00000FFFF0000000000AA5505010000012DFB
:1024B000202D2D202D2D2D2D202D2D2D2D000000FA
:1024C0000000000000000000000000000000AA550D
:1024D0000B010000AA5507010000AA5509020000DF
:1024E0000000000001000000C012AA5503009F0078
:1024F0000403090412010002020200408304405751
:1025000000020102030100002562030811630308B1
:10251000E15C030835CB02089164030845CB02084F
:1025200061CB020825CB020815CB02080000000091
:102530000000000008000000000000010000000092
:10254000000000000000000049CF020801CF02088F
:1025500079E2020800000000F1CA020855CE020824
:10256000D5CE0208BDCD020800000000000000002A
:10257000E5CA020855800308538003085180030808
:102580004B800308498003084F8003084D800308EF
:102590006580030857800308758103088981030853
:1025A000618103084D810308398103080101D601C7
:1025B000FDB403080000000000000000DCA00408D7
:1025C00000000000000000004D010208A08601008C
:1025D00004000000000000000000000000000000F7
:1025E00000000000000000000000000000000000EB
:1025F00098B3040830A00408000000007993010893
:102600007D00000006000000000000000000000047
:1026100000000000000000000000000000000000BA
:1026200000000000E8BB04080000000000000000FB
:10263000914F0108E80300000300000000000000C3
:10264000000000000000000000000000000000008A
:102650000000000000000000F0BB040800000000C3
:1026600000000000911C0208102700000300000079
:10267000000000000000000000000000000000005A
:10268000000000000000000000000000FCBB040887
:1026900000000000ADB9030859290108204E0000D0
:1026A0000500000000000000000000000000000025
:1026B000000000000000000000000000000000001A
:1026C0006CA20408000000000000000045D90008CA
:1026D00010270000010000000000000000000000C2
:1026E00000000000000000000000000000000000EA
:1026F0000000000000BC0408000000000000000012
:10270000B1B90008E8030000050000000000000067
:1027100000000000000000000000000000000000B9
:1027200000000000000000000CBC040800000000D5
:1027300000000000AD030208204E0000030000006E
:102740000000000000000000000000000000000089
:102750000000000000000000000000001CBC040895
:102760000000000000000000B5010208204E00003B
:102770000300000000000000000000000000000056
:102780000000000000000000000000000000000049
:102790002CBC040800000000000000008153010868
:1027A000400D0300030000000000000000000000D6
:1027B0000000000000000000000000000000000019
:1027C00000000000A0A104080000000000000000BC
:1027D000710904081027000001000000000000003B
:1027E00000000000000000000000000000000000E9
:1027F00000000000000000004CA0040800000000E1
:1028000000000000CD17030810270000030000009F
:1028100000000000000000000000000000000000B8
:1028200000000000000000000000000074A2040886
:102830000000000000000000BDFE0008A00F000026
:102840000100000000000000000000000000000087
:102850000000000000000000000000000000000078
:102860003CBC0408000000000000000095E50208E0
:102870001027000001000000000000000000000020
:102880000000000000000000000000000000000048
:1028900000000000CCA104080000000000000000BF
:1028A000B5050208A00F00000100000000000000B4
:1028B0000000000000000000000000000000000018
:1028C0000000000000000000A8A1040800000000B3
:1028D00000000000FDF502081A41000001000000A0
:1028E00000000000000000000000000000000000E8
:1028F000000000000000000000000000D8A2040852
:102900000000000000000000496C030810270000D0
:1029100001000000000000000000000000000000B6
:1029200000000000000000000000000000000000A7
:1029300048BA0408000000000000000075A4020866
:102940001A4100000100000000000000000000002B
:102950000000000000000000000000000000000077
:102960000000000048BC0408000000000000000057
:1029700055560108400D0300000000000000000053
:102980000000000000000000000000000000000047
:10299000000000000000000050BC0408000000001F
:1029A00000000000F1550108400D03000000000088
:1029B0000000000000000000000000000000000017
:1029C00000000000000000000000000058BC0408E7
:1029D0000000000000000000898B0208A0860100B2
:1029E00003000000000000000000000000000000E4
:1029F00000000000000000000000000000000000D7
:102A00000000803F01000000BC2200200000000008
:102A100000000000000000000000000000000000B6
:102A200000000000000000000000000000000000A6
:102A30000000000000000000000000000000000096
:102A40000000000000000000000000000000000086
:102A50000000000000000000000000000000000076
:102A60000000000000000000000000004300000023
:102A70000000000000000000000000000000000056
:102A80000000000000000000000000004300000003
:102A90000000000000000000000000000000000036
:102AA00000000000000000000000000043000000E3
:102AB0000000000000000000000000000000000016
:102AC00000000000000000000000000043000000C3
:102AD00000000000000000000000000000000000F6
:102AE00000000000000000000000000043000000A3
:102AF00000000000000000000000000000000000D6
:102B00000000000000000000000000004300000082
:102B100000000000000000000000000000000000B5
:102B20000000000000000000000000004300000062
:102B30000000000000000000000000000000000095
:102B400000000000000000000000000073360408D0
:102B50004F36040800000000D1C1040858B0040832
:102B60008B8504088B8504088B8504088B850408F5
:102B70008B8504088B8504088B8504088B850408E5
:102B80008B850408FFFFFFFFFFFFFFFFFFFFFFFF35
:102B9000FFFF0000010041534349490000000000CD
:102BA0000000000000000000000000000000000025
:102BB00000000000000041534349490000000000AC
:102BC0000000000000000000000000000000000005
:0C2BD000000000000000000001000000F8
:108000004FF40063838270474FF4006383827047AC
:108010004FF4805383827047012380F845307047C6
:10802000BFF34F8F0549064BCA6802F4E062134361
:10803000CB60BFF34F8F00BFFDE700BF00ED00E056
:108040000400FA0570B4037B04681F2B08D9203B99
:108050002021626801FA03F31A421CD170BC7047F8
:108060002021226801FA03F31A42F7D04269144929
:108070005C2000FB021251685689CD6808682968A7
:1080800021F001012960828992B222EA06028281EE
:10809000A36070BC7047426909495C2000FB021272
:1080A00051685689CD680868296821F00101296066
:1080B000828992B222EA06028281E36070BC704734
:1080C0004C7E00202B4B1978002951D02A4B30B41C
:1080D0001C68988800226262A5899A80284380B231
:1080E0000129A08143D09C6898896262A5892843B0
:1080F00080B20229A0819A8139D01C69988A626273
:10810000A589284380B20329A0819A822FD09C6937
:10811000988B6262A589284380B20429A0819A8342
:1081200025D01C6A988C6262A589284380B20529F3
:10813000A0819A841BD09C6A988D6262A58928438D
:1081400080B20629A0819A8511D01C6B988E62623C
:10815000A589284380B20729A0819A8607D0986B09
:10816000998F42628489214389B281819A8730BC88
:10817000704700BF2C8100203081002010B4037BA9
:1081800001681F2B09D9203B20224C6802FA03F317
:108190001C4214D15DF8044B704720220C6802FA8F
:1081A00003F31C42F6D00C4A4068002414700268A5
:1081B0005DF8044B22F0010202608B607047064AB2
:1081C00040680024147002685DF8044B22F001023C
:1081D0000260CB60704700BFD55E0020F0B58769B4
:1081E00083B0064617B13B68BA885A837069DFF8D6
:1081F000A4E08389C3244FF47A734FF0060C6D46D4
:108200004FF6FF710EF1010E03E0013B9BB28B4272
:1082100020D002899207F8D5A3B283814FF47A73F4
:1082200002E0A3B28B4215D00289D20703F1FF34DA
:10823000F7D5828992B20DB12A700135BCF1000FD9
:108240000BD00CF1FF3CFF24BEF1000FE1D09EF8F3
:108250000040D7E70FF01AFDB76917B13B68BA883D
:108260001A839DF805009DF801509DF802109DF8B5
:1082700003409DF804209DF8063041EA052143EAB9
:10828000002342EA0422012031877287B38703B0BA
:10829000F0BD00BFB0480408F8B5057B4669036827
:1082A0001F2D29D9A5F120045F682021A1400F428C
:1082B0002A4613D01022A240D960DA605A68E24000
:1082C000D10703D5012202FA04F4DC6004463046EB
:1082D00005F042FA227B23681F2A20D9A2F1200050
:1082E00008215A688140114200D0D960042259689F
:1082F00082400A4221D1F8BD20211C68A9400C42CD
:108300002A460CD01022AA4099609A601A68EA4066
:10831000D207DBD5012202FA05F59D60D6E70821D8
:1083200018689140014200D099600421186801FA50
:1083300002F2024203D09A60F8BDDA60F8BDF8BDDF
:10834000144B984224D003F58063984220D00288D1
:1083500022F040021204120C0280028822F038033C
:108360001B041B0C59B141F48071002991FAA1F250
:10837000B2FA82F108BF4FF0FF310139C9000B4357
:108380009BB2038003889BB243F040030380704795
:108390004908DCE700380040A849A948A94A2DE966
:1083A000F84F012303700B88128823F040031B044D
:1083B0001B0C0B800B8823F038031B0452084FEA78
:1083C00013430BD042F48072002A92FAA2F1B1FA60
:1083D00081F208BF4FF0FF32013AD2001343974AAF
:1083E0009BB2138013889BB243F040031380964BDB
:1083F0001B6813B11A689B885383904940F2E93394
:1084000002E0002B00F09E810A89013B12F0020F6E
:108410009BB2F6D005238B8140F2E933874902E015
:10842000002B00F08F810A89013B12F0010F9BB2F3
:10843000F6D08B89814940F2E93302E0002B00F04D
:10844000A5810A89013B12F0020F9BB2F6D00023EE
:108450008B8140F2E933794902E0002B00F09681EC
:108460000A89013B12F0010F9BB2F6D08B89734948
:1084700040F2E93302E0002B00F084810A89013BDD
:1084800012F0020F9BB2F6D006238B8140F2E93343
:108490006A4902E0002B00F075810A89013B12F065
:1084A000010F9BB2F6D08B89644940F2E93302E0B8
:1084B000002B00F063810A89013B12F0020F9BB28E
:1084C000F6D000238B8140F2E9335C4902E0002BB7
:1084D00000F054810A89013B12F0010F9BB2F6D0E3
:1084E0008B89DFF86CA155499AF8004040F2E933D6
:1084F00044F0010402E0002B00F03C810A89013BBA
:1085000012F0020F9BB2F6D004238B8140F2E933C4
:108510004A4902E0002B00F02D810A89013B12F04C
:10852000010F9BB2F6D08B89444940F2E93302E057
:10853000002B00F01B810A89013B12F0020F9BB255
:10854000F6D0A4B28C8140F2E9333C4902E0002B22
:1085500000F00C810A89013B12F0010F9BB2F6D0AA
:108560008B893A4F3B88002B47D0DFF8E890DFF843
:10857000E880324C4FF0000B072699F8015040F28A
:10858000E93302E0002B00F0D5802089013B10F098
:10859000020F9BB2F6D0A68140F2E93302E0002B35
:1085A00000F0C8802089013B10F0010F9BB2F6D08B
:1085B000A38940F2E93302E0002B00F0BF8020895C
:1085C000013B10F0020F9BB2F6D0ADB2A58140F294
:1085D000E93302E0002B00F0B1802089013B10F06C
:1085E000010F9BB2F6D0A3893B8819F8010F08F858
:1085F000010F0BF1010B9B45BFDB104840F2E93343
:1086000002E0002B00F0AE800289013B12F0020F65
:108610009BB2F6D007238381084940F2E93302E098
:10862000002B00F09F800A89013B12F0010F9BB2E2
:10863000F6D08B89014840F2E93311E0003C00405C
:10864000FF530020E41D0020D88D002024010020CD
:1086500090240020EF51002093240020002B7DD097
:108660000289013B12F0020F9BB2F7D0FF238381F6
:10867000484940F2E93301E0002B6FD00A89013B01
:1086800012F0010F9BB2F7D08B899AF80040414855
:1086900040F2E93301E0002B5CD00289013B12F08B
:1086A000020F9BB2F7D0042383813A4940F2E933A9
:1086B00001E0002B4ED00A89013B12F0010F9BB262
:1086C000F7D08B89334840F2E93301E0002B3DD0ED
:1086D0000289013B12F0020F9BB2F7D0A4B22D49E0
:1086E000848140F2E93301E0002B2FD00A89013B5D
:1086F00012F0010F9BB2F7D08B89274B1B6813B187
:108700001A689B881383234A138823F040031B04B1
:108710001B0C1380138823F038031B041B0C1380DD
:1087200013889BB243F0400313801C4B0021197047
:10873000BDE8F88F20460FF0A9FA3AE720460FF07F
:10874000A5FA51E713480FF0A1FA73E611480FF0AC
:108750009DFAD2E70F480FF099FAB3E70D480FF0F2
:1087600095FA92E70B480FF091FA63E709480FF08A
:108770008DFAF6E607480FF089FAD5E605480FF0BE
:1087800085FAAEE603480FF081FA8DE601480FF056
:108790007DFA6CE6003C0040D88D0020FF5300209D
:1087A00008B540F2E93300E0A3B10289013B12F0C1
:1087B000020F9BB2F8D089B2818140F2E93300E028
:1087C00043B10289013B12F0010F9BB2F8D08089BE
:1087D000C0B208BD0FF05AFAC0B208BD38B50446A1
:1087E0000D4600BF80680FF001F929466068FFF769
:1087F000D7FFA0680FF0FFF800BF38BDA6490A8870
:1088000022F040022DE9F0471204A44F120C3B88DD
:108810000A800A8822F0380212045B084FEA1242EA
:1088200000F0388143F4807090FAA0F10028B1FA8A
:1088300081F108BF4FF0FF310139C9000A43964961
:10884000974D92B20A800A8892B242F040020A80A2
:10885000296811B10A6888885083924A1278012ADF
:1088600000F04981C0F03081022A40F0FF808E4E36
:10887000082232704FF4C372DFF848828648A8F8A5
:108880000020028822F040021204120C02800288AA
:1088900022F038021204120C5BB143F4807090FA9B
:1088A000A0F30028B3FA83F308BF4FF0FF33013B76
:1088B000DB001343784A9BB2138013889BB243F0CA
:1088C0004003138011B10B688A885A83724C4FF0B1
:1088D00010094FF0010A40F2E93302E0002B00F0EA
:1088E000CF802289013B12F0020F9BB2F6D01FFA13
:1088F00089F3A38140F2E93302E0002B00F0C0804D
:108900002289013B12F0010F9BB2F6D0A38940F2FD
:10891000E93302E0002B00F0B7802289013B12F01E
:10892000020F9BB2F6D0A4F80CA040F2E93302E0AB
:10893000002B00F0A9802289013B12F0010F9BB2AD
:10894000F6D0A38909F10109B9F1200FC3D1296833
:1089500011B10B688A881A834F4B1A8822F04002A3
:108960001204120C1A801A8822F038021204120C17
:108970001A801A8892B242F040021A8018883A8807
:1089800020F040000004000C18801B8823F03803FE
:108990001B0452084FEA13430BD042F48072002AA2
:1089A00092FAA2F0B0FA80F208BF4FF0FF32013A1B
:1089B000D2001343384A9BB2138013889BB243F012
:1089C0004003138011B10B688A885A833478324887
:1089D0000021FFF7E5FE21462F48FFF7E1FE334B6C
:1089E0002D481C780221FFF7DBFE21462A48FFF7BD
:1089F000D7FE2F4B28481C780321FFF7D1FE2146D4
:108A00002548FFF7CDFE2B4B23481C7804210C434F
:108A1000FFF7C6FE21462048FFF7C2FE2B6813B1C0
:108A20001A689B8813831C4A234C1388234823F01D
:108A300040031B041B0C1380138823F038031B0412
:108A40001B0C138013889BB243F040031380B8F8CB
:108A5000002000213BF0BDFE2378CBB1184B1B78E2
:108A6000002B4ED000232370BDE8F0870E4E3278E5
:108A700012F0400F0CBF4FF4C3724FF4F072FBE6DC
:108A800020460FF003F942E720460FF0FFF859E7C0
:108A9000BDE8F0871946D1E6003C0040E41D002007
:108AA000D88D0020EC8D002004030020F38D0020E1
:108AB000F48D002090240020000000209424002049
:108AC000FF53002024010020A0211448FFF768FE76
:108AD00000211248FFF764FE00F00603022B03D0CA
:108AE00000F00500012812D00D4E3B8829680822AD
:108AF00032705B08BEE60A4E482232704FF4F072C4
:108B0000BAE6FFF749FC00232370BDE8F087044E66
:108B10003B882968482232705B08EFE7003C004040
:108B2000040300202DE9F04F85B0019090F8550026
:108B3000002840F07185019B1B7C022B00F0AE8564
:108B4000BB4CBC4DDFF8F492BB48DFF8F4E24FF0C9
:108B5000640A4FF0100C4FF47A76D9F80430C3F35E
:108B60000803002B40F05684EFF31183002B40F0F4
:108B700051842168826800BF23689942F9D12F6827
:108B800006FB07F39B1AB3FBF7F306FB0131012742
:108B90000091D9F80430C3F30803002B40F000849F
:108BA000EFF31183002B40F0FB832368816800BF43
:108BB00022689342F9D1D5F800B006FB0BF2521AA5
:108BC000B2FBFBF206FB0323009A9B1AB3F57A7FF4
:108BD000DFD3BAF1010AC0D1019B1B7C022B00F04C
:108BE0003586DFF858929448DFF854E24FF0640A73
:108BF0004FF0100C4FF47A76D9F80430C3F3080321
:108C0000002B40F0EB83EFF31183002B40F0E68361
:108C10002168826800BF23689942F9D12F6806FB5A
:108C200007F39B1AB3FBF7F306FB01310127009111
:108C3000D9F80430C3F30803002B40F09483EFF31A
:108C40001183002B40F08F832368816800BF226866
:108C50009342F9D1D5F800B006FB0BF2521AB2FBE1
:108C6000FBF206FB0323009A9B1AB3F57A7FDFD34E
:108C7000BAF1010AC0D1019B1B7C022B00F0CE850A
:108C8000DFF8B8916C48DFF8B8E14FF0640A4FF0B4
:108C9000100C4FF47A76D9F80430C3F30803002B94
:108CA00040F06484EFF31183002B40F05F8421686F
:108CB000826800BF23689942F9D12F6806FB07F349
:108CC0009B1AB3FBF7F306FB013101270091D9F89A
:108CD0000430C3F30803002B40F02883EFF3118323
:108CE000002B40F023832368816800BF22689342F1
:108CF000F9D1D5F800B006FB0BF2521AB2FBFBF229
:108D000006FB0323009A9B1AB3F57A7FDFD3BAF1EF
:108D1000010AC0D1019B1B7C022B00F06785DFF8A4
:108D20001C914548DFF818E14FF00F0A4FF0100C86
:108D30004FF47A76D9F80430C3F30803002B40F0DF
:108D4000F883EFF31183002B40F0F38321688268EE
:108D500000BF23689942F9D12F6806FB07F39B1ADD
:108D6000B3FBF7F306FB013101270091D9F804307A
:108D7000C3F30803002B40F0BC82EFF31183002BF8
:108D800040F0B7822368816800BF22689342F9D11E
:108D9000D5F800B006FB0BF2521AB2FBFBF206FB51
:108DA0000323009A9B1AB3F57A7FDFD3BAF1010A45
:108DB000C0D1019991F84F200B7C032A8CBF1A2651
:108DC0001826022B00F0FB84DFF870901A48DFF8B9
:108DD00070E04FF00F0A4FF0100C4FF47A76D9F88C
:108DE0000430C3F30803002B40F0F983EFF3118341
:108DF000002B40F0F4832168826800BF2368994209
:108E0000F9D12F6806FB07F39B1AB3FBF7F306FBB8
:108E1000013101270091D9F80430C3F30803002B76
:108E200040F04A82EFF31183002B40F0458209E0C5
:108E300058AA00205CAA002010E000E000ED00E04D
:108E400054AA00202368816800BF22689342F9D1A8
:108E5000D5F800B006FB0BF2521AB2FBFBF206FB90
:108E60000323009A9B1AB3F57A7FD4D3BAF1010A8F
:108E7000B5D1019B1B7C022B00F08984DFF8DC92CA
:108E8000B448DFF8D4E24FF00F0A4FF0100C4FF463
:108E90007A76D9F80430C3F30803002B40F08383BB
:108EA000EFF31183002B40F07E832168826800BFBE
:108EB00023689942F9D12F6806FB07F39B1AB3FB8D
:108EC000F7F306FB013101270091D9F80430C3F311
:108ED0000803002B40F0D381EFF31183002B40F007
:108EE000CE812368816800BF22689342F9D1D5F80A
:108EF00000B006FB0BF2521AB2FBFBF206FB032397
:108F0000009A9B1AB3F57A7FDFD3BAF1010AC0D178
:108F1000019B1B7C022B00F02084DFF840928D48DF
:108F2000DFF834E24FF00F0A4FF0100C4FF47A766E
:108F3000D9F80430C3F30803002B40F0A482EFF308
:108F40001183002B40F09F822168826800BF236854
:108F50009942F9D12F6806FB07F39B1AB3FBF7F38D
:108F600006FB013101270091D9F80430C3F308034F
:108F7000002B40F06781EFF31183002B40F06281FA
:108F80002368816800BF22689342F9D1D5F800B008
:108F900006FB0BF2521AB2FBFBF206FB0323009A0C
:108FA0009B1AB3F57A7FDFD3BAF1010AC0D1019BD6
:108FB0001B7C022B00F0B883DFF8A0916548DFF836
:108FC00098E14FF0640A4FF0100C4FF47A76D9F81C
:108FD0000430C3F30803002B40F03982EFF3118310
:108FE000002B40F034822168826800BF23689942D8
:108FF000F9D12F6806FB07F39B1AB3FBF7F306FBC7
:10900000013101270091D9F80430C3F30803002B84
:1090100040F0FB80EFF31183002B40F0F6802368D3
:10902000816800BF22689342F9D1D5F800B006FBF1
:109030000BF2521AB2FBFBF206FB0323009A9B1AB7
:10904000B3F57A7FDFD3BAF1010AC0D1019B1B7C53
:10905000022B00F05283DFF804913E48DFF8F8E07D
:109060004FF00F0A4FF0100C4FF47A76D9F8043015
:10907000C3F30803002B40F04082EFF31183002B71
:1090800040F03B822168826800BF23689942F9D191
:109090002F6806FB07F39B1AB3FBF7F306FB0131BE
:1090A00001270091D9F80430C3F30803002B40F0E6
:1090B0008F80EFF31183002B40F08A802368816852
:1090C00000BF22689342F9D1D5F800B006FB0BF23D
:1090D000521AB2FBFBF206FB0323009A9B1AB3F56C
:1090E0007A7FDFD3BAF1010AC0D1019B1B7C022B2E
:1090F00000F0EC82DFF864801649174F4FF00F093B
:109100004FF0100E4FF47A70D8F80430C3F3080310
:10911000002B40F0D481EFF31183002B40F0CF817E
:1091200022688E6800BF23689A42F9D1D5F800C042
:1091300000FB0CF39B1BB3FBFCF300FB023300931F
:109140000126D8F80430C3F308032BBBEFF31183D7
:1091500013BB05E010E000E054AA002000ED00E0A1
:109160002368D1F808A000BF22689342F8D1D5F84F
:1091700000B000FB0BFCACEB0A0CBCFBFBFC00FBE7
:1091800003C3009A9B1AB3F57A7FDAD3B9F10109C8
:10919000BAD105B0BDE8F08FEFF3118A8EF31288D3
:1091A0008A680B68DB0344BF3E608A682368D7F88F
:1091B00000C05FFA8AFA8AF31188D5F800A09C44AF
:1091C00000FB0AF39B1AB3FBFAF300FB0C33D8E75E
:1091D000EFF311888CF3128881680368DB0344BFC6
:1091E000CEF8007081682368DEF800205FFA88F806
:1091F00088F31188D5F800801A4406FB08F35B1A3F
:10920000B3FBF8F306FB023367E7EFF311888CF347
:10921000128881680368DB0344BFCEF80070816860
:109220002368DEF800205FFA88F888F31188D5F803
:1092300000801A4406FB08F35B1AB3FBF8F306FB45
:109240000233FBE6EFF311888CF312888168036820
:10925000DB0344BFCEF8007081682368DEF800208D
:109260005FFA88F888F31188D5F800801A4406FB65
:1092700008F35B1AB3FBF8F306FB02338FE6EFF358
:1092800011888CF3128881680368DB0344BFCEF831
:10929000007081682368DEF800205FFA88F888F3A0
:1092A0001188D5F800801A4406FB08F35B1AB3FB5B
:1092B000F8F306FB023323E6EFF311888CF31288F0
:1092C00081680368DB0344BFCEF8007081682368BF
:1092D000DEF800205FFA88F888F31188D5F800805E
:1092E0001A4406FB08F35B1AB3FBF8F306FB0233E0
:1092F000B7E5EFF311888CF3128881680368DB030C
:1093000044BFCEF8007081682368DEF800205FFA61
:1093100088F888F31188D5F800801A4406FB08F312
:109320005B1AB3FBF8F306FB02333AE5EFF311885F
:109330008CF3128881680368DB0344BFCEF80070A9
:1093400081682368DEF800205FFA88F888F31188C6
:10935000D5F800801A4406FB08F35B1AB3FBF8F358
:1093600006FB0233CEE4EFF311888CF31288816898
:109370000368DB0344BFCEF8007081682368DEF821
:1093800000205FFA88F888F31188D5F800801A4425
:1093900006FB08F35B1AB3FBF8F306FB023362E447
:1093A000EFF311888CF3128881680368DB0344BFF4
:1093B000CEF8007081682368DEF800205FFA88F834
:1093C00088F31188D5F800801A4406FB08F35B1A6D
:1093D000B3FBF8F306FB0233FFF7F6BBEFF31182A2
:1093E0008CF3128887680368D90303D50123CEF86C
:1093F000003087682368DEF80010D2B282F311884B
:109400002A68194406FB02F3DB1BB3FBF2F306FBED
:1094100001310BE4EFF311828CF312888768036843
:10942000D90303D50123CEF8003087682368DEF81E
:109430000010D2B282F311882A68194406FB02F3A5
:10944000DB1BB3FBF2F306FB0131FFF7A0BBEFF32D
:1094500011828CF3128887680368D90303D501232E
:10946000CEF8003087682368DEF80010D2B282F3AD
:1094700011882A68194406FB02F3DB1BB3FBF2F3E5
:1094800006FB0131BDE5EFF311828CF3128887688A
:109490000368D90303D50123CEF800308768236819
:1094A000DEF80010D2B282F311882A68194406FB54
:1094B00002F3DB1BB3FBF2F306FB013152E5EFF3E2
:1094C00011868EF31288D1F808C00B68DA0303D531
:1094D00001233B60D1F808C023683A68F6B286F3EE
:1094E00011882E681A4400FB06F3A3EB0C03B3FBB0
:1094F000F6F300FB0233009322E6EFF311828CF3C4
:10950000128887680368D90303D50123CEF8003099
:1095100087682368DEF80010D2B282F311882A68C7
:10952000194406FB02F3DB1BB3FBF2F306FB01312C
:10953000B6E5EFF311828CF3128887680368D903CC
:1095400003D50123CEF8003087682368DEF80010C9
:10955000D2B282F311882A68194406FB02F3DB1B9E
:10956000B3FBF2F306FB0131FFF7FEBBEFF3118211
:109570008CF3128887680368D90303D50123CEF8DA
:10958000003087682368DEF80010D2B282F31188B9
:109590002A68194406FB02F3DB1BB3FBF2F306FB5C
:1095A0000131FFF792BBEFF311828CF312888768C9
:1095B0000368D90303D50123CEF8003087682368F8
:1095C000DEF80010D2B282F311882A68194406FB33
:1095D00002F3DB1BB3FBF2F306FB013173E4EFF3A1
:1095E00011828CF3128887680368D90303D501239D
:1095F000CEF8003087682368DEF80010D2B282F31C
:1096000011882A68194406FB02F3DB1BB3FBF2F353
:1096100006FB0131FFF7FDBB0DF09EFF044600285D
:1096200000F0318100689E4900F13F4303F57E035D
:109630009A0A20258A5CA57102F01F0652090123AF
:109640000021032A03FA06F3E17100F03181042AB4
:1096500000F02181022A00F01181A388029302A95F
:10966000002303932DF0C8F901998E4B41F80C3F6C
:10967000204635F0D5FFA388B3FA83F3C3F11F0367
:10968000012212FA03F33FF456AA87490A681343EA
:109690000B60019B1B7C022B7FF452AA019B9B69F0
:1096A00013B11A689B885383019C6B216069FFF793
:1096B00077F880216069FFF773F8A369002B3FF406
:1096C0003FAA1A689B881383FFF73ABA019B9B69EC
:1096D00013B11A689B885383019E38217069FFF784
:1096E0005FF801217069FFF75BF8B369002B3FF465
:1096F00001AD1A689B881383FCE4019B9B6913B13D
:109700001A689B885383019E37217069FFF748F8D8
:1097100010217069FFF744F8B369002B3FF49BAC4C
:109720001A689B88138396E4019A936992F85060B3
:1097300013B11A689B885383019F19217869FFF739
:109740002FF831467869FFF72BF8BB69002B3FF4FF
:1097500033AC1A689B8813832EE4019A936992F8BC
:109760004E6013B11A689B885383019F1A21786950
:10977000FFF716F831467869FFF712F8BB69002B3E
:109780003FF4CBAB1A689B881383FFF7C6BB019BE2
:109790009B6913B11A689B885383019E1C217069D1
:1097A000FEF7FEFF18217069FEF7FAFFB369002B80
:1097B0003FF464AB1A689B881383FFF75FBB8B6928
:1097C00013B11A689B885383019F1B217869FEF7A8
:1097D000E7FF31467869FEF7E3FFBB69002B3FF4F2
:1097E000F3AA1A689B881383FFF7EEBA019B9B6963
:1097F00013B11A689B885383019E6B217069FEF731
:10980000CFFF01217069FEF7CBFFB369002B3FF456
:1098100086AA1A689B881383FFF781BA019B9B690C
:1098200013B11A689B885383019E6B217069FEF700
:10983000B7FF00217069FEF7B3FFB369002B3FF457
:109840001FAA1A689B881383FFF71ABA019B9B69AA
:1098500013B11A689B885383019E68217069FEF7D3
:109860009FFF07217069FEF79BFFB369002B3FF450
:10987000B8A91A689B881383FFF7B3B90B4A516CD8
:109880000B435364E9E60199064B41F80C3F35F070
:10989000C7FEFFF750B9054A116B0B431363DCE6B3
:1098A0000075040819800008003C0140003802409F
:1098B000024A116C0B431364CFE600BF003802402C
:1098C0002DE9F04FAC4A436983B09342019000F018
:1098D000A281AA498B420CBF282130211A88A84CAA
:1098E000DFF8A882A74E22F040021204120C1A8060
:1098F0001A8892B222F03802114319801A8892B263
:1099000042F040021A8003F05DFCDFF884E29E49D9
:10991000844610274FF47A750120DEF80430C3F333
:109920000803002B40F03681EFF31183002B40F049
:1099300031812368D1F8089000BF22689342F8D1A2
:10994000D8F800A005FB0AF2A2EB0902B2FBFAF27A
:1099500005FB03239C45E0D0019D2846FFF7E2F874
:10996000AB6913B11A689B885383019B586940F215
:10997000E93302E0002B00F046810289013B12F03E
:10998000020F9BB2F6D06A23838140F2E93302E0F2
:10999000002B00F038810289013B12F0010F9BB2CD
:1099A000F6D0838940F2E93302E0002B00F03081E9
:1099B0000289013B12F0020F9BB2F6D01023838183
:1099C00040F2E93302E0002B00F022810289013BE2
:1099D00012F0010F9BB2F6D08389019B9B6913B1F2
:1099E0001A689B881383DFF8A8916748654F4FF08A
:1099F000640A4FF0100E4FF47A75D9F80430C3F3AF
:109A00000803002B40F0E480EFF31183002B40F0BB
:109A1000DF802168826800BF23689942F9D1D8F8B5
:109A2000006005FB06F39B1AB3FBF6F305FB01315F
:109A300001260091D9F80430C3F30803002B63D149
:109A4000EFF31183002B5FD12368816800BF226888
:109A50009342F9D1D8F800B005FB0BF2521AB2FBD1
:109A6000FBF205FB0323009A9B1AB3F57A7FE1D33F
:109A7000BAF1010AC1D1019B3F4A5B69934207D009
:109A8000DFF8F8A0534514BF4FF0080A4FF0000A62
:109A90001A883D4D3B4F22F040021204120C1A80EE
:109AA0001A8892B222F038024AEA020AA3F800A009
:109AB0001A8892B242F040021A8003F083FBDFF86A
:109AC000D0C081464FF0100E4FF47A760120DCF8BA
:109AD0000430C3F30803002B31D1EFF3118373BBC0
:109AE0002368A96800BF22689342F9D1D8F800A082
:109AF00006FB0AF2521AB2FBFAF206FB032399455F
:109B0000E5D003B0BDE8F08FEFF3118C8EF312882F
:109B100081680368DA0344BF3E60816823683A685D
:109B20005FFA8CFC8CF31188D8F800C01A4405FB4E
:109B30000CF35B1AB3FBFCF305FB023393E7EFF383
:109B400011818EF31288D5F808A02B68DB0344BF7F
:109B50003860D5F808A023683A68C9B281F3118843
:109B6000D8F800101A4406FB01F3A3EB0A03B3FB79
:109B7000F1F306FB0233C2E700380040003C00402E
:109B800058AA002054AA002010E000E05CAA00209F
:109B900000ED00E0EFF3118987F31288D1F808A0F7
:109BA0000B68DB0344BF3060D1F808A0236832683B
:109BB0005FFA89F989F31188D8F800901A4405FBF7
:109BC00009F3A3EB0A03B3FBF9F305FB0233C1E688
:109BD000EFF311828EF3128886680368D90302D5E9
:109BE00001233B60866823683968D2B282F311880A
:109BF000D8F80020194405FB02F39B1BB3FBF2F3DA
:109C000005FB013114E70EF041F8019B5869C9E6E4
:109C10000EF03CF8E1E6282160E600BF2DE9F84FA0
:109C2000A94F3B7803B1FEE7A84CA94A01233B703A
:109C30002388128823F040031B041B0C23802388F5
:109C400023F038031B0452084FEA13430BD042F4AD
:109C50008072002A92FAA2F4B4FA84F208BF4FF09C
:109C6000FF32013AD2001343984ADFF870829BB268
:109C7000138013889BB243F040031380D8F8003060
:109C800013B11A689B885383924B01220D461A70B8
:109C900004468E4940F2E93302E0002B00F0A38134
:109CA0000A89013B12F0020F9BB2F6D000238B8190
:109CB00040F2E933854902E0002B00F094810A89E3
:109CC000013B12F0010F9BB2F6D08B897F4940F225
:109CD000E93302E0002B00F09A810A89013B12F07F
:109CE000020F9BB2F6D000238B8140F2E933774913
:109CF00002E0002B00F08B810A89013B12F0010F7A
:109D00009BB2F6D08B89714940F2E93302E0002B17
:109D100000F079810A89013B12F0020F9BB2F6D064
:109D200009238B8140F2E933684902E0002B00F0FF
:109D30006A810A89013B12F0010F9BB2F6D08B8930
:109D4000624940F2E93302E0002B00F058810A89B1
:109D5000013B12F0020F9BB2F6D0A4B28C8140F20C
:109D6000E9335A4902E0002B00F049810A89013B9E
:109D700012F0010F9BB2F6D08B89574E534C013D28
:109D80004FF0000A4FF00A0B40F2E93302E0002BDB
:109D900000F010812289013B12F0020F9BB2F6D035
:109DA000A4F80CB040F2E93302E0002B00F002818D
:109DB0002289013B12F0010F9BB2F6D0A38940F239
:109DC000E93302E0002B00F0F9802289013B12F018
:109DD000020F9BB2F6D01FFA8AF3A38140F2E93357
:109DE00002E0002B00F0EA802289013B12F0010F13
:109DF0009BB2F6D0A38915F8019F40F2E93302E047
:109E0000002B00F0DF802289013B12F0020F9BB291
:109E1000F6D00B23A38140F2E93302E0002B00F0DF
:109E2000D1802289013B12F0010F9BB2F6D0A389A9
:109E300040F2E93302E0002B00F0C8802289013BA8
:109E400012F0020F9BB2F6D01FFA89F9A4F80C9019
:109E500040F2E93302E0002B00F0B8802289013B98
:109E600012F0010F9BB2F6D0A389336833B11A68A0
:109E70009B8851690B4214BF538313830AF1010A73
:109E8000BAF1360F80D140F2E933104802E0002BDE
:109E900000F0B1800289013B12F0020F9BB2F6D0B4
:109EA00008238381094940F2E93302E0002B00F0E6
:109EB000A2800A89013B12F0010F9BB2F6D08B8978
:109EC000024840F2E9330EE0FF530020003C00401E
:109ED000E41D00200554002024AA0020D88D002075
:109EE000002B00F084800289013B12F0020F9BB22C
:109EF000F6D0A0238381484940F2E93301E0002BEA
:109F000075D00A89013B12F0010F9BB2F7D08B8903
:109F1000414CA02540F2E93301E0002B5AD02289C0
:109F2000013B12F0020F9BB2F7D0A58140F2E9335A
:109F300001E0002B4ED02289013B12F0010F9BB2B1
:109F4000F7D0A38940F2E93301E0002B46D0228903
:109F5000013B12F0020F9BB2F7D00023A38140F225
:109F6000E93301E0002B39D02289013B12F0010FC7
:109F70009BB2F7D0A089C0B28306CBD4D8F800300A
:109F800013B11A689B881383234A138823F0400374
:109F90001B041B0C1380138823F038031B041B0CB9
:109FA000138013889BB243F0400300211380397063
:109FB000BDE8F88F20460DF069FE00E720460DF061
:109FC00065FE18E720460DF061FE31E720460DF0F2
:109FD0005DFE4AE720460DF059FEB3E720460DF03E
:109FE00055FEC0B2C8E70C480DF050FE6EE60A48B8
:109FF0000DF04CFE8CE708480DF048FE60E706487F
:10A000000DF044FEB9E604480DF040FE98E6024823
:10A010000DF03CFE77E600BF003C004030B4147801
:10A0200074B11E23074D13FB01012944801A8318C4
:10A030001D2BD8BF0C7012F8014F0131002CF6D146
:10A0400030BC7047F0510020F8B5434C434A238898
:10A05000128823F040031B041B0C23802388C1F1CA
:10A06000030123F0380341EA80071B045208FFB2C2
:10A070004FEA13430BD042F48072002A92FAA2F105
:10A08000B1FA81F208BF4FF0FF32013AD200134318
:10A09000314A334D9BB2138013889BB243F0400387
:10A0A00013802B6813B11A689B8853832A4CBFB264
:10A0B000102640F2E93301E0002B45D02289013B14
:10A0C00012F0020F9BB2F7D0B3B2A38140F2E93392
:10A0D00001E0002B38D02289013B12F0010F9BB226
:10A0E000F7D0A38940F2E93301E0002B30D0228978
:10A0F000013B12F0020F9BB2F7D0A78140F2E93387
:10A1000000E02BB32289013B12F0010F9BB2F8D083
:10A11000A3890136202ECCD12B6813B11A689B88F5
:10A1200013830D4A138823F040031B041B0C138078
:10A13000138823F038031B041B0C138013889BB275
:10A1400043F040031380F8BD20460DF09FFDC9E7A2
:10A1500020460DF09BFDDCE7003C0040E41D0020A4
:10A16000D88D002038B5454B1D7800287BD105F0EF
:10A17000F70543491D700B88424A23F040031B0436
:10A180001B0C12880B800B8823F038031B04520829
:10A190004FEA13430BD042F48072002A92FAA2F1E4
:10A1A000B1FA81F208BF4FF0FF32013AD2001343F7
:10A1B000334A354C9BB2138013889BB243F0400363
:10A1C0001380236813B11A689B88538340F2E933E4
:10A1D0002B4901E0002B49D00A89013B12F0020F04
:10A1E0009BB2F7D004238B8140F2E933244901E08C
:10A1F000002B3BD00A89013B12F0010F9BB2F7D034
:10A200008B891F4940F2E93301E0002B32D00A89E3
:10A21000013B12F0020F9BB2F7D0ADB28D8140F23C
:10A22000E933174900E02BB30A89013B12F0010F13
:10A230009BB2F8D08B89236813B11A689B8813836B
:10A240000F4A138823F040031B041B0C1380138850
:10A2500023F038031B041B0C138013889BB243F0BC
:10A260004003138038BD45F0080582E704480DF02F
:10A270000DFDC6E702480DF009FDDCE79024002043
:10A28000003C0040E41D0020D88D00200C4B98427B
:10A2900013D0A3F5806398420FD003F58043984212
:10A2A0000BD003F58063984207D003F58063984292
:10A2B00003D0044B186840087047024B1868704779
:10A2C0000004014020740020F0B5774B774A87B036
:10A2D0001968914200AF00F0DB800023744A3B60B4
:10A2E0007B60136843F48033136003E03B68B3F58D
:10A2F000A04F09D0136803F400337B603B6801333F
:10A300003B607B68002BF1D0694B1B6813F4003372
:10A3100018BF01237B607B68012B7BD0654D644BAC
:10A32000654AEA606549586F654A0860AA605E6BD5
:10A33000644C654A654826F080065E635E6F46F0B1
:10A3400080765E67196B0C431C63596B5963996B7C
:10A350009963196C41F05B5141F47B1141F41F6129
:10A3600041F00F011964596C07F118040A4348F2CF
:10A37000FF715A6444F8101D002621460123FB7327
:10A380003E737E73BE732CF037FB21464FF6FF738E
:10A390004F48BB602CF030FB4FF6FF7321464D4811
:10A3A000BB602CF029FB21464B482CF025FB2146B5
:10A3B0004A482CF021FB214649482CF01DFB214640
:10A3C00048482CF019FB214647482CF015FB214644
:10A3D00046482CF011FB20462CF0CCF8444B454C61
:10A3E0001B68BA6844484549A4FB03439B09A0FB8A
:10A3F0000202013B920CB3F1807F0A6007D2404A0F
:10A40000F0200721536085F82300966011601C3707
:10A41000BD46F0BD264B3B4C1A6C3B4942F0805286
:10A420001A6420688A684D68C96840F4404020601A
:10A43000986898609868120640F40040986042EA74
:10A440008512986842F48002490842F008020139F6
:10A4500042EA014240F4A05098605A601A6842F003
:10A4600080721A601A689201FCD52849104A40F29D
:10A4700005700860996821F003019960996841F0BE
:10A4800002019960936803F00C03082BFAD145E7A9
:10A4900000221A6062B61E4B1B6883F308881D4BAE
:10A4A0001B689847FEE700BFFCFF0120EFBEADDE52
:10A4B0000038024000ED00E00005FA0530AD002054
:10A4C00000000008FF916700335F070000000240B2
:10A4D0000004024000080240000C0240001002404C
:10A4E0000014024000180240001C024000200240FC
:10A4F00020740020D34D621083DE1B435CAA002031
:10A5000010E000E00070004000000020003C02402D
:10A510000000FF1F0400FF1F08B5054B1B6803B1B7
:10A520009847044B044A1A6072B6FDF779FD00BFE4
:10A53000A85A0020FCFF0120EFBEADDE08B5034B9A
:10A540001B6803B1984772B6FDF76AFDA85A002050
:10A55000084B10B507281B68C8BF143818440C46B0
:10A56000807D0CF0F9FF20B12146BDE810400DF0D0
:10A5700047BA10BDAC46002038B50C4B07281B6805
:10A58000CCBFA0F11404044623440546987D0CF08A
:10A59000E3FF50B128220134C471827134F0DCFF32
:10A5A00028460021BDE83840D2E738BDAC4600203F
:10A5B000064A00235168814202F11C0204D0013393
:10A5C000102BF7D100207047D8B27047801B0020B5
:10A5D00070B50F4C0F4DC0EBC00004EB8004286B2E
:10A5E00026693043286382B09209667BA16000250A
:10A5F000012101A863618DF804608DF805208DF8B4
:10A6000006508DF807102BF06DFF02B070BD00BF33
:10A61000801B002000380240074BC0EBC00030B464
:10A6200003EB8000054C0569236B2B432363017604
:10A63000427630BC704700BF801B002000380240CB
:10A640002DE9F04F534C54F8204083B0002C00F01B
:10A650009C80256E002D00F09A8017464E4A984641
:10A66000064604F166032869226004F266226361EB
:10A67000A2614FF400736A68A160E3602361A26580
:10A68000A24668B1FFF794FF721CD2B20C21FFF70B
:10A69000C3FFA36DA9682A6962630433E16363653C
:10A6A000E868A0B1FFF784FF721C8146D2B20B218B
:10A6B000FFF7B2FF2346EA7F38494846FFF788FF95
:10A6C000A36DA968EA68A26304332164236594F842
:10A6D00065000CF041FF814694F864000CF03CFFEB
:10A6E0008346287F00284DD118F0080F36D1BA07CD
:10A6F0000DD5B9F1000F0AD00B22731C89F8062082
:10A7000089F8073048466A7F22210CF0EBFFFB07EF
:10A7100015D4E36B7BB995F82020A97F8DF806301E
:10A7200001A8930901228DF805308DF804108DF8E9
:10A7300007202BF0D7FE504603B0BDE8F08FBBF1E9
:10A74000000FE6D001360C238BF807608BF806303B
:10A7500058466A7F22210CF0C5FFDAE70136F6B2CF
:10A76000B9F1000F04D00B2389F8076089F806308F
:10A7700018F0100F484614BF022112216A7F0CF016
:10A78000B1FFC6E734F0CAFEAEE7A246D3E7AA4659
:10A79000D1E700BF8C460020B84804089982000821
:10A7A00000B97047F0B599B0064635F089F9814D8A
:10A7B000C36802682A600446002B00F0DF80304640
:10A7C0000CF0CAFE7C4BC3F8E40118B12922002327
:10A7D0008271C371227A2A210CF084FF286802F06A
:10A7E0006BFB34F09BFE2E68338823F001031B04BF
:10A7F0001B0C33803046FFF749FD704A90420346F8
:10A8000000F2BE80002218A9DFF8D4E16C4F21F8D5
:10A810005C2D304601326B4EB3FBF2F30322B3FBE7
:10A82000F6F3002602939BB2B3FBF2F3AEF80030CE
:10A830005B003B80ADF80C60ADF806608DF80E60F3
:10A8400035F0F6F8E379ADF8126060229907ADF8BB
:10A8500014600696ADF81C60ADF81E60ADF820607F
:10A86000ADF82260ADF8102040F1948013F0010F94
:10A870000CBF324608220423ADF81E20ADF8143078
:10A88000002304AA61792868069301F0E7FE617944
:10A8900028684D4E35F09CF82B68B3F844206FEAD9
:10A8A00042426FEA524292B2A3F844201A8892B20E
:10A8B00042F080021A80E2796079198C92074CBFCD
:10A8C00004220122824092B289B221EA0201198453
:10A8D000198C89B20A431A841A8892B242F0010292
:10A8E0001A80207D00222921FFF796FE6022374939
:10A8F000207D0023FFF76CFEE06830602BF022FF24
:10A900003068036823F0010303602BF01BFF09A8E4
:10A910002BF0DAFE2B6862792169306809913433B3
:10A920001A4440F22A330A920D934FF48062284B66
:10A930000F920B9340224FF48053002709A90C92E9
:10A9400010934FF480424FF4403311920E971297B8
:10A9500013932BF0CBFE637929681E480C2B9CBF08
:10A960001D4A32F813708B8932689BB23B438B814E
:10A970001368012143F010031360017019B0F0BD9A
:10A9800000F1B77202F558521449B2FBF1F2013AE4
:10A9900092B238E713F0010F0CBF0021022101220F
:10A9A0004FF48073ADF81C10ADF81220ADF82030D4
:10A9B00066E700BF8054002090240020FF6BDC027B
:10A9C0007654002000350C007C5400207D81000866
:10A9D000A8600020785400205C700408006CDC0241
:10A9E000745400200348D0F8AC3113B100F5D27094
:10A9F00018477047801B00200348D0F8903113B1EE
:10AA000000F5C47018477047801B00200348D0F839
:10AA1000743113B100F5B67018477047801B0020E1
:10AA20000348D0F8583113B100F5A87018477047A3
:10AA3000801B00200348D0F83C3113B100F59A7018
:10AA400018477047801B00200348D0F8203113B10D
:10AA500000F58C7018477047801B00200348D0F821
:10AA600004310BB1FC301847704700BF801B002039
:10AA70000348D0F8E8300BB1E0301847704700BF0A
:10AA8000801B00200348D0F8CC300BB1C4301847ED
:10AA9000704700BF801B00200348D0F8B0300BB1D6
:10AAA000A8301847704700BF801B00200348D0F82B
:10AAB00094300BB18C301847704700BF801B0020CA
:10AAC0000248836F0BB1703018477047801B00201D
:10AAD0000248C36D0BB1543018477047801B0020EB
:10AAE0000248036C0BB1383018477047801B0020B8
:10AAF0000248436A0BB11C3018477047801B002086
:10AB00000248836803B11847704700BF801B0020CC
:10AB1000F8B584894FF6FF764FF47A7433B319B3DE
:10AB20000F78013101E0B44218D00589013CAD072E
:10AB3000A4B2F8D5BCB284814FF47A7402E0BCB2FE
:10AB4000B4420BD00589ED0704F1FF37F7D58589AD
:10AB5000ADB20AB115700132013BDFE70DF096F896
:10AB6000003018BF0120F8BDFF27DEE70120F8BD47
:10AB70009249934A2DE9F84F012313700B88914AAB
:10AB800023F040031B041B0C12880B800B8823F05E
:10AB900038031B0452084FEA13430BD042F480726F
:10ABA000002A92FAA2F1B1FA81F208BF4FF0FF3207
:10ABB000013AD2001343814A9BB2138013889BB29F
:10ABC00043F040031380804B1B6813B11A689B88C5
:10ABD000538380217948FDF7E3FD00217748FDF795
:10ABE000DFFD794B1B6813B11A689B881383734A86
:10ABF000764C1388764D23F040031B041B0C138006
:10AC0000138823F038031B041B0C138013889BB29A
:10AC100043F04003138023782F68834262D0FDF70E
:10AC2000EDFD6C4E6C4BB6F8F221B3F80080DFF806
:10AC3000B8C100210D464FF0050B4FF0060A4FF04A
:10AC40000709B4181CF802002379834202F10107B6
:10AC500005F1050312D006EB030E73192071140AD7
:10AC600083F8F4B183F8F6A183F8F72183F8F8911B
:10AC700083F8F541013106358EF8F401BAB2424548
:10AC800001F1010109D26329DBDDA6F8F2214DB9FA
:10AC90004B4A00231370BDE8F88F0023A6F8F23169
:10ACA000002DF5D0474B45481988FDF749FB464B29
:10ACB0001B6813B11A689B8853832B4600224749AF
:10ACC0003E48FFF725FF404B1B6813B11A689B886D
:10ACD000138304213948FDF733FB394A00231370ED
:10ACE000BDE8F88F3E4B3B4E1B78002B9AD1D6F82F
:10ACF000E831FB1AB3F57A7F94D9324B10461988A4
:10AD0000FDF71EFB304B1B6813B11A689B885383F9
:10AD1000A0212A48FDF744FD00212848FDF740FD09
:10AD2000294B1B68814613B11A689B881383DFF88F
:10AD3000BC8022480421FDF703FB98F80030182B53
:10AD400018D019F0040F11D109F00503012B1FD001
:10AD50004BB923785B0606D5D6F8EC212B68DAB11F
:10AD60009B1A642B1BD8C6F8E8715BE70023C6F872
:10AD7000EC31F8E723781B4A03F04003002B09F07D
:10AD800007010CBF0D20102013805180D080D8E720
:10AD900023785A06E0D5E6E7C6F8EC31E3E7FDF79D
:10ADA0002DFD98F80030182BDDD1B6F8F0310D4AA2
:10ADB00001339BB2A6F8F0319380D4E7003C004009
:10ADC000FF530020E41D0020D88D00200403002044
:10ADD00058AA00209024002024010020842600206E
:10ADE000EC8D0020E48D0020F0510020E18D00204A
:10ADF000037C022B01D00020704770B5836982B0BC
:10AE000013B11A689B8853830446C3214069FDF738
:10AE1000C7FC06236A4600216069FFF779FEA36933
:10AE200013B11A689B8813839DF804009DF8006095
:10AE30009DF801109DF802509DF803209DF8053003
:10AE400041EA062143EA002342EA05220120218744
:10AE50006287A38702B070BD2DE9F04F90F855309E
:10AE600085B00646002B40F0C882474B93F84C341F
:10AE7000002B00F08F807069444B984200F04782AD
:10AE8000434A90420CBF30223822038823F040030B
:10AE90001B041B0C038003889BB223F038031A4366
:10AEA000028003889BB243F040030380B36996F8A5
:10AEB0004E4013B11A689B88538340F2E93304E093
:10AEC000013B9BB2002B00F00E8402899207F7D55C
:10AED0001A23838140F2E93304E0013B9BB2002B4B
:10AEE00000F001840289D707F7D5838940F2E9335E
:10AEF00004E0013B9BB2002B00F0F283028995072E
:10AF0000F7D5A4B2848140F2E93304E0013B9BB25F
:10AF1000002B00F0E5830289D107F7D58389B36957
:10AF200013B11A689B88138302F04CF9044602F0AF
:10AF300049F98442FBD07069144B984200F0CE83EB
:10AF4000134A904214BF08220022038823F04003D2
:10AF50001B041B0C038003889BB223F038031A43A5
:10AF6000028003889BB243F040030380337C022BB2
:10AF700000F03283B6F93A305BB2013300F09382CD
:10AF800005B0BDE8F08F00BF9024002000380040DD
:10AF9000003C00407069614B984200F09D83604A1C
:10AFA00090420CBF30223822038823F040031B0458
:10AFB0001B0C038003889BB223F038031A430280E2
:10AFC00003889BB243F040030380B36913B11A684E
:10AFD0009B8853836B21FDF7E3FB80217069FDF7AC
:10AFE000DFFBB36913B11A689B88138396234D4C1A
:10AFF0004D4DDFF83CA14D48DFF838C101934FF0CB
:10B0000010084FF47A77B146DAF80430C3F3080336
:10B01000002B40F0D681EFF31183002B40F0D1815B
:10B020002368816800BF22689342F9D12A6807FB30
:10B0300002FEAEEB010EBEFBF2FE07FB03EE0126A5
:10B04000DAF80430C3F30803002B40F08081EFF3FB
:10B050001183002B40F07B812368816800BF226848
:10B060009342F9D1D5F800B007FB0BF2521AB2FBAC
:10B07000FBF207FB0323A3EB0E03B3F57A7FDFD3C9
:10B08000019B013B0193BFD1D9F818304E4613B153
:10B090001A689B88538368217069FDF781FB03213F
:10B0A0007069FDF77DFBB36913B11A689B88138340
:10B0B0009623DFF87CA01D48DFF878C001934FF09D
:10B0C00010084FF47A77B146DAF80430C3F3080376
:10B0D000002B40F05A81EFF31183002B40F0558193
:10B0E0002368816800BF22689342F9D12A6807FB70
:10B0F00002FEAEEB010EBEFBF2FE07FB03EE0126E5
:10B10000DAF80430C3F30803002B40F00281EFF3B8
:10B110001183002B40F0FD800EE000BF003800409E
:10B12000003C004058AA00205CAA002010E000E08B
:10B1300000ED00E054AA00202368816800BF226867
:10B140009342F9D1D5F800B007FB0BF2521AB2FBCB
:10B15000FBF207FB0323A3EB0E03B3F57A7FCFD3F8
:10B16000019B013B0193AFD1D9F818304E4613B182
:10B170001A689B8853836B217069FDF711FB0321CB
:10B180007069FDF70DFBB36913B11A689B881383CF
:10B190000F2002F063F8B36913B11A689B885383D8
:10B1A0006A217069FDF7FCFA10217069FDF7F8FA61
:10B1B000B36913B11A689B8813830F2002F04EF80D
:10B1C000B36913B11A689B8853836C217069FDF7CA
:10B1D000E7FA00217069FDF7E3FAB36913B11A6861
:10B1E0009B8813830F2002F039F8B36996F850401A
:10B1F00013B11A689B88538319217069FDF7D0FA3F
:10B2000021467069FDF7CCFAB36913B11A689B88BF
:10B2100013830F2002F022F8B36913B11A689B88D8
:10B2200053831B217069FDF7BBFA18217069FDF784
:10B23000B7FAB36913B11A689B8813830F2002F021
:10B240000DF8B36913B11A689B8853831C21706988
:10B25000FDF7A6FA10217069FDF7A2FAB36913B1E0
:10B260001A689B8813830F2001F0F8FFB36913B1AC
:10B270001A689B88538337217069FDF791FA102172
:10B280007069FDF78DFAB36913B11A689B8813834F
:10B290000F2001F0E3FFB36913B11A689B88538351
:10B2A00038217069FDF77CFA01217069FDF778FAA1
:10B2B000B36913B11A689B8813830F2001F0CEFF86
:10B2C0007369B74A934200F00582B6498B4214BFB6
:10B2D000082100211A8822F040021204120C1A8060
:10B2E0001A8892B222F03802114319801A8892B259
:10B2F00042F040021A80012001F0B0FFAA4A7069B2
:10B30000012382F84C34A64B98427FF4B9AD302229
:10B31000BBE5EFF3118188F31288D0F808B0036819
:10B32000DB0344BFCCF80060D0F808B02368DCF839
:10B330000020C9B281F3118829681A4407FB01F380
:10B34000A3EB0B03B3FBF1F307FB023303E7EFF3CC
:10B35000118188F31288D0F808B00368DB0344BF7A
:10B36000CCF80060D0F808B02368DCF80020C9B23F
:10B3700081F3118829681A4407FB01F3A3EB0B033F
:10B38000B3FBF1F307FB023375E6EFF3118388F3A8
:10B39000128881680268D20303D50122CCF800200C
:10B3A00081682668DCF800E0DBB283F311882A6844
:10B3B000B64407FB02F35B1AB3FBF2F307FB0E3E46
:10B3C0009DE6EFF3118388F3128881680268D20347
:10B3D00003D50122CCF8002081682668DCF800E063
:10B3E000DBB283F311882A68B64407FB02F35B1AC9
:10B3F000B3FBF2F307FB0E3E21E61D09013D032DD1
:10B4000003F00F0300F25D81684A32F8150040FA3C
:10B4100003F2D10740F15581012404FA03F3013B03
:10B42000184037F0D1FD624B624A5B5D184412EB65
:10B43000C00500F0468100232021EB71A97152F86C
:10B4400030005D4A00F13F4303F57E039B0AD25C66
:10B4500002F01F035209032A04FA03F300F02C81BF
:10B46000042A00F02481022A00F01C81AB88029398
:10B4700002A9002303932BF0BFFA31464F4B41F84A
:10B480000C3F284634F0CCF8AB88B3FA83F3C3F111
:10B490001F03012212FA03F33FF4E7AC48490A689C
:10B4A00013430B60E1E496F9383001337FF468AD63
:10B4B0000A23444C444D454E454F0193322034F00D
:10B4C000E1FCDFF810914FF4FA7A4FF0100801F028
:10B4D00079FE4FF47A7186460120D9F80430C3F31F
:10B4E0000803002B40F0C080EFF31183002B40F0E5
:10B4F000BB80AC462368B56800BF22689342F9D18F
:10B500006246AC46D2F800B0154601FB0BF2A2EB46
:10B510000C02B2FBFBF201FB0323A3EB0E03B3F51A
:10B520007A7FDAD3BAF1010AD1D1072034F00CFBCB
:10B53000DFF8A0904FF47A7A4FF0100801F042FE45
:10B540004FF47A7186460120D9F80430C3F308031A
:10B55000002B6BD1EFF31183002B67D1AC4623682E
:10B56000B56800BF22689342F9D16246AC46D2F872
:10B5700000B0154601FB0BF2A2EB0C02B2FBFBF292
:10B5800001FB0323A3EB0E03B3F57A7FDCD3BAF1FF
:10B59000010AD3D1019B013B01938FD1FEF7BCFF80
:10B5A00000380040003C004090240020FC75040856
:10B5B000F875040858A800200075040819800008D0
:10B5C000003C014058AA00205CAA002010E000E0E6
:10B5D00054AA002000ED00E0B36913B11A689B88FB
:10B5E0005383C321FDF7DCF8062302AA002170690A
:10B5F000FFF78EFAB36913B11A689B8813839DF81D
:10B600000A509DF80B309DF808409DF809109DF8F0
:10B610000C009DF80D2043EA05231BB241EA0421EA
:10B6200042EA002273873187B287A5E4EFF3118CD9
:10B6300088F31288D6F808B03368DB0344BF38605B
:10B64000D6F808B023683A685FFA8CFC8CF311884E
:10B65000D5F800C01A4401FB0CF3A3EB0B03B3FBBA
:10B66000FCF301FB02338DE7EFF3118C88F31288B2
:10B67000D6F808B03368DA0344BF3860D6F808B0AB
:10B6800023683A685FFA8CFC8CF31188D5F800C007
:10B690001A4401FB0CF3A3EB0B03B3FBFCF301FB1C
:10B6A00002333AE7124A516C0B435364DEE6104A08
:10B6B000116B0B431363D9E60D4A116C0B431364F2
:10B6C000D4E631460B4B41F80C3F002033F0A8FF85
:10B6D000FFF7CBBB0021FDE5302265E4002234E416
:10B6E0000CF0D4FA1BE40CF0D1FA7069FFF7FEBB42
:10B6F0000038024019800008037A022B01D0002094
:10B70000704770B5036982B013B11A689B88538380
:10B710000446BB21C068FDF743F806236A460021B2
:10B72000E068FFF7F5F9236913B11A689B88138362
:10B730009DF804009DF800609DF801109DF80250EE
:10B740009DF803209DF8053041EA062143EA0023D5
:10B7500042EA05220120E1822283638302B070BDA8
:10B76000F8B50501684C694B625961199A4204EBBE
:10B77000050704BF01230B730646387A33F0CEFE6B
:10B780003B7A03F01F015B090122032B02FA01F24D
:10B790006DD0042B66D0022B5CD06319013618796A
:10B7A0000BF0DAFEF6B2074610B11223C6718371B0
:10B7B000631958790BF0D0FE10B11323C671837151
:10B7C000631998790BF0C8FE10B11423C671837108
:10B7D00066190A21F27938460BF084FF70790BF074
:10B7E000BBFEF2790A210BF07DFFB0790BF0B4FEBD
:10B7F000F2790A210BF076FF6359454A934247D00C
:10B80000424A934250D0434A934259D0424A9342CB
:10B8100062D0424A93426BD0414A93422CD02C448E
:10B82000227BE2B901200222198801F4415141F43E
:10B8300045710A4302431A809A8B22F40062120473
:10B84000120C07219A8319821A8892B242F04002A0
:10B850001A80F8BD334B596A0A435A629DE70020AB
:10B860000246E1E72F4B19690A431A6195E72D4B10
:10B87000196A0A431A6290E702F564424FF4001015
:10B88000536A43F4001353622AF064FE6359C6E717
:10B8900002F584324FF48050536A43F4805353626C
:10B8A0002AF058FE6359BAE702F500324FF480409F
:10B8B000136A43F4804313622AF054FE6359AEE7DF
:10B8C00002F5FE324FF40040136A43F40043136262
:10B8D0002AF048FE6359A2E702F582324FF4005085
:10B8E000536A43F4005353622AF034FE635996E7D7
:10B8F00002F568424FF48010536A43F48013536298
:10B900002AF028FE63598AE70C8E00200038004098
:10B9100000300140003C0040003401400050014034
:10B9200000540140003802401549164B16484A6839
:10B9300010B4CC681549B2FBF4F203FB02F30360C8
:10B94000D1F88820124B134C42F47002C1F88820C1
:10B950001A68002042F001021A6098601A6822F00A
:10B96000847222F480321A605C601A684FF00064BE
:10B9700022F480221A60D8608C605DF8044B704716
:10B980000000002040420F002074002000ED00E085
:10B990000038024010300024044B4FF4F0700221B4
:10B9A0000A225860D9609A60FFF7BEBF00000020ED
:10B9B00038B50B4C23688BB15A68821A002A0546A9
:10B9C00004DA0CE05A68AA1A002A07DB9A68226097
:10B9D00018461A6890472368002BF3D138BD38BD4C
:10B9E000A0A400200B4B002210B40272114603F1F8
:10B9F000900402E0072909DC9A79920702D51A79A6
:10BA0000425401319C4203F11803F3D15DF8044B19
:10BA1000704700BF5075040810B40D4C0023214638
:10BA20001A4600E08B7913F0010301F1180106D1E9
:10BA30000132072AF6D103705DF8044B704702EB20
:10BA4000420204EBC2025DF8044B137903707047A5
:10BA500050750408012310B431213224332244707C
:10BA60004171C27003720370037183705DF8044BFF
:10BA7000704700BF2322032302704370704700BF4A
:10BA80002DE9F0410B78047BDB43DEB200F11002BC
:10BA900000F1380342F8044F9342FBD1DFF89CC019
:10BAA00000F16001002243F8042F8B42FBD14FF0DC
:10BAB000140E0521002546FA01F303F00103002BC3
:10BAC0001D4414BF4FF019084FF00A0811F0010F80
:10BAD000EDB214BF2746002700220EEB02039BB2F3
:10BAE00000EB8303013242455F61F6D1013A92B225
:10BAF000013201390EEB02034A1C9BB201D09E4673
:10BB0000D9E715F0010F14BF19250A2500215A188D
:10BB100092B200EB82020131A9425461F7D10B4489
:10BB20009BB21A1D00EB8202013300219BB25160CF
:10BB3000ACF800300361BDE8F08100BFE0280020D0
:10BB4000254B5B880B332DE9F04F8A4601F1060B3C
:10BB50001FFA83F94FF00108002100271AF801EBC2
:10BB60003E464C460122A4F10B039BB207E0013391
:10BB70009BB2B0F80CC0C5F814C09C420AD000EBD0
:10BB80008305002AF3D100EB830501339BB29C426D
:10BB90006A61F4D1231D00EB83030136092FF6B24D
:10BBA00059600CD0092E14D008FA07F313EA0E0FCF
:10BBB00014BF012200220C34A4B20137D3E709F1EB
:10BBC0007809DA451FFA89F9C7D1034B5980BDE8D6
:10BBD000F08F0022EFE700BFE02800202DE9F047BA
:10BBE000DFF85C80B8F8043004338A461FFA83FC1F
:10BBF00001F109094FF0010E1AF8017B6446002695
:10BC0000231F0EFA06F29BB23A40BAB1818900EBCB
:10BC1000830501339BB29C426961F6D1013604343D
:10BC2000082EA4B2ECD10CF1200CCA451FFA8CFCF2
:10BC3000E2D10023A8F80430BDE8F0871146E6E71A
:10BC4000E028002010B5027B01681F2A4FF0200376
:10BC50000ED94C68203A93401C4216D00B4A4068DB
:10BC600000241470026822F001020260CB6010BD53
:10BC70000C6893401C4208D0044A406800241470A9
:10BC8000026822F0010202608B6010BD6B3400205C
:10BC9000436A8269D154436A0169826B01338B42E2
:10BCA00028BF00234362002A2FD0EFF311825023D4
:10BCB00083F31288836B1968C9072CD470B45E684B
:10BCC0006EB9456A816A8D4217D084690C44DC6084
:10BCD0000ED9691A59608562002180F85C101968D4
:10BCE00041F00101D2B2196082F3118870BC704733
:10BCF0000469611A59608662EEE7012380F85C30BE
:10BD0000D2B282F3118870BC7047826DD36843F061
:10BD10008003D3607047D2B282F31188704700BFAE
:10BD2000426B10B462B1C36CC2684469D11A013B62
:10BD3000615C5DF8044B08BF1346C364C8B270472A
:10BD4000016A4369C4685B5C0131A14228BF1146A6
:10BD500001625DF8044BD8B2704700BF836B13B12A
:10BD600090F85C007047836A406A181AB0FA80F055
:10BD700040097047416A836A99420AD3CB1A816BA2
:10BD8000026961B14968501E0B4483420AD2C01A4D
:10BD9000704702691144CB1A816B0029F2D1501E01
:10BDA000C01A704700207047436B43B1C26C5B6898
:10BDB00093422FBF981AC0689B1AC0187047C26977
:10BDC000036A9A422FBFD01AC0688018C01A704701
:10BDD0000A4B30B503F1140493F900205D78072A6B
:10BDE000C8BF143A81180433CD7213F8025C85542D
:10BDF00013F8012C8A75A342EED130BDE048040847
:10BE000003682DE9F041DF691FB13B46BDE8F04111
:10BE10001847002A164611DD04460D460E4400E080
:10BE200023689B68204698470028F9D0236815F8B6
:10BE3000011B1B6820469847AE42F1D1BDE8F08156
:10BE400000232522027043708370C370704700BFC7
:10BE5000038A2DE9F0478589ADB21D4029D00F46F0
:10BE600006464FF000484FF00009B5FA85F328FA6E
:10BE700003F2D24391B21B3B15403182042B16D8FA
:10BE8000DFE803F03129211903007B6A002B32D04F
:10BE900003F1FF3A1FFA8AFAC7F824903C6A34B1DA
:10BEA00023682046514698476468002CF8D1002D3D
:10BEB000DBD1BDE8F0873868716B036889B29847B9
:10BEC000002DD2D1F5E77868B16B036889B2984745
:10BED000002DCAD1EDE7B868F16B036889B29847C5
:10BEE000002DC2D1E5E7F868316C036889B2984744
:10BEF000002DBAD1DDE7F36A1FFA83FACEE700BF5F
:10BF000030B50446806D61718389A26823F40053C3
:10BF10001B041B0C838185B0A379009213F00402EB
:10BF200030D04FF4805213F00203ADF804205CD1FE
:10BF3000ADF806304FF480630022ADF8083011F000
:10BF40000103ADF80C2028D1ADF80A3008238D0785
:10BF5000694648BFADF80A302AF054FBA279A36DB8
:10BF6000D10724D412F0080F9A8A1BD122F00802BC
:10BF70001204120C9A829A8992B242F400529A8167
:10BF800005B030BD13F00203ADF804202AD04FF401
:10BF900000551346ADF80650CEE70423ADF80A303D
:10BFA0000C23D4E792B242F008029A82E3E71049E8
:10BFB0008B4215D0A1F548418B420FD001F580612D
:10BFC0008B4209D00B498B42CCD105200121FEF7D1
:10BFD000BFFAA279A36DC5E70320F7E70220F5E7D2
:10BFE0000020F3E7ADF80630A6E74FF400539FE7D3
:10BFF000001001400014014010B50446806DA1609E
:10C00000838923F400531B041B0C8381A37984B020
:10C0100013F00402009135D04FF4805213F0020364
:10C02000ADF804205CD1ADF806304FF4806362793E
:10C03000ADF80830D1074FF00003ADF80A30ADF885
:10C040000C3045BF0423ADF80A3008230C236946A1
:10C05000920748BFADF80A302AF0D4FAA279A36D4E
:10C06000D1071FD412F0080F9A8A16D122F00802C5
:10C070001204120C9A829A8992B242F400529A8166
:10C0800004B010BD13F00203ADF8042025D04FF426
:10C0900000511346ADF80610C9E792B242F008020B
:10C0A0009A82E8E710498B4215D0A1F548418B42AE
:10C0B0000FD001F580618B4209D00C498B42D1D160
:10C0C00005200121FEF744FAA279A36DCAE70320F7
:10C0D000F7E70220F5E70020F3E7ADF80630A6E722
:10C0E0004FF400539FE700BF0010014000140140CF
:10C0F000022828BF022010B4084C094B207000EB26
:10C100008002C0EBC20207495DF8044B013003EB2B
:10C110004203C0B20B6034F00BBD00BF407300207F
:10C1200016550020CCA5002008B530F0DBFC0BF044
:10C13000E1FEBDE8084030F0BDBC00BF38B5484B5B
:10C140005A899989914224BF00225A81198ADA8931
:10C15000914224BF0022DA81DA78CAB1072A414924
:10C160006AD091F85300404D012400210A282C7018
:10C170009C70D9715DD00C2807D0002A6CD0DFEDFF
:10C180003B7A072A0ED00A2862D0DFED397A09E01F
:10C19000344A92F853000A2856D00C285BD1D9793A
:10C1A000DFED347A344C9FED350AA278002918BFB0
:10C1B000F0EE407A062A04D8314901EB820191ED74
:10C1C000050A217979B1013A032A0BD8F7EE007AF2
:10C1D00087EE800A37F040FB2388984228BF184634
:10C1E000208038BD38BD9B781F4A07EE103A117881
:10C1F000B8EEC77A67EE277A07EE101AB8EEC77A5C
:10C2000027EE277AB4EEC70AF1EE10FAEADD80EEE7
:10C21000277AFDEEC77A17EE903A102BA8BF1023AD
:10C22000012BB8BF0123DBB28B4238BF0B46137022
:10C2300038BDDFED147AA4E791F853000A2803D043
:10C240000C28ACD0D9799AE7D979DFED0E7AA9E735
:10C25000DFED0D7AA6E7D979DFED047AA2E700BF1A
:10C26000007C002024740020ECA700206F1203390A
:10C270006F12833A0AD7A339247E00206F12033845
:10C28000E04804085304E9380F506E3A2DE9F047AE
:10C29000A84FA94E30F026FCBE421ED2DFF8148310
:10C2A000DFF814934446258862197DB14A450DD2C2
:10C2B000052D0BD933886188C3F30B03994200F035
:10C2C000DC80144625886219002DEFD17168304654
:10C2D00014360BF09BFDBE42E4D3984A1378A3F1C9
:10C2E000170102290FD9964911F83300002840F0B0
:10C2F000F380D8000144497829B1924911F83330CC
:10C300000BB918231370904B5A78022A00F2D5808B
:10C310008E498F4802EB420201EB82011A780160DC
:10C32000022A00F2D38002EB82018A4BC2EBC102E7
:10C3300003EB4203998C5A8C874C9142236001D3C2
:10C3400000225A84854B9A78042A00F0E68032B99C
:10C350001A88B2F5F07F84BF4FF4F0721A80804DD6
:10C36000FFF7ECFE2B687F4A1A40002A00F0DE80BF
:10C37000D80700F1CD80590400F1C5801A0700F1FB
:10C38000B4809B0400F1B8802EF038FB10B97648D9
:10C3900033F00EFF4FF400700BF06EFD4FF40030E1
:10C3A0000BF06AFD4FF000700BF066FD4FF08060FF
:10C3B0000BF062FD35F03CFD002130226B4838F077
:10C3C00008FA206817F026F8694B256803F1500138
:10C3D00002E0043399427DD01A78002AF9D19C7882
:10C3E000D8788442F5D26349634B0A7028461D60B1
:10C3F0001CF074FD614A62491079624A624B116017
:10C40000C822642111FB0021002259609A60DA6081
:10C410001A615A619A61DA6183F8202083F8212039
:10C4200030F046F9594B9FED5A5A1B88594A9FEDF7
:10C430005A6A5079594906EE903AF8EEE66A13883E
:10C44000C5EE265A07EE103A53881279C1ED005A0C
:10C4500007EE903AB8EEC77A514BF8EEE77A1872C9
:10C460005A7227EE067A67EE867ABDE8F04783EDCA
:10C47000017AC3ED007A30F01DBB63799B077FF42E
:10C4800020AF716894F804A030460BF0BFFC3388ED
:10C49000BAEB133F04D01436BE42FFF403AF1CE7DF
:10C4A00073887068AA1FC3F30B039A4204F1060154
:10C4B000A8BF1A4636F0FAFFEDE700225A701A7844
:10C4C000234822490160022A7FF62DAF00221A700C
:10C4D000204B2FE7012286E7D8000C186468002C57
:10C4E0007FF408AF1724147004E72E480BF0C4FC47
:10C4F0002B689B047FF548AF2B480BF0BDFC402018
:10C500000BF0BAFC40E729480BF0B6FC2B6835E786
:10C5100027480BF0B1FC2B682DE79A8AB2F57A7F99
:10C52000BFF41DAF4FF47A729A8218E743F0080304
:10C530002B601DE75406000890010008A45A002053
:10C54000347804084C690408407300202256002007
:10C55000D0A5002016550020CCA50020247E002068
:10C560006C5600200960000250950020D02C00205D
:10C570005C500020B4220020042D0020944D0020A7
:10C58000FEA70020182D0020386F0020EC2E002080
:10C59000C0C9FB485029002017B7D138F02E002021
:10C5A00064470020016000020940000209200002E7
:10C5B00008600002024000080080000808B530F062
:10C5C00091FA0BF097FC30F075FAFFF75FFE01204F
:10C5D000BDE8084034F0ACBA38B50C4C0C4DAC4258
:10C5E00006D26168204614340BF010FCAC42F8D33C
:10C5F000084A094B094C1460002209491A705A7004
:10C6000008480860BDE8384024F066BC9001000886
:10C6100054060008CCA500204073002016550020C9
:10C62000D0A500202256002008B5FFF7D5FF30F036
:10C6300059FA0BF05FFCBDE8084030F03BBA054BFF
:10C6400010B59A68044C2178501C09B99A6010BD45
:10C650000246F8E7E02800206B340020F0B50C29F2
:10C6600034D8DFE801F0893333335E333333343386
:10C6700033330700048C9689B2F802E01788734DB3
:10C6800024F480542404240C0484038C8488818B37
:10C6900023F4005321F4E6411B0409041B0C46EA71
:10C6A0000E06090C43EA063341EA0721A8429BB271
:10C6B000A4B289B200F09E8005F58065A84200F022
:10C6C000998092688480818302640384F0BD048C25
:10C6D0009589B2F802C0B2F800E05C4F24F480748F
:10C6E0002404240C0484038C8688818B23F4007337
:10C6F0001B0421F073011B0C45EA0C04090443EAF6
:10C700000423090CB8429BB2B6B241EA0E015CD0D8
:10C710004F4CA04259D0926886808183C2630384C3
:10C72000F0BD048C9589B2F802C0B2F800E0474E23
:10C7300024F010042404240C0484038C8788018BC7
:10C7400023F0200321F4E6411B0409041B0C45EAF5
:10C750000C04090C43EA041341EA0E21B0429BB2D7
:10C76000BFB289B25DD03A4CA0425AD0926887805D
:10C77000018382630384F0BD048C9789B2F802E0E0
:10C780001688324D24F001042404240C0484038C04
:10C790008488018B23F002031B0421F073011B0C1E
:10C7A00047EA0E0709043B43090CA8429BB2A4B216
:10C7B00041EA060125D005F58065A84221D092689E
:10C7C0008480018342630384F0BDD589148A578A2B
:10C7D00023F4006343EA05254FF6FF332B40958889
:10C7E00026F440563C4343EA052346EA04169BB22E
:10C7F000B6B290E7158A24F4804444EA8514A4B2C2
:10C800005FE7D689158A578A23F00803334324F457
:10C81000407496883D4323F004032C433343A4B271
:10C82000CDE7D489158A568A23F0800343EA04139E
:10C830004FF6BF741C40938827F44067354344EAA1
:10C84000031347EA85079BB2BFB28FE700000140A0
:10C85000000401402DE9F04FF022002183B08A4806
:10C860008A4CDFF84C928A4D8A4E8B4FDFF8448217
:10C8700037F0AFFF89488A49DFF83CE2DFF83CC275
:10C8800000221359834200F0D480B3F1804F00F0AE
:10C89000E480AB4200F0E380B34200F0E280BB42B0
:10C8A00000F0E180734500F0E080634500F0DF8038
:10C8B000434500F0DE80DFF808A2534500F0DB803E
:10C8C0000AF5806A534500F0D8800AF5806A53451E
:10C8D00000F0D580AAF5983A534500F0D2800AF5C9
:10C8E000806A53457BD00AF5806A534508BF0D2303
:10C8F00076D01832A82AC4D1644C6A4E6A4F6B4D68
:10C9000004F1A80802E01834A04565D0A379002BF3
:10C91000F9D023794FEA131909F1FF39B9F1030F5F
:10C9200003F00F03EFD836F8190040FA03F2D207EC
:10C93000E9D54FF0010A0AFA03F3013B184036F03B
:10C9400043FB17F80930184415EBC002DBD055F84B
:10C950003000DFF870E1217A00F13F4303F57E03F8
:10C960009B0A1EF8033003F01F0E5B09032B0AFA23
:10C970000EFA60D0042B67D0022B51D0938800931D
:10C98000B3FA83F3C3F11F039BB2DA0800EB820210
:10C9900003F00703D2F820E09B004FF00F0C0CFAD5
:10C9A00003FC2EEA0C0EC2F820E0D2F820E001FAD7
:10C9B00003F343EA0E03136269460023022218348C
:10C9C0008DF804208DF805308DF806308DF807308D
:10C9D0002AF012F8A04599D103B0BDE8F08F0C23DE
:10C9E00009EBC3034FF0010A1B7903F01F0B5B092E
:10C9F000032B0AFA0BFA09D0042B0CD0022B7FF47C
:10CA000078AF4B6C4AEA03034B6472E70B6C4AEA5B
:10CA100003030B646DE70B6B4AEA03030B6368E7E0
:10CA2000DFF87CE0DEF844304AEA0303CEF8443015
:10CA3000A4E70023D4E7DFF868E0DEF840304AEAF4
:10CA40000303CEF8403099E7DFF854E0DEF83030E9
:10CA50004AEA0303CEF8303090E70123C0E702230F
:10CA6000BEE70323BCE70423BAE70523B8E70623A0
:10CA7000B6E70723B4E70823B2E70923B0E70A23A0
:10CA8000AEE70B23ACE700BF408E002050750408D2
:10CA90000004004000080040000C0040000001407D
:10CAA00000380240FC750408F875040858A80020F6
:10CAB0007870040800040140001000400014004099
:10CAC000004001400075040801490248FFF7C0B961
:10CAD000088F00200048014001490248FFF7B8B91B
:10CAE000E08E00200004014001490248FFF7B0B980
:10CAF000E08E00200004014001490248FFF7A8B978
:10CB0000B88E00200008004001490248FFF7A0B994
:10CB1000908E00200004004002494FF08040FFF753
:10CB200097B900BF688E002001490248FFF790B90D
:10CB3000408E00200000014001490248FFF788B9FB
:10CB4000408E002000000140F0B504684B4DA30A60
:10CB5000AB4276D009D94A4DAB425CD01135AB42DD
:10CB600073D0123DAB425AD0F0BDB3F5801F64D0F4
:10CB7000013DAB4257D14FF0700E02264779B0000D
:10CB80004FEA970C002964D063460227A5899F408D
:10CB900083190CEB43032F4303F1040C394DBFB24F
:10CBA00045F8231045F82C20A781EFF3118150227E
:10CBB00082F31288821905EBC2021369002B33D06D
:10CBC00013620433821905EBC202576917B11F6063
:10CBD00053690433821905EBC202976917B11F60CC
:10CBE00093690433821905EBC202D76917B11F603C
:10CBF000D36904330027CAB21F6082F3118830441E
:10CC000005EBC000036A93B9A38923F001031B0459
:10CC10001B0CA381F0BD4FF0C00E0426AEE74FF011
:10CC2000200E0026AAE7F0BD05EB0E03CAE7A38994
:10CC30009BB243F00103A381F0BD4FF0480E0126E3
:10CC40009CE74FF0980E032698E74FF0E80E052674
:10CC500094E70223BF0803FA07F7A389094D9BB2A3
:10CC600023EA070387190CEB470CA3810CF104039B
:10CC700045F82C1045F8232097E700BF020010006C
:10CC800041001000408E002010B503688248013931
:10CC9000834282B089B200F0CA80A0F580608342EE
:10CCA00000F0C58000F58040834200F0B78000F5B9
:10CCB0008060834200F0B28000F58060834200F023
:10CCC000AD80764C188824686408B4FBF2F4013C0B
:10CCD000A4B282B2B3F1804F0AD07148834207D028
:10CCE00000F58060834203D000F58060834202D16A
:10CCF00022F0700292B26B48834200F0A18000F5EE
:10CD00008060834200F0A68022F4407200F56C40FF
:10CD100092B283421A80D9621C854FD05E4A9342F8
:10CD20004CD001229A821A8892B242F001021A80F3
:10CD3000B3F1804F00F09880594A934200F09680FA
:10CD400002F58062934200F0938002F58062934284
:10CD500000F0908002F58062934200F08D8002F531
:10CD60008062934200F08A8002F57042934200F0A4
:10CD7000878002F57052934200F0848002F5806251
:10CD8000934200F0818002F5806293427ED0A2F54A
:10CD9000983293427CD002F5806293427AD002F5B9
:10CDA0008062934208BF0D2215D002A84FF00123E4
:10CDB00040F8043D29F096FB02B010BD012200218D
:10CDC00019869A821A88384892B242F00102834248
:10CDD0001A80ADD10A46354B03EBC20301A85C793A
:10CDE0008DF80440012300228DF805308DF80730BE
:10CDF0008DF8062029F076FB1B2C08D02E2CDBD1D9
:10CE00002B4B019301A829F06DFB02B010BD294BFB
:10CE1000019301A829F066FB02B010BD1F4C1888D1
:10CE20002468B4FBF2F4013CA4B282B252E71B4C7A
:10CE300018882468B4FBF2F4013CA4B282B257E72C
:10CE400001201A80D9621C8598821A8892B2024306
:10CE50001A8071E701201A80D9621C8598821A888D
:10CE600092B202431A8063E70122B4E70222B2E7DA
:10CE70000322B0E70422AEE70522ACE70622AAE7C8
:10CE80000722A8E70822A6E70922A4E70A22A2E7C8
:10CE90000B22A0E70C229EE7000401402074002032
:10CEA00000040040001000400000014078700408B9
:10CEB0002C010001190100012B4B98423CD0B0F12C
:10CEC000804F3BD0A3F57C43984239D003F5806373
:10CED000984237D003F58063984235D003F58063DC
:10CEE000984233D003F58063984231D003F5704304
:10CEF00098422FD003F5705398422DD003F58063EC
:10CF000098422BD003F58063984229D0A3F598333B
:10CF1000984227D003F58063984207D003F58063D9
:10CF2000984208BF0D2202D0002070470C220F4B00
:10CF300003EBC203187970470022F8E70122F6E7F5
:10CF40000222F4E70322F2E70422F0E70522EEE7EB
:10CF50000622ECE70722EAE70822E8E70922E6E7EB
:10CF60000A22E4E70B22E2E700000140787004089F
:10CF70002DE9F04F013085B0C3B203930B46029107
:10CF80008B4C8C4E002B00F09A8032208A4D8B4FB8
:10CF9000DFF82C9232F076FF4FF4FA7A4FF0100C53
:10CFA0004FF47A70D9F80430C3F30803002B40F033
:10CFB000DE80EFF31183002B40F0D9802968A2684E
:10CFC00000BF2B689942F9D1D7F800E000FB0EF3BF
:10CFD0009B1AB3FBFEF300FB01314FF0010E0191F0
:10CFE000D9F80430C3F30803002B40F08780EFF337
:10CFF0001183002B40F082802B68A16800BF2A6853
:10D000009342F9D1D7F800B000FB0BF2521AB2FBF1
:10D01000FBF200FB0323019A9B1AB3F57A7FDFD35F
:10D02000BAF1010ABED1039B002B40F0BD804FF442
:10D030007A7ADFF88C9150464FF0100CD9F8043012
:10D04000C3F30803002B75D1EFF31183002B71D1CB
:10D050002968A26800BF2B689942F9D1D7F800E08F
:10D0600000FB0EF39B1AB3FBFEF300FB01314FF004
:10D07000010E0191D9F80430C3F3080313BBEFF399
:10D080001183FBB92B68A16800BF2A689342F9D1CC
:10D09000D7F800B000FB0BF2521AB2FBFBF200FB18
:10D0A0000323019A9B1AB3F57A7FE3D3BAF1010AFD
:10D0B000C4D1029B013B0293002B7FF466AF05B005
:10D0C000BDE8F08FEFF311888CF31288A168236814
:10D0D000DB0344BFC6F800E0A1682B6832685FFA42
:10D0E00088F888F31188D7F800801A4400FB08F309
:10D0F0005B1AB3FBF8F300FB0233D2E7EFF31188BE
:10D100008CF31288A1682368DB0344BFC6F800E0F3
:10D11000A1682B6832685FFA88F888F31188D7F81D
:10D1200000801A4400FB08F35B1AB3FBF8F300FB22
:10D13000023370E7EFF311828CF31288D4F808E021
:10D140002368D90303D501233360D4F808E02B68A2
:10D150003168D2B282F311883A68194400FB02F3B5
:10D16000A3EB0E03B3FBF2F300FB01317FE7EFF318
:10D1700011828CF31288D4F808E02368D90303D510
:10D1800001233360D4F808E02B683168D2B282F30F
:10D1900011883A68194400FB02F3A3EB0E03B3FBBA
:10D1A000F2F300FB013118E7184632F0CDFC3EE700
:10D1B00010E000E054AA002058AA00205CAA002039
:10D1C00000ED00E0204B5B68C3F3080330B4BBB94B
:10D1D000EFF31183A3B91D4B1D4C1868A16800BF64
:10D1E0001A689042F9D11B4B1C684FF47A7202FB0B
:10D1F00004F3591AB1FBF4F130BC02FB0010704784
:10D20000EFF31182102383F3128811498C680B68A5
:10D2100013F4803F104B02D0012018608C680B493A
:10D22000D2B20D68186882F311880A4B19684FF45E
:10D230007A72284402FB01F31B1B30BCB3FBF1F3F1
:10D2400002FB0030704700BF00ED00E058AA00204C
:10D2500010E000E05CAA002054AA00202DE9F84F5D
:10D260008046FFF7AFFF254E2549DFF8A0E0254AAD
:10D27000254D844610274FF47A740120DEF80430DF
:10D28000C3F30803D3B9EFF31183BBB90B68D2F82A
:10D2900008A000BFD1F800904B45F7D1D6F800B0F8
:10D2A00004FB0BF9A9EB0A09B9FBFBF904FB039397
:10D2B000A3EB0C034345E1D3BDE8F88FEFF3118AEC
:10D2C00087F31288D2F808B01368DB0344BF2860E4
:10D2D000D2F808B00B68D5F800905FFA8AFA8AF3A2
:10D2E0001188D6F800A0994404FB0AF3A3EB0B03C2
:10D2F000B3FBFAF304FB0933DAE700BF5CAA0020B2
:10D3000058AA002010E000E054AA002000ED00E040
:10D310002DE9F04FDFF830C1474A4849484E494DA2
:10D320008046102718F1FF38C0F08480DCF8043004
:10D33000C3F30803002B5CD1EFF31183002B58D10A
:10D340000B68946800BF08688342F9D1D6F8009052
:10D350004FF47A7000FB09FEAEEB040EBEFBF9FE43
:10D3600000FB03EEDCF80430C3F308034FF47A74D7
:10D370000120FBB9EFF31183E3B90B68D2F808A0E1
:10D3800000BFD1F800904B45F7D1D6F800B004FBB0
:10D390000BF9A9EB0A09B9FBFBF904FB0393A3EB17
:10D3A0000E03B3F57A7FBDD2DCF80430C3F3080373
:10D3B000002BDFD0EFF3118A87F31288D2F808B080
:10D3C0001368DB0344BF2860D2F808B00B68D5F8B7
:10D3D00000905FFA8AFA8AF31188D6F800A099447F
:10D3E00004FB0AF3A3EB0B03B3FBFAF304FB0933CF
:10D3F000D5E7EFF3118487F31288D2F80890136809
:10D40000D80303D501232B60D2F808900B68286855
:10D41000E4B284F31188D6F800A04FF47A7400EBDC
:10D42000030E04FB0AF3A3EB0903B3FBFAF304FBBB
:10D430000E3E97E7BDE8F08F10E000E058AA00200C
:10D440005CAA002054AA002000ED00E030B4EFF305
:10D450001183102282F312880649074C0A68074894
:10D46000013200250A602560DBB2026883F311886F
:10D4700030BC704758AA002054AA002010E000E0F9
:10D480000F4B1B88014643B90E4B0F4A1B7810689F
:10D490000BB981F001010AF0B3BA0C4B5A691AB109
:10D4A00018B91A68106058747047094A18681188CA
:10D4B000084A92FBF1F2012102605974704700BFE3
:10D4C00030AA002032AA002034AA002038AA002066
:10D4D00050AA002020A1070038B5264B5C69636B79
:10D4E00073B1A36DA26BD2B1998A1A88C90592B2A1
:10D4F00001D5D20700D438BD4FF6F7721A8038BD77
:10D50000A36D99891A88890692B2EBD59206E9D55E
:10D51000E26AD2B19888216B80B29047E1E799899D
:10D520001A880D0692B2DFD51006DDD5A26A616AAF
:10D530008A4219D0A1692569885C98800132B2FBC2
:10D54000F5F105FB1122A262CEE79B88E2696169D1
:10D55000DBB28B54E269E068A36D0132B2FBF0F1FB
:10D5600000FB1122E261BDE7DA6822F08002DA6096
:10D57000BAE700BF8C46002038B5264BDC68636BE9
:10D5800073B1A36DA26BD2B1998A1A88C90592B200
:10D5900001D5D20700D438BD4FF6F7721A8038BDD6
:10D5A000A36D99891A88890692B2EBD59206E9D5BE
:10D5B000E26AD2B19888216B80B29047E1E79989FD
:10D5C0001A880D0692B2DFD51006DDD5A26A616A0F
:10D5D0008A4219D0A1692569885C98800132B2FB22
:10D5E000F5F105FB1122A262CEE79B88E269616931
:10D5F000DBB28B54E269E068A36D0132B2FBF0F15B
:10D6000000FB1122E261BDE7DA6822F08002DA60F5
:10D61000BAE700BF8C46002038B5264B9C68636B88
:10D6200073B1A36DA26BD2B1998A1A88C90592B25F
:10D6300001D5D20700D438BD4FF6F7721A8038BD35
:10D64000A36D99891A88890692B2EBD59206E9D51D
:10D65000E26AD2B19888216B80B29047E1E799895C
:10D660001A880D0692B2DFD51006DDD5A26A616A6E
:10D670008A4219D0A1692569885C98800132B2FB81
:10D68000F5F105FB1122A262CEE79B88E269616990
:10D69000DBB28B54E269E068A36D0132B2FBF0F1BA
:10D6A00000FB1122E261BDE7DA6822F08002DA6055
:10D6B000BAE700BF8C46002038B5264B1C68636B68
:10D6C00073B1A36DA26BD2B1998A1A88C90592B2BF
:10D6D00001D5D20700D438BD4FF6F7721A8038BD95
:10D6E000A36D99891A88890692B2EBD59206E9D57D
:10D6F000E26AD2B19888216B80B29047E1E79989BC
:10D700001A880D0692B2DFD51006DDD5A26A616ACD
:10D710008A4219D0A1692569885C98800132B2FBE0
:10D72000F5F105FB1122A262CEE79B88E2696169EF
:10D73000DBB28B54E269E068A36D0132B2FBF0F119
:10D7400000FB1122E261BDE7DA6822F08002DA60B4
:10D75000BAE700BF8C46002070B4EFF31186502367
:10D7600083F31288836B1A68D20720D45D686DB981
:10D77000446A826A944217D081691144D9600ED9F3
:10D78000A21A5A608462002280F85C201A6842F073
:10D790000102F1B21A6081F3118870BC704701690F
:10D7A0008A1A5A608562EEE7012380F85C30F3B292
:10D7B00083F3118870BC704703685B6A03B1184734
:10D7C000704700BF03681B6A03B11847704700BF6A
:10D7D00003682DE9F041DF691FB13B46BDE8F04128
:10D7E0001847002A164611DD04460D460E4400E097
:10D7F00023689B68204698470028F9D0236815F8CD
:10D80000011B1B6820469847AE42F1D1BDE8F0816C
:10D8100003689B69184700BF03685B69184700BF2E
:10D8200003681B69184700BF0368DB68184700BF1F
:10D8300003689B68184700BF03685B68184700BF10
:10D8400003681B68184700BF38B50C46097849B112
:10D85000054601342B6828461B68984714F8011BBD
:10D860000029F7D138BD00BF10B40B4B0B4A1C7810
:10D8700001238340234052F8200031B9B3FA83F1E9
:10D8800049095DF8044B0AF0BBB8191C18BF012107
:10D890005DF8044B0AF0B4B820AA002024AA0020A6
:10D8A0001C4C08B501210220FFF7DEFF237803F0AE
:10D8B0000502052A29D003F00903092B08D000210D
:10D8C0000120FFF7D1FF00210846FFF7CDFFFEE75B
:10D8D000114A124B11681A680B68114C23F00103AE
:10D8E0000B601388206823F001031B041B0C1380BA
:10D8F00018B12A2200238271C37103224A2109F040
:10D90000F1FE20680AF072F8D9E716F04DF9237895
:10D91000D1E700BF8846002074340020783400200E
:10D92000D8460020064B53F820302BB11A689B884C
:10D9300051690B4201D1138370475383704700BF75
:10D9400024AA00202DE9F04FBC4B1E788BB0002E8E
:10D9500040F08180BA4BBB4C1D78BB4FDFF80CB355
:10D9600005F00105A4F10A0954F80A0CB8B14FF00A
:10D97000CC0808FB0698FFF75FFF80B154F80A0C4B
:10D98000FFF752FF14F8023C024683B924283BD02B
:10D9900075B354F80A0CFFF74FFF0028EED101369B
:10D9A000032E04F1CC04DFD10BB0BDE8F08F012BC6
:10D9B0002ED0022B33D0032B40D0042B00F06981F2
:10D9C000052B00F05781062BE3D114F801ECBEF1D2
:10D9D000000F00F0D881BEF1010F00F01B8201366C
:10D9E0000023032E04F8023C04F1CC04BCD1DBE795
:10D9F000232A54F80A0C00F08281944B93F83230B9
:10DA00009342B8D1FCF788FD012304F8023CC0E73B
:10DA10004D2800F06781002304F8023CB9E7002399
:10DA20003C2804F8023C00F057813E28B1D1012285
:10DA3000032304F8012C04F8023CAAE7C028EAD822
:10DA40000021042304F8050C04F8040C04F8061C57
:10DA500004F8023C9DE77E4B18680028A4D00AF029
:10DA600037F9DFF80CA27B4DDFF8F891DAF8000007
:10DA7000FFF7E2FE002897D0DAF80000FFF7D4FEA7
:10DA800009281BD03F2819D02B68002B67D1042808
:10DA900000F0BA810C2800F0CA807F28E6D0A0F1FF
:10DAA0002002D2B25E2AE1D80BB92028DED05A1C5F
:10DAB00009F803002A6016F02FFDD7E72C68002C28
:10DAC0005AD1654FA34607F52478BBF1000F08BF74
:10DAD000BB4610374745F8D1BBF1000F00F04E812F
:10DAE000103FDBF800003A68065D135D9E4220445B
:10DAF00002EB040140F04081661E4E4422460BB901
:10DB0000FD2A5CD906F8013F01322A6010F8013F76
:10DB100011F801EF9E45F2D00AB15F4512D04F488F
:10DB200016F002FD5F4508D35BF8100B16F0FCFC05
:10DB3000092016F0F1FCBB45F6D9494816F0F4FC73
:10DB40002A680024944291D2661E4E4416F8010FB2
:10DB500016F0E2FC2B6801349C42F7D386E70C28D0
:10DB600065D00A2834D00D2832D07F2800F0BE803E
:10DB7000FF2B3FF67BAF92E7374E002706F5247860
:10DB8000BB4602E0103646450DD022463168484675
:10DB90000AF0FCFB0028F5D1B346002FF2D137463E
:10DBA00010364645F1D13B465F469B46002B98D147
:10DBB000002F3FF45BAF294816F0B6FCB4E7511CC8
:10DBC000202009F80200296009F801300A46A4E77C
:10DBD00016F02BFD2321234836F012FE002800F01A
:10DBE0001181A0EB0900286090B1431E19F80310C1
:10DBF000202940F02C8109EB030243B112F8011DEA
:10DC0000202903F1FF304FD10346002BF6D12B60C2
:10DC10004FF480720021484636F0DBFD074B1B783D
:10DC2000002B3FF4C1AE0E4816F07EFC1EE70E48F6
:10DC300016F07AFC0A4816F077FC17E7FE5300202E
:10DC4000708200200EC80020E0280020509500209F
:10DC5000902F00209430002074500408247E040883
:10DC60002C7E0408942F0020347E040810490408F8
:10DC70008C2F002014F8063C14F8051C99426FD82C
:10DC800014F8043C83427FF4C6AE062304F8023C39
:10DC90009BE614F8043C04F8030C5A40052304F8EE
:10DCA000042C04F8023C74E62B606A4C002204F554
:10DCB000247809F8032002E0103444454CD0216850
:10DCC000484611F035FE0028F6D0444544D2E368BA
:10DCD000984700232B609BE7032204F8013C04F8DB
:10DCE000022C56E6022304F8023C52E6013B0022D5
:10DCF00059482B6009F8032016F016FCB6E6574B7E
:10DD00005749DB78574ADFF888E11060003318BFC5
:10DD100001230B70544B554ACEF80030544B3A61F6
:10DD20004FF0400E012187F818E0F86078617D76A9
:10DD30005048197017F09EFA4F4816F0F5FB4FF453
:10DD4000006008F0B9FE4D4B93F83230232B3FF4BE
:10DD500059AE14F8023C36E6494816F0E5FBB8E740
:10DD600014F8041C08EB03005140013304F8041CB0
:10DD700004F8063C82720CE62246CDE64148103F8C
:10DD800016F0D2FBD0E69BE80F000DF1280C0DF148
:10DD9000080888E80F004CF824ED14F8053C14F846
:10DDA00003AC0694624623444FF0010C414606A89A
:10DDB000ADF822E00793ADF820A08DF824C000F064
:10DDC00069F840B1029A304B03924146A4F10A002F
:10DDD000029312F061FEDDF80480002304F8023C97
:10DDE000B8F1000F3FF4DBAD54F80A0C12F014FF49
:10DDF000013654F80A0CC047032E04F1CC047FF41A
:10DE0000B3ADD1E52868EFE6204811F0F7F80BB084
:10DE1000BDE8F08F14F8053C14F8032C0694234455
:10DE200007936E2A4FF0000308930993ADF8202062
:10DE30007FF4D5AD06A80AF028FB06A80AF01AFB65
:10DE400006A80AF017FB06A80AF014FBC7E503466C
:10DE50002BE700BF745004085C7E04084073002068
:10DE6000D83400208C2F0020F028002001BE0008AC
:10DE7000FE530020607E04082C7E0408509500208C
:10DE8000407E0408247E040878D40020942F0020CB
:10DE9000902F00202DE9F04F9BB0B0F908500D8174
:10DEA000EDB2442D00AF0C46904600F0838206464A
:10DEB00043D9812D00F0C48200F29980542D00F0E6
:10DEC000CE8040F20E826E2D00F04282802D40F016
:10DED00024819F4B93F800A00AF1020A1AF0FF0A6E
:10DEE00000F099809B4BDFF8A0829B4EDFF89CB23C
:10DEF0009A4403F101090A2516E0322D00F002864A
:10DF0000A5F13C00C0B2132840F205860023226828
:10DF1000511C216015702268D14502F10101216078
:10DF2000137078D019F8015B0A2DE6D1BBF80030E8
:10DF3000FF2BA8BFFF23DBB2E9E7052D00F0288205
:10DF400020D8022D00F0838040F2B881032D00F02C
:10DF5000F481042D40F0E1802A46804920460AF0F1
:10DF600099FA002120460AF0DAFA22680221531CAD
:10DF70000125236028462B466C3711706381BD460E
:10DF8000BDE8F08F242D60D040F24E81282D00F0A6
:10DF90001982382D40F0C1800A68714B0125511C4F
:10DFA00021601570226805215019206011702268C7
:10DFB0000A21501920601170226800215019206038
:10DFC00011702268197850192060117022685978F0
:10DFD00050192060117022689978531923602B46DC
:10DFE000117028466C376381BD46BDE8F08FA02DC7
:10DFF00019D040F23881B82D00F02082FE2D40F07B
:10E000008C80584D05F1080635F8021B20460AF0B1
:10E0100086FAB542F8D101252B4628466C37638134
:10E02000BD46BDE8F08F504B084619680AF060FA0B
:10E030004E4B204619680AF05BFA4D4B1968204692
:10E0400001250AF055FA2B46E7E74A4BF6E704228A
:10E050004949204601250AF01DFA2B46C1E70B6805
:10E06000464ADFF82C81581C112120601970236862
:10E070001278591C21601A70236898F85520591C91
:10E0800021601A70236898F85420591C21601A7076
:10E09000B8F8501020460AF042FA23680022591CB2
:10E0A00021601A7023682822591C21601A70B8F860
:10E0B000521020460AF033FAA8F1020508F14E0684
:10E0C00035F8021F20460AF02AFAB542F8D1226834
:10E0D0002B4B0D21501C20605D181170226813F825
:10E0E000011F501CAB4220601170F7D1236802223F
:10E0F000591C21601A70B8F8561020460AF00FFA21
:10E10000B8F8581020460AF00AFA0125B8F85A1053
:10E1100020460AF004FA2B4663E72146284607F01A
:10E12000E7FB034600287FF476AF742D00F0F780FC
:10E13000772D2FD13268716891421EBF531C336016
:10E140001178104A08BF1946204632F0A7FD62E751
:10E15000C5820020204904080834002046730020AE
:10E1600001550020E48D0020107AFF1F147AFF1F54
:10E17000187AFF1F6C560020987E0408F08D00204E
:10E18000A95E0020A5010408676666663034002099
:10E190004C5E0020F52D00F0B585762D00F09782BD
:10E1A000472D00F0E98470683268A5F12103811AD7
:10E1B000362B00F2BF82DFE813F06B02BD02BD0216
:10E1C000BD02BD02BD02BD02BD020E02BD02BD0206
:10E1D000BD02BD02BD02BD02BD02BD02BD02BD0247
:10E1E000BD02BD02BD02BD02BD025B02BD02BD0299
:10E1F000BD02BD02BD02BD02BD02BD02BD02BD0227
:10E20000BD02BD02BD02BD02BD02BD02BD02BD0216
:10E21000BD02BD02BD02BD02BD02BD02BD0226029D
:10E22000BD02E801BD02D301202D7FF476AF0B685B
:10E23000B74D591C6A7821601A7023682A78591CD6
:10E2400021601A702368AA78591C21601A702989E4
:10E2500020460AF064F923686A79591C21601A7013
:10E260002268A97983E6822D7FF457AF0B68A94A0B
:10E27000A94D1178A64A581C2060197011892046B2
:10E280000AF04DF9A54B22681B88FF2B02F1010112
:10E29000A8BFFF2321601370A96881F3100189B220
:10E2A00020460AF03CF9296801F30F0189B22046A3
:10E2B0000AF035F99A4B2268197858E6012D7FF457
:10E2C0002CAF0B680022591C21601A7023685A1C5D
:10E2D00022601D7022682521531C23602B4611707B
:10E2E0007FE6522D7FF419AF0A688E4D531C03212F
:10E2F000236005F10C0E2B461170062601202268C2
:10E30000511C216010702268734502F101012160E7
:10E31000167000F0DE809879DE790633EFE7326818
:10E32000716891421EBF531C336011787E4A08BF4A
:10E330001946204632F0B2FC6DE60B685A1C0A60A2
:10E340001D700B685A1C0A601D70226800210EE6C1
:10E35000724B0A681B88704DFF2BA8BFFF23511C0E
:10E3600021601370A96881F3100189B220460AF078
:10E37000D6F86E4B204619880AF0D1F8296801F3C7
:10E380000F0189B2204601250AF0C9F82B4628E67C
:10E390000B22674920460AF07DF80822654920468D
:10E3A0000AF078F801250722634920460AF072F83E
:10E3B0002B4616E6002A3FF42EAE604B1360012573
:10E3C0002B460EE60B68DFF890915D4E591C022239
:10E3D00021601A7023684FF006085A1C226083F8E7
:10E3E000008023680A22591C21601A7023680125C5
:10E3F0005A1922601D70B9F8001020460AF08FF8F3
:10E40000B9F8021020460AF08AF823685A192260E7
:10E4100083F8008023685022591921601A702368FC
:10E420000022591921601A70318820460AF077F8C5
:10E43000718820460AF073F82B46D2E5414BFDE582
:10E44000414B1E78033616F0FF063FF4E4AD3F4B18
:10E45000DFF808811E4403F1010A4FF00A0920E0A9
:10E46000B9F1500F00F05583B9F1320F00F0698314
:10E47000A9F13C00C0B2132840F26683002529466A
:10E4800023685A1C2260204683F800900AF047F85F
:10E49000294620460AF043F8B2453FF4BCAD1AF8CD
:10E4A000019BB9F10A0FDBD1294B9D68196805EB77
:10E4B00085054FF6FF736D009D42A8BF1D4699422A
:10E4C000A8BF194625EAE57521EAE171ADB289B226
:10E4D000D6E7204B21681A78481C20600A70002A71
:10E4E0003FF499AD013AD2B202EB420205EB42028F
:10E4F0005278002A3FF48FAD0132D51801332268DB
:10E5000013F8011F501C9D4220601170F7D182E565
:10E5100064A50020F28300204CA50020DC830020AD
:10E52000B85E00205067040809020408A4600020B7
:10E53000A07E0408AC7E0408B87E040835560108A5
:10E54000F033002098300020C582002030490408B4
:10E55000BC33002084950020E8A700200034002070
:10E56000531C336012F8370B07F127010133336076
:10E5700013F8015C01F8015F9342F7D107F128011C
:10E580000125FBF74BFB2B462BE5531C336092F820
:10E590000080B8F1FF0F00F04385B8F1FE0F00F0E6
:10E5A0002785304609F066FF33687268D21A002A60
:10E5B00007DD5A1C32601B781BB9B8F10C0F40F212
:10E5C0005C85B8F1270F00F28684534B012523F8B0
:10E5D00018002B4605E5531C336013780A2B00F016
:10E5E000B784502B40F0AC84304609F043FFDFF88D
:10E5F0004081A8F80000304609F03CFF0125A8F84A
:10E6000002002B46EDE4531C33601078032800F21F
:10E610006284431E414D424ADBB203EB430305EBE8
:10E62000430310705D7800283FF4F5AC4B1EDBB25D
:10E63000AB4240F050840021C2F80610C2F802102C
:10E6400091725BB1581C336810440132013333605E
:10E6500013F8011C02F8011F9042F7D1314B1B78CF
:10E66000002B3FF4D8AC01252CF056FC2B46B8E427
:10E67000531C336013780A2B00F0A084304609F055
:10E6800004FF304609F001FF304609F0FEFEC2E407
:10E690001346511C3160244D13F8021B697033601E
:10E6A00053782B70D31C33609378AB70304609F0ED
:10E6B000E1FE33682881591C1A46316012F8021BAA
:10E6C000697132605B78AB7101252B4689E4326851
:10E6D000511C31601278002A00F04184102A00F0A9
:10E6E0009A84124D1E4619462368581C20601A70E1
:10E6F000204609F0FDFE3146204609F0F9FEE968A2
:10E70000204609F0F5FE2046002109F008FF00210F
:10E71000204609F004FF18E64C5E0020506704080C
:10E72000849500206934002064A500204029002041
:10E73000F03300200B3DEF2D00F2CD8301A353F801
:10E7400025F000BF63FE0008D7EE0008D7EE0008F2
:10E75000D7EE0008D7EE0008D7EE0008D7EE000885
:10E76000D7EE0008D7EE0008D7EE0008D7EE000875
:10E77000D7EE0008D7EE0008D7EE0008D7EE000865
:10E78000D7EE0008D7EE0008D7EE0008D7EE000855
:10E79000D7EE0008D7EE0008D7EE0008D7EE000845
:10E7A000D7EE000809FE0008D7EE0008E7FD0008D4
:10E7B000D7EE0008BDFD0008D7EE0008D7EE000830
:10E7C000D7EE000895FD0008D7EE0008E5FC00082C
:10E7D000D7EE0008B3FC0008D7EE00088DFC000857
:10E7E000D7EE00087BFC0008D7EE000823FC0008E9
:10E7F000D7EE000889EE0008D7EE0008D7EE000833
:10E80000D7EE0008D7EE000817E00008D7EE0008A2
:10E8100061FB0008D7EE0008D7EE000847FB0008B0
:10E82000D7EE0008F7EE0008D7EE0008D7EE000894
:10E83000D7EE0008D7EE00083BFB0008D7EE000833
:10E84000D7EE0008D7EE0008FBFA0008D7EE000864
:10E85000F5F90008D7EE0008D7EE0008B5F9000872
:10E86000D7EE0008D7EE0008D7EE0008D7EE000874
:10E87000D7EE0008D7EE0008D7EE00085BFA0008D4
:10E88000D7EE000833F90008D7EE000879F8000841
:10E89000D7EE000887F70008D7EE00085FF70008FA
:10E8A00041F700080BF70008D7EE0008D7EE000884
:10E8B000D7EE0008D7EE0008D7EE0008D7EE000824
:10E8C000D7EE0008D7EE0008D7EE0008D7EE000814
:10E8D000D7EE0008D7EE0008D7EE0008D7EE000804
:10E8E000D7EE0008D7EE0008D7EE0008D7EE0008F4
:10E8F000D7EE0008D7EE0008D7EE0008D7EE0008E4
:10E90000D7EE0008D7EE0008D7EE0008D7EE0008D3
:10E91000D7EE0008D7EE0008D7EE0008D7EE0008C3
:10E92000D7EE0008D7EE0008D7EE0008D7EE0008B3
:10E93000D7EE0008D7EE0008D7EE0008D7EE0008A3
:10E94000D7EE0008D7EE0008D7EE0008D7EE000893
:10E95000D7EE0008D7EE0008D7EE0008D7EE000883
:10E96000D7EE0008D7EE0008D7EE0008D7EE000873
:10E97000D7EE0008D7EE0008D7EE0008D7EE000863
:10E98000D7EE0008D7EE0008D7EE0008D7EE000853
:10E99000D7EE0008D7EE0008D7EE0008D7EE000843
:10E9A000D7EE0008D7EE0008D7EE0008D7EE000833
:10E9B000D7EE0008D7EE0008D7EE0008D7EE000823
:10E9C000D7EE0008D7EE0008D7EE0008D7EE000813
:10E9D000D7EE0008D7EE0008D7EE0008D7EE000803
:10E9E000D7EE0008D7EE0008D7EE0008D7EE0008F3
:10E9F000D7EE0008E5F60008D7EE0008C1F60008DB
:10EA00009BF60008D7EE0008D7EE0008D7EE000806
:10EA1000D7EE0008D7EE0008D7EE0008D7EE0008C2
:10EA2000D7EE0008D7EE0008D7EE0008D7EE0008B2
:10EA3000D7EE0008D7EE000833F60008E3F500082B
:10EA4000ABF50008D7EE000809F500089DF40008B2
:10EA500081F40008D7EE000867F40008D1F300083D
:10EA600095F0000847EF0008B3F20008D7EE000861
:10EA700083F20008D7EE0008D7EE000859F200082C
:10EA80002BF2000817F20008EFF10008CFF10008A0
:10EA9000A5F1000835F10008D7EE0008D7EE000810
:10EAA000D7EE0008D7EE0008D7EE0008D7EE000832
:10EAB000D7EE0008D7EE0008D7EE0008D7EE000822
:10EAC000D7EE0008D7EE0008D7EE0008D7EE000812
:10EAD000D7EE000815F10008D7EE0008D7EE0008C1
:10EAE00077F30008D7EE0008D7EE0008D7EE00084D
:10EAF00013F30008D7EE0008D7EE0008D7EE0008A1
:10EB0000BBF000083388FF2BA8BFFF23DBB2FFF761
:10EB1000FEB9BE4BC9E428F015FF00283FF4F6A962
:10EB200003780A2B26D8B0F9023088FB0312DB17D2
:10EB3000C3EBA2039BB2FF2BA8BFFF23DBB2FFF7FF
:10EB4000E6B998E82200B2E428F0FCFE00283FF481
:10EB500095AC03780A2B3FF691ACB0F90430B0F9CC
:10EB6000061003EB830383F3500521EAE171ADB294
:10EB700089B285E40023E1E7726835687B6230463C
:10EB8000551B09F060FC052D38627B6A00F26F812D
:10EB90008026B346012594E80600521A103AB24284
:10EBA000B8BF1FFA82FB9A4A396A92683A61521AD0
:10EBB0009345396A7B622046FA6088BF1FFA82FB60
:10EBC00009F096FC7B6A002B00F03081002D40F0AC
:10EBD000F6802368C7F800D05D71C0B00533C7F870
:10EBE00004D0FB61BBF1000F00F077823B6A3A6909
:10EBF000934280F06F823E6A7D62AA46A846BC605E
:10EC00008025FB68A3EB0808814BB8F5807F9B68E3
:10EC100028BF4FF4807808EB06029A4288BFA3EB26
:10EC200006080AF0B5FA7C684246214630460AF0EA
:10EC300035FBF969B86104EB000C0B787B61644526
:10EC40002ED2DFF8E0910CF1FF3C04F1FF3E1EF8FC
:10EC5000013F09EB830219F823405688ECB10023E9
:10EC60004FF4004204F1FF3832424FEA520202D020
:10EC70000878284308706D0806D10AF1010A4D7022
:10EC80001FFA8AFA01318025D34503D8E64533D3EC
:10EC9000434531DB01339C42E6D1E645D7D1F961EA
:10ECA0007B6ABA6913449BB2D3457B6206D97B6AFF
:10ECB0003A6A9846D6183B699E42A2D3BC68802D1A
:10ECC0001CBF0AF101031FFA83FA0AF1020189B29B
:10ECD000204609F024FC2368796A01255A1922602C
:10ECE00020461D7009F01BFC2368534423602B460B
:10ECF000D7F800D0FFF775B9FB69BC681A463B7DB1
:10ED00001370DCE7336872689A4240F02E81414B01
:10ED1000FF221A704FF0000A3F4D23F04DFD51467F
:10ED200020223E4885F800A035F053FD87F828A042
:10ED300097F82830072B00F2AB81DFF8EC90374EC4
:10ED4000524697F8283003EB430309EBC3035B7C7F
:10ED5000E3B197F8283003EB430309EBC303202109
:10ED60005B699BB197F8283003EB430309EBC303BE
:10ED7000586946F8220008F081FD2B7856F82300E8
:10ED800008F039FE2A780132D2B22A7097F828307A
:10ED90000133DBB287F8283097F82830072BD0D919
:10EDA0002368591C21601A70B8F1000F3FF433A991
:10EDB0001B4BC8F8003001252B46FFF712B9144B46
:10EDC0003A6A9B68D4F800905A449A4240F288808C
:10EDD0003A6AA3EB02080AF0DBF942464946386A70
:10EDE0000AF05CFA236803442360002D3FF413A962
:10EDF000B042BFF610A9002100E0236801305A1C80
:10EE0000B04222601970F8D1FFF705B9F433002041
:10EE1000E81D0020402900202B510020E04F002059
:10EE2000FD78020840490408647D0020002DC6D109
:10EE30005946204609F073FB23685A1C22601D7056
:10EE4000C74B26689D683B6A0BEB03029542C0F0F6
:10EE500048810AF09DF95A463146386A0AF01EFA8E
:10EE600023680125034423602B46FFF7BAB83046D8
:10EE700009F000FB326871687B6A9142834640F07A
:10EE8000AE8006461D4686E60723B1FBF3F3C3EBCF
:10EE9000C300091A1FD1DBB203F1FF3A5FFA8AFA05
:10EEA000002B3FF4B8A8DFF8BCB20AF1010A0D4606
:10EEB000531C336092F90020AA4B4FF0000893F9DD
:10EEC0000210914203F1080300F0868608F1010860
:10EED000B8F1060FF3D14FF0FF352B46FFF781B89D
:10EEE0000AF056F95A464946386A0AF0D7F92368B3
:10EEF000034423607CE7531C33609B4B1278DFF89C
:10EF000098821A700023C8F80030304609F09BFA46
:10EF10003368D8F800209549954D10435A1CC8F81D
:10EF2000000032601B780B72304609F0A3FA2860AB
:10EF3000304609F09FFA6860304609F09BFAA860F5
:10EF4000304609F097FA304609F094FAFFF763B8B3
:10EF5000304609F08FFADFF84482FFF74ABB854B51
:10EF6000854D93E84200FFF7BFBB5A1C194632603B
:10EF7000814811F8022B027031605B784370042ADB
:10EF800003D9FF2A7FF4E1A9C4E67C4909789942B4
:10EF900005D8022A7FF4D9A9FF2B7FF4D6A92368CC
:10EFA00001255A1922601D70B8F1000F3FF433A8F3
:10EFB000734BC8F800302B46FFF713B8931C33602F
:10EFC000704B51781970D11C316091785970111DB6
:10EFD0003160D2789A7001252B46FFF702B8511C98
:10EFE000316012781D46131C064618BF0123D2E576
:10EFF000931C33605578022D3FF66DAF304609F013
:10F0000039FA614B03EB45034FF0FF35A3F8560087
:10F010002B46FEF7E6BF584D6968AE68FFF764BB44
:10F02000931C3360594B51781970D31C3360DFF84F
:10F030005881937888F85530131D3360D37888F859
:10F040005430304609F016FAA8F85000304609F05E
:10F0500011FA304609F00EFA96E80C009B1A012BC3
:10F06000A8F852007EF7D7AF304609F003FA012521
:10F07000A8F85A002B46FEF7B4BF434B0030984423
:10F0800018BF0120012588F85E002B46FEF7A9BFB6
:10F09000524685E6531C3360107806062FD43C4B4D
:10F0A0001B78DD073EF5B7AF032828BF00200125F8
:10F0B000FDF71EF82B46FEF794BF354B1B78DB0798
:10F0C0003FF509AF0125FDF72FF8FDF7DFF82B46D7
:10F0D000FEF787BF7D62AA46F7E5DA46C7F824B097
:10F0E000F3E53B6AED1A0AF053F82A463146386ACE
:10F0F0000AF0D4F8236803442360FEF78CBF00F0C5
:10F100007F00032828BF0020012524F01FFD2B4687
:10F11000FEF767BF304609F0ADF9DFF88480A8F844
:10F120000E00304609F0A6F90125A8F80C002B4680
:10F13000FEF757BF1146531C3360164B11F8020BF4
:10F140001870316051785970D11C31609178997084
:10F15000111D3160D278DA7001252B46FEF741BFD0
:10F16000E81D002050950020A45A0020249500207E
:10F17000BC4600206871002040290020C582002084
:10F1800041560108015500204C5E0020F08D002002
:10F1900070820020646F00206C560020E8A70020D9
:10F1A000F8A70020304609F065F9DFF84C83A8F88D
:10F1B0001000304609F05EF9A8F81200304609F058
:10F1C00059F90125A8F814002B46FEF70ABF13468B
:10F1D000511C316013F8020B3360D31C517833603B
:10F1E00092781FF005FD00287EF415AF73E61346F4
:10F1F000511C3160B04913F8020B08703360AF49FD
:10F2000053788B70D31C3360AD4B92789A70012584
:10F210002B46FEF7E6BEAB4BAB4918684E220125E4
:10F2200034F044F92B46FEF7DCBE1146531C336024
:10F23000A64B11F8020B1870316051785970D11C2F
:10F24000316092789A70304609F014F9A04B01258C
:10F25000D8802B46FEF7C5BE304609F00BF9DFF823
:10F260007082A8F80000304609F004F9A8F80200FE
:10F27000304609F0FFF80125A8F804002B46FEF7F8
:10F28000B0BEDFF8789299F80030002B3EF4C3AEA0
:10F29000DFF86C820025304609F0ECF814F070FBC2
:10F2A00099F80030A8EC010A01359D42F3DBFEF726
:10F2B000B2BE0D297FF40FAE531C33601578072DB5
:10F2C0003FF609AEDFF83C9230464FF00C0809F0EB
:10F2D000D1F808FB05F809EB0805A880304609F0CD
:10F2E000C9F8E880304609F0C5F8336828811A4625
:10F2F000591C316012F8021BA97232605B78EB7204
:10F30000304609F0A0F8012549F808002B46FEF721
:10F3100068BE304609F0AEF8336838851A46591C85
:10F32000316012F8021B326087F82A105A7887F889
:10F330002B20DA1C32609A7887F82C201A1D326054
:10F34000DA7887F82D205A1D32601B7987F82E3025
:10F3500007F1280000233B8608F0E6FF5D4A5E4B7C
:10F360001268801A4FF0010561F10001C3E906013E
:10F370002B46FEF736BE531C336013780F2B3FF637
:10F38000AAAD911C3160C3EBC30354495078C854F3
:10F39000D01C30600B4491785970111D3160D178C8
:10F3A0009970511D31601179D970911D3160517979
:10F3B0001971D11D31609179597102F108013160E3
:10F3C000D2799A71012513F063FD2B46FEF709BE31
:10F3D000531C3360304692F800A009F034F881469F
:10F3E000304609F030F80546304609F02CF88046E2
:10F3F000304609F03FF8304609F03CF8304609F055
:10F4000044F8BAF1000F17D0BAF1100F7EF403AE32
:10F41000314BC3F804909D60B8F1000F01D0C3F8E0
:10F420000C802F492F4B0222081F01251A7019F05A
:10F43000FFFC2B46FEF7D5BD2B4B1020C3F80090E8
:10F440005D6007F009FB294A137843F0010313704C
:10F45000B8F1000F3EF4DFAD1F4B0125C3F80C805F
:10F460002B46FEF7BEBD224B1B78D8073EF5D3AD29
:10F470000125FDF7D9F8FCF709FF2B46FEF7B1BDD2
:10F480001B4B1B78DA073EF5C6AD184A13780125E9
:10F4900043F0040313702B46FEF7A3BD144B1B78F7
:10F4A000D9073EF5B8AD134B4FF4C87201251A8049
:10F4B0002B46FEF796BD00BF007C0020F8A7002079
:10F4C00008A80020CCA50020FC680408F0A70020B4
:10F4D0007C4D002058AA00204029002064310020E3
:10F4E000482900207471002068710020CAA50020FE
:10F4F000708200206ED40020247E0020C58200206F
:10F500006C2F0020A430002009297FF7E4ACDFF83D
:10F5100060831346511CD8F80050316013F8021B69
:10F52000297033605378AB70D31C33609378642BAD
:10F5300002F10401A8BF64236B713160D378642B9E
:10F5400002F10501A8BF6423AB7131601379EB713F
:10F55000931D33605379642B02F10701A8BF642324
:10F560002B7231609379EB7002F108033360D37929
:10F570002B71304608F07EFF726833686881D11ABB
:10F5800000290CDD591CD8F800003160521A002AFD
:10F590001978417203DD9A1C32605B784370012553
:10F5A00032F046FC2B46FEF71CBDA24B1868D31C5C
:10F5B000014621329D1E356013F8035C0D705D1EFF
:10F5C000356013F8025C4D70336013F8015C8D7088
:10F5D00003339A4201F10301ECD114F07BF8FEF7FA
:10F5E0001ABD531C336013789349002B46D00B7817
:10F5F00043F00203901C0B70904D306053782B75D4
:10F60000304608F020FF2860304608F01CFF686094
:10F61000304608F02FFF2881304608F02BFF884A3B
:10F62000E8811378012543F0020313702B46FEF79F
:10F63000D8BCC1F34705122D3FF64DAC15B307F109
:10F64000680307F1260A03EB4508D146A8F14208F2
:10F65000304608F00FFF29F8020FC845F8D1794B62
:10F660003AF8022F23F8022FD145F9D1112D09D9EB
:10F67000754A01231D461370FEF7B3BC0B7803F0E7
:10F68000FD03B7E7714A6B00023B134400212232AD
:10F6900023F8021F9A42FBD1EAE7531C6C483360FF
:10F6A00001781378D1B9042202706A4A9B00138052
:10F6B000FDF788FD684B012518622B46FEF791BCCB
:10F6C000DFF8B08100233046C8F8003008F0BBFEF8
:10F6D0000125C8F800002B46FEF783BC04297EF400
:10F6E0009AACE2E71346511C316013F8025B3360B9
:10F6F000D31C5078336091789DB1012D7EF48BAC92
:10F7000024F008FA2B46FEF76CBC531C33601378C8
:10F710006BB14FF40040012507F0CEF92B46FEF700
:10F7200060BC012513F05AFE2B46FEF75ABC4B4A2B
:10F730001368012523F4004313602B46FEF751BCE8
:10F74000474B1B7813F001017FF4C5AB531C3360AA
:10F750001078012524F024F92B46FEF742BC13460D
:10F76000511C31603F4913F8020BC87033603E49A9
:10F7700053784B71D31C33603C4B9278DA7001257F
:10F780002B46FEF72EBC304608F074FE304608F0DB
:10F7900071FE304608F06EFE304608F076FE3368A3
:10F7A000244D1946581C2A68306011F8020B82F863
:10F7B0002C003160597882F83610D91C31609B7862
:10F7C00082F83730304608F060FE304608F05DFEC3
:10F7D000304608F05AFE3046D5F8008008F04AFE60
:10F7E000A8F83A003046D5F8008008F043FE3368A8
:10F7F0007268A8F83800D11A01290ADD591C2A6854
:10F8000031601B7882F82E30304608F03EFE3368B7
:10F810007268D31A032B0BDD3046D5F8008008F050
:10F8200029FEA8F8320030462E6808F023FEB08684
:10F830002868D2E6CCA50020CAA500203CAD002057
:10F8400072710020DE4E0020044F0020E04E0020A8
:10F8500096A30020A460002040290020C4A5002019
:10F8600070820020F8A7002090A7002008A80020A0
:10F87000D0A5002098300020531C3360C34DDFF822
:10F880004C83137888F805303046D5F8009008F09E
:10F89000F1FDA9F820003046D5F8009008F0EAFD07
:10F8A00072683368A9F81E00D11A072919DD30469D
:10F8B00008F0E0FDA8F80A00304608F0DBFDA8F8E3
:10F8C0000C003046D5F8009008F0D4FDA9F82200CD
:10F8D0003046D5F8009008F0CDFD33687268A9F87D
:10F8E0002400D11A03290BDD304608F0C3FDA8F827
:10F8F0000E00304608F0BEFD33687268A8F81000AC
:10F90000D21A002A05DD591C2A6831601B7882F85A
:10F910002630FCF713FC24F0B3FB9D4B28681B68D2
:10F92000002B00F0D080012513F048FB2B46FEF79A
:10F9300058BB1346511C3160DFF8908213F8021B4C
:10F9400088F802103360934953780B70D31C3360EE
:10F95000914D93782B71131D3360D378092BA8BF79
:10F9600009233046AB7008F085FD33687268288043
:10F97000D11A012905DD304608F07CFD3368726834
:10F98000E8819A4207D05A1C32601B78003318BFB6
:10F99000012388F80730FCF7D1FB336872689A427C
:10F9A0003EF439AB5A1C32601B78EB7001252B46B4
:10F9B000FEF717BB794B1B78012B3EF62CAB11469B
:10F9C000531C3360DFF8088211F8023B88F80230DC
:10F9D0003160D31C92F801E03360C31A012B917897
:10F9E0002FDD304608F046FD0125A8F800002B4623
:10F9F000FEF7F7BA531C336092F80080B8F1110F8C
:10FA00003FF669AA931C3360654D537805F81830AA
:10FA1000304608F02FFD40F6CA039842A8BF1846AA
:10FA200040F2EE23984205EB4801B8BF1846012585
:10FA3000A0F2EE222B46192092FBF0F24A70FEF75C
:10FA4000D0BA584B1A88012512FB0EF22B4692FBB6
:10FA5000F1F2A8F80020FEF7C4BA534B1B68002B44
:10FA60003EF4D9AA19F0DCFAFF283EF4D4AA3046B5
:10FA700008F000FD3F2831D9DFF85881002588F8CB
:10FA8000005033687268A8F80400D21A012A7EF781
:10FA9000C2AA1A46591C316012F8021B88F80210DB
:10FAA00007F16800326000225D7800F8402D19F0FF
:10FAB00089FA97F82830AB423EF4ADAA284619F0EF
:10FAC000A5FAFEF7A8BA394839493A4A3A4B0360D1
:10FAD00001250B6013602B46FEF783BAC50800F0C2
:10FAE000070301350133EDB2DFF8E88028461946F7
:10FAF00088F8013027F090FEC1E71346511C2F4DC6
:10FB0000316013F8021B2971336053786B713046F2
:10FB100008F0B0FC336828805A1C32601B78AB7147
:10FB2000304608F0A7FC336868805A1C32601B78A6
:10FB3000EB7101252B46FEF754BA012509F08AFB2B
:10FB40002B46FEF74EBA1E4B02F10801013232601D
:10FB500012F8010C03F8010F9142F7D1FEF75BBADE
:10FB60001346511C3160174913F8025B8D703360E6
:10FB700055784D7083423EF44EAAD31C3360124B2D
:10FB800092781A7501252B46FEF72BBACCA50020DA
:10FB9000A05A0020ECA70020247E00205856002008
:10FBA00074510020C8A70020748200202048002043
:10FBB00074480020744C00209F700108944D002070
:10FBC0002395002018A8002040290020007C002058
:10FBD000806D0020788200200BEBC809304689F840
:10FBE000022008F047FC33682BF838001A46591CED
:10FBF000316012F8021B89F8031032605A7889F8D4
:10FC00000420DA1C32609A7889F806201A1D3260C6
:10FC10000135DB7889F80530AA457FF449A9FEF75C
:10FC2000FAB9531C336013780E2B3FF654A9911C7C
:10FC300031605578032D3FF64EA99748062101FB08
:10FC400003F1431802F1030E5D71C6F800E09578E8
:10FC50004554111D3160D1785970511D31601179B1
:10FC60009970911D31605179D970D11D31609279AF
:10FC70001A7101252B46FEF7B4B9531C3360874B2C
:10FC800012785A7501252B46FEF7ABB9531C336029
:10FC900015781F2D3FF61FA905297FF41CA93046B2
:10FCA00008F0D1FB7E4B43F8250021F015F9FEF753
:10FCB000B2B97B4D05F14008304608F0DBFB3368F4
:10FCC000A5F88000591C1A46316012F8021B85F80D
:10FCD000821032605B7885F883300435A845EBD11B
:10FCE000FEF799B9531C6D4D336013782B72304673
:10FCF00008F0C0FBA883304608F0BCFB28833046E0
:10FD000008F0B8FB32686883531C33601278EA74D9
:10FD10007268D31A032B1FDC3368D11A05290EDD54
:10FD20005A1C32601B78EB72304608F08CFB33684B
:10FD3000E8605A1C32601B782B7433687268D21AE0
:10FD4000002A7EF768A95A1C32601B7885F821309A
:10FD500001252B46FEF745B9304608F08BFBA884F9
:10FD6000304608F087FB33687268E884D11A0329AB
:10FD7000D3DD1A46591C316012F8021BA977326094
:10FD80005B7885F82030304608F074FB3368726881
:10FD90006884C2E7531C3360424915780D70C01A5D
:10FDA00000287EF738A9931C33605378003318BFBE
:10FDB000012301254B702B46FEF713B9304608F09E
:10FDC00059FBDFF8F080C8F80000304608F052FB1D
:10FDD000C8F80400304608F04DFB0125C8F80800BB
:10FDE0002B46FEF7FEB8DFF8D0800023C8F80030BD
:10FDF000304608F028FBD8F8003001250343C8F846
:10FE000000302B46FEF7EDB8531C33601578132DE8
:10FE10003FF661A8931C336050787A6230F078FF27
:10FE200000283FF458A87A6A1F4B017803F8251080
:10FE3000D11C316003EB850391785970111D31603D
:10FE4000D1789970511D31601279DA70002031F04B
:10FE500031FF164B80F00100012518702B46FEF78C
:10FE6000C0B8134B10294FF0000228BF10211A60B0
:10FE70005A609A60DA601A7400293EF4CCA832689D
:10FE8000013B11440132326012F8010C03F8010FFA
:10FE90008A42F7D1FEF7BFB85032002024950020E7
:10FEA000D85E0020A45A00205C500020B42200201C
:10FEB0005A6D0020BC4600206C5600202DE9F04F02
:10FEC0002DED028B93B005462DF090FF994B1E78D7
:10FED00026B113B0BDEC028BBDE8F08F964B1B68CA
:10FEE0005805F6D5DFF89C82D8F80020002A00F0EB
:10FEF0001E81924CD4F8283103F5F43348339D42E7
:10FF0000C0F015818E4F94F82C313968C4F828510F
:10FF10000133DBB2890784F82C3101F1ED8513F050
:10FF2000070901F02B85282B864B029301F02687C9
:10FF30005E209047844B1B78002B6BD07F4C834A0C
:10FF4000D4F83431EB1A934201F2D683DFF838A2A9
:10FF50009AF80080B8F1000F33D1DFF80092D9F899
:10FF60000000FDF769FCC0B201280ED90228784FC5
:10FF700041F0C4873B78002B42F01D81D4F83C311E
:10FF8000EB1AB3F57A6F82F07B8172480768002F15
:10FF900040D09AF80030BBB96F4BD9F800001B680D
:10FFA0009B781E3B012B4FF0020142F2148104307A
:10FFB0002DF0D4FD012200238AF8002084F8483176
:10FFC00026E0644807682FB3D4F8443140F6B732CE
:10FFD000EB1A93421ED994F84031002B01F084872C
:10FFE000013BDBB284F84031002B01F0F28517F8B9
:10FFF000011B94F84821076094F8493157480A4496
:020000040801F1
:100000000133006884F8482184F84931FDF718FC71
:10001000C4F84451524A029B12781B68012A03F12A
:1000200001030A9301F092824E4B1B787BB1DFF8FB
:100030005C81D8F8003053B1029B404CD3F800B03B
:10004000D4F85C31ABEB0303632B01F2BC81DFF826
:10005000408198F800A0BAF1020F01F096853C4F5C
:1000600097F87430032B01F050843F4B1B7873B129
:100070003E4E33685BB1314CFDF7A4F8D4F86831DB
:10008000039044F61F62C31A934200F22581384B55
:100090001B78002B7ED1374B1B7843B1274CD4F80B
:1000A000B83203F50043E8339D4281F0C582324BFC
:1000B0001B78002B3FF40DAF204E304C304D06F234
:1000C000C1272068FDF7B8FB00283FF402AF206885
:1000D000FDF7AAFB2B7880465A1E33B120682A70A0
:1000E000FDF7AAFB0028F2D1F3E603223946781E79
:1000F00034F055FB96F8C03296F8C12286F8C382D8
:1001000083F47F4383F0FF039B1A1FFA88F89BB2A6
:10011000B8EB132FD5D196F8C222DBB29A42D0D1D8
:10012000781E27F08FFC2B7818442870C9E7054B00
:100130000293FFE6FE530020247C0020702900205B
:1001400074A5002058AA00207EA600203F0D0300C1
:1001500020000020E4A50020E0A50020DCA5002070
:100160007FA600208CA6002094A6002098A6002040
:1001700004A7002015A700209EA60020A4A600200A
:10018000A8A60020ECA50020E8A50020B08500204E
:10019000D64F0020444C2278002A41F0CE81DFF86F
:1001A000349199F80040002C72D1404E30780028EC
:1001B00041F08C873E4C3F4ED4F8B02231783E4B14
:1001C00093FBF1F313449D42FFF465AF94F8B4320E
:1001D0003A4AC4F8B052D75CFB0702F16781B8070E
:1001E00002F1B080790702F16D803A0745D5344BB2
:1001F000344F0B930DF14809A3F13D0249F8202D2E
:100200000021A3F1400203F8401C02231121517088
:1002100093704846396808F047F94846796808F00D
:1002200043F9FB89284903EBC3039B00053381FB9A
:100230000321DB17C3EBA10189B2484608F04BF953
:100240003B8A03EB8303590089B2484608F043F91F
:100250001E4B1B789B0743BF398901F57A7189B220
:100260004FF47A71484608F036F90A9B3A7D591CDA
:100270000A9148461A702DF05FFD94F8B432317837
:10028000013393FBF1F201FB123384F8B43202E73D
:100290000F4E376E002F41F02585054B89F8007011
:1002A000C3F8B052F7E600BF70A600200CA70020EC
:1002B0007029002014A70020A086010010A70020AC
:1002C00030A600203CAD002067666666CAA5002007
:1002D0001CA700200DA7002094F86E31002B41F0E0
:1002E0008084DF4B1B6803F00802002A48F60341B4
:1002F0004AF60B404BF60F4249F6074704BF024649
:100300000F4613F0040F4FF0190118BF17469B0654
:1003100084F86E1103D547F4804747F0200710F0AA
:100320009FF9C7F30909002842F0C781CD4B9B799B
:10033000002B42F04F82984664204FF0FF3A4FF076
:10034000000C0A970B97ADF834C0CDF83AC0CDF841
:100350003EC0CDF842C0CDF83090ADF83680ADF853
:1003600038A08DF846000AAF0FCFDFF808E384F815
:1003700005C0AEE80F0097E80F00AEE807002EF8C2
:10038000023B71464FF0010C1B0CFE271F20C822B8
:1003900001F81E39A770A27184F807C0E07094F8C4
:1003A0007E01207180F0F10383EA0313DAB21309AE
:1003B00083F0E70343EA022383EAC2031BB283EA22
:1003C0000312D2B2C3F3072383EA121343EA0223D0
:1003D00083EAC2031BB283F0C80282EA0212D2B2DD
:1003E000C3F3072383EA121343EA022383EAC20317
:1003F0001BB283EA0C0787EA0717FFB2C3F3072291
:1004000082EA171242EA072200EB0C0382EAC707CE
:100410000EEB0C0084F87E31278011F8013B7B4005
:1004200083EA0313DBB21A0982EA172242EA0322A3
:1004300082EAC3031BB29FB281422780EDD183F0D1
:100440007C0383EA0313DBB24FEA131E8EEA172EF6
:100450008EEA032E8EEAC30E0FFA8EFE1FFA8EF975
:10046000DFF814C2A4F800905FFA8EFE4FEA192953
:1004700084F8289084F827E00CF5D37804F1220A58
:10048000DCF80000DCF80410DCF80820DCF80C30A4
:1004900047460FC70CF1100CD445B846F0D1DCF834
:1004A00000003860704F9CF8043088F8043007F181
:1004B000270884F8CDE184F8CE9117F8011F306841
:1004C000FDF7BEF9B845F8D194F86F21002A41F044
:1004D000F4836649029B08781B680A2184F86F112F
:1004E000002801F02C85DFF894E10128BEF8001007
:1004F000059142F2FE810228BEF8028002F0F580EA
:10050000BEF804100491032802F00E820428BEF8FD
:1005100006A002F004820528BEF8087002F0FB81F4
:100520000628BEF80AC002F0F3810728BEF80C10B6
:1005300001D0BEF80E2094F87EB10A938BF0300300
:1005400083EA0313DBB24FEA131E494884F804B070
:100550008EF07A0E4EEA032E00888EEAC303DFF88F
:1005600020E1C0EB00208EFB009E8644C0171BB22A
:10057000C0EB6E200690C3F3072E83EA0310059BA1
:10058000C0B24FF0000963F30F098EEA1013059310
:100590004FF0000E049B68F31F4967F30F0E4FF0F6
:1005A0000008002763F30F0861F30F07059BCDF8E0
:1005B0002C906CF31F4E62F31F474FF0000C9DF818
:1005C0001820CDF834E06AF31F48CDF830800E973C
:1005D0008DF83CC08DF83D2043EA00230DF128083A
:1005E00083EAC007B8E80F003FB287F0C80989EA7C
:1005F0000919DFF880E084F805C05FFA89F9C7F3CC
:100600000727AEE80F0087EA191747EA092398E899
:10061000030083EAC9031BB283F023074EF8040BDF
:1006200087EA0717FFB2C3F3072282EA1712704660
:1006300042EA072282EAC70720F814190BF1010BDE
:100640004FF0230CFE211622C82384F87EB12780A8
:1006500084F807C00EF1020EA170E270A37111E0E0
:1006600074A5002064A50020172B002020A30020E3
:10067000A4600020782900207229002074600020E6
:100680000308208010F8013B7B4083EA0313DBB2B0
:100690001A0982EA172242EA032282EAC3031BB242
:1006A0009FB270452780EDD183F0F40383EA0313F2
:1006B000DBB24FEA131E8EEA172E8EEA032E8EEA65
:1006C000C30E0FFA8EFE1FFA8EFCCA4FA4F800C0AC
:1006D0004FEA1C295FFA8EFE84F81EE084F81F9012
:1006E0007968BA683868FB6807F5D37CACE80F0016
:1006F00038697969BA6904F2C518ACE8070004F2F0
:10070000A71784F8C59184F8C4E117F8011F306871
:10071000FDF796F8B845F8D194F87231002B41F006
:10072000DC82B54B1B681922980684F8722140F1CF
:10073000F482B24BB24F1B78990741F147863B7D5B
:10074000042B8CBF4FF003084FF00208FCF73AFD72
:100750003B8A3A890A9003EB83035B00ADF8423091
:100760004FF47A703B680C93B7F80EE0397D7B68E4
:100770008DF8448000FB02F24FF0000C4FF0FF3088
:100780000DF12809ADF840E0CDF82CC00E920D9384
:100790008DF845100F90C846B8E80F00DFF86CE2FE
:1007A000AEE80F0098E80F00AEE807007246182187
:1007B00022F81C39E17194F87E1184F805C081F0AB
:1007C000780383EA0313D8B2030983F0F60343EAFC
:1007D000002383EAC0031BB283EA0310C0B2C3F351
:1007E000072383EA101343EA002383EAC0031BB202
:1007F00083F0C80080EA001C5FFA8CFCC3F307207A
:1008000080EA1C1040EA0C2080EACC0000B280F0A4
:10081000180383EA031C5FFA8CFCC0F3072383EA06
:100820001C1343EA0C2383EACC03C82001F1010A1C
:100830004FF0FE084FF01E0CA0710EF1020E217158
:1008400084F87EA1238084F8028084F803C01846CF
:1008500012F8011B414081EA0111C9B20B0983EA78
:10086000102343EA012383EAC10109B288B2724529
:100870002080EDD181F0180181EA0111C9B24FEA5F
:10088000111B8BEA102B8BEA012B8BEAC10B0FFAA1
:100890008BFB1FFA8BF3574A23805FFA8BFB1B0AF3
:1008A0000492059384F8273084F826B0964602F522
:1008B000D37A04F12208DEF80000DEF80410DEF836
:1008C0000820DEF80C30D446ACE80F000EF1100E14
:1008D000C645E246EFD1DEF80000CCF80000DFF8B4
:1008E00030819DF8143084F8CCB108F1260A84F8E0
:1008F000CD31C3461BF8011F3068FCF7A1FFDA4574
:10090000F8D1FCF75FFC3F4B3F4AB3F90410B7F84E
:1009100008E03B680B930A907B680C9382FB0127ED
:100920004FF47A70C9174FF0000C00FB0EF0C1EBCA
:10093000A701ADF83CC0ADF83EC0ADF840C0ADF881
:1009400042100D900E90CE46BEE80F002F4F84F857
:1009500005C00FC79EE807004FF0210C87E807008D
:100960001C23C8224FF0FE0EE370A27184F807C06A
:1009700084F802E094F87E11217181F06A0383EA21
:100980000313DAB2130983F0D50343EA022383EA9F
:10099000C2031BB283EA0312D2B2C3F3072383EA72
:1009A000121343EA022383EAC2031BB283F0C80294
:1009B00082EA0212D2B2C3F3072383EA121343EA94
:1009C000022383EAC2031BB283EA0C0282EA02100A
:1009D000C0B2C3F3072282EA101242EA00220131B8
:1009E00082EAC0020C3784F87E112280A7F11C0134
:1009F00010460FE07229002074A50020CAA500202F
:100A00003CAD002078A50020676666667829002046
:100A1000172B002011F8013B434083EA0313DBB29C
:100A20001A0982EA102242EA032282EAC3031BB2B5
:100A300098B2B9422080EDD183F0680383EA0313B2
:100A4000DBB24FEA131B8BEA102282EA032B8BEAFC
:100A5000C30B0FFA8BFB1FFA8BF3DA4F23804FEA9D
:100A6000132C5FFA8BFB04F1220384F825C084F871
:100A700024B007F5D37A0593FB6838687968BA68BB
:100A8000D646AEE80F00059B10379F42F246F3D1E1
:100A90003B88CD4FAEF80030C24684F8CAB184F826
:100AA000CBC11AF8011F3068FCF7CAFE5745F8D1D0
:100AB00094F87EC1C54A84F804C08CF0EB0383EA45
:100AC0000313D9B20B0983F0C50343EA012383EA78
:100AD000C1031BB283EA0310C0B2C3F3072181EA4A
:100AE000101141EA002181EAC00109B20CCA81F06B
:100AF000C80787EA0717FFB24FF0000EC1F30721BE
:100B00000B93CDF830E081EA17130A9299E80700B9
:100B100043EA072383EAC7030FFA83F9AC4B84F84F
:100B200005E089F0310783E8070087EA0717FFB27D
:100B3000C9F3072383EA171343EA072383EAC703AA
:100B4000277A607AA27AE17A94F80CE094F811900E
:100B50001BB25F4087EA0717FFB2C3F3072383EA9C
:100B6000171343EA072383EAC7031BB2584080EAFE
:100B70000010C0B2C3F3072383EA101343EA002333
:100B800083EAC0031BB25A4082EA0210C0B2C3F328
:100B9000072282EA101242EA002282EAC00212B25E
:100BA000514081EA0111C9B2C2F3072383EA11134C
:100BB00043EA012383EAC1031BB28EEA030E8EEAE5
:100BC0000E1E5FFA8EFEC3F3072383EA1E1343EA69
:100BD0000E23677BA07BE17B227C83EACE031BB2E2
:100BE0005F4087EA0717FFB2C3F3072383EA1713AF
:100BF00043EA072383EAC7031BB2584080EA001088
:100C0000C0B2C3F3072383EA101343EA002383EA45
:100C1000C0031BB2594081EA0111C9B2C3F30723D3
:100C200083EA111343EA012383EAC1031BB25A404A
:100C300082EA0212D2B2C3F3072383EA121343EA11
:100C4000022383EAC2031BB289EA030989EA09196C
:100C50005FFA89F9C3F3072383EA191343EA0923E7
:100C600083EAC903A17CE27CDFF870911BB2594092
:100C700081EA0111C9B2C3F3072383EA111343EADE
:100C8000012383EAC1031BB25A4082EA0212D2B2A4
:100C9000C3F3072383EA121343EA022383EAC2035E
:100CA0001BB283F0270787EA0712D2B2C3F30727E4
:100CB00087EA121747EA022787EAC2073FB20CF118
:100CC0000103BAB25FFA87FA4FF0310CFE200C2113
:100CD00084F87E31C8234FEA122E228084F807C0A0
:100CE000A070E170A37184F814A0049F84F815E04B
:100CF0007968BA68FB683868B7F810C0A9E80F00CF
:100D000029F803CB84F8BBE184F8BAA118F8011FD5
:100D10003068FCF795FDC145F8D194F87671002F45
:100D200040F0D6872B4B94F87E81B3F90010B3F9CD
:100D30000220B3F904309FED286ADFF894906771C0
:100D400007EE103A029B1B680A9388F06A0383EA55
:100D5000031306EE901AD9B20B0983F0D50343EAC8
:100D6000012383EAC1031BB283EA03115242C9B2D1
:100D700007EE902AC3F3072383EA111343EA012302
:100D8000F8EEE77AF8EEE66AB8EEC77A83EAC103CE
:100D90001BB267EE867A66EE866A27EE067A002038
:100DA00083F0C80CCDED0C7ACDED0B6A8DED0D7A8C
:100DB0000E900F9010908CEA0C1E0DF1280A5FFA2D
:100DC0008EFE0DE0722900203B2B00206871002070
:100DD0007829002078A5002088C3E43A182B002049
:100DE000C3F3072CBAE80F008CEA1E1C4CEA0E2C49
:100DF0008CEACE0C0FFA8CFCA9E80F008CF01E0ECA
:100E00009AE807008EEA0E17FFB2CCF3072E8EEA9F
:100E1000171E4EEA072E89E807008EEAC70E1C212E
:100E2000FE274FF0050A4FF01E0CC82208F10103FF
:100E3000A770E17084F876A184F807C0A9F11001C9
:100E4000A27109F10C0784F80480A4F800E084F88A
:100E50007E3111F8013B83EA0E0383EA0313DBB210
:100E60001A0982EA1E2242EA032282EAC3031BB263
:100E70001FFA83FEB942A4F800E0EAD183F0270309
:100E800083EA0313DBB21A0982EA1E2282EA0322F2
:100E900082EAC3031BB21FFA83FCDFF8E083A4F8E5
:100EA00000C05FFA83FE4FEA1C2C84F825C084F84A
:100EB00024E008F5D37904F1220AD8F80000D8F824
:100EC0000410D8F80820D8F80C304F460FC708F1A6
:100ED0001008D045B946F0D1DF4FB8F80030A9F876
:100EE000003007F1240884F8CAE184F8CBC117F870
:100EF000011F3068FCF7A4FCB845F8D194F877A13D
:100F0000BAF1000F40F0DE86D44B1B68052284F84E
:100F100077219A0641F10D80D14BDFEDD26ADA8953
:100F20001B8907EE902A07EE103AF8EEE77AB8EE42
:100F3000477A67EEA67A94F87EC1CB4BCB4AB3F9D9
:100F40000410B2F90620CA4FCA48CDED0B7A8CF0D6
:100F5000220383EA03135FFA83FE4FEA1E1383F032
:100F6000590343EA0E23B2F5FA6F83EACE031BB2AC
:100F7000A8BF4FF4FA6283EA0318B2F57A7F5FFAEA
:100F800088F8C3F3072EB8BF4FF47A72A2F57A72CD
:100F90008EEA181E642303FB02F34EEA082E87FB39
:100FA00003278EEAC80EDA17C2EBA71280FB0130C6
:100FB0000FFA8EF7CB174FF0000BC3EBA00387F0AF
:100FC000C8080DF128098DED0C7AADF83A20ADF87E
:100FD0003830CDF828B0CDF834B0CE4688EA0818BD
:100FE000BEE80F005FFA88F8C7F3072787EA1817EB
:100FF00047EA082787EAC8089F4FDEF800E084F830
:1010000004C00FC70FFA88F888F04A0383EA031078
:10101000C0B2C8F3072383EA10133A460CF101016A
:1010200043EA002383EAC00342F810E900204FF0AE
:101030004A084FF0FE0C4FF0140E84F87E11C821C0
:1010400060712380043784F8078084F802C084F834
:1010500003E0A171184612F8011B414081EA011119
:10106000C9B20B0983EA102343EA012383EAC101D1
:1010700009B288B2BA422080EDD181F0140181EA30
:101080000111C9B24FEA111E8EEA102E8EEA012E0E
:101090008EEAC10E794B0FFA8EFE1FFA8EFC1F46A8
:1010A0004FEA1C2B5FFA8EFE84F81DB084F81CE01A
:1010B000596838689A68DB68A4F800C007F5D37CE3
:1010C000ACE80F0038697969B7F818800497ACE884
:1010D000030004F2A717ACF8008084F8C3B1B84647
:1010E00084F8C2E104F2C31B18F8011F3068FCF752
:1010F000A7FBC345F8D1624B624A1B781278013BCB
:1011000012F00100DBB214BFC0214021172B03D81D
:101110005D4A134493F80CA05C4B1A8893071ABFDE
:10112000002341F01001012312F4027F18BF0223B3
:1011300012F0100F18BF062312F0200F18BF102353
:10114000002841F093804FF0030894F87EC10A9381
:101150008CF0460383EA0313DAB2130983F0920397
:1011600043EA022383EAC2031BB283EA0310C0B23C
:10117000C3F3072282EA101242EA002282EAC00286
:1011800012B282F0C80E8EEA0E1E00235FFA8EFEA7
:101190000320C2F307228DF82CA08DF82F8082EA5D
:1011A0001E128DF82D308DF82E108DF8300042EA89
:1011B0000E2899E8070088EACE0E0FFA8EF8DFF8BD
:1011C000B8A0E37188EA0819AAE803005FFA89F970
:1011D000C8F3072888EA191848EA092181EAC909E9
:1011E00094F808808AF800200FFA89F988EA090241
:1011F00082EA02185FFA88F8C9F3072282EA181215
:1012000042EA0822607AA17A94F80B90637182EA2C
:10121000C80212B2504080EA0010C0B2C2F30722E6
:1012200082EA101242EA002282EAC00212B251405F
:1012300081EA0111C9B2C2F3072282EA111242EA1D
:10124000012282EAC10212B289EA020989EA091975
:101250005FFA89F91CE000BF172B002074A500205D
:101260003CAD00200AD7233C78A500207460002004
:10127000D34D6210676666667829002072290020C7
:10128000A45A002070820020444D0408C8A5002004
:10129000C2F3072282EA191242EA092294F80C806A
:1012A000607BA17B84F804C082EAC90212B288EA9A
:1012B000020888EA08185FFA88F8C2F3072282EA6F
:1012C000181242EA082282EAC80212B2504080EAAA
:1012D0000010C0B2C2F3072282EA101242EA0022D2
:1012E00082EAC00212B2514081EA0111C9B2C2F3CE
:1012F000072282EA111242EA012282EAC102E17B5C
:1013000094F8109013B281EA030282EA0212D2B278
:10131000C3F3072383EA121343EA022383EAC203D7
:101320001BB289EA030282EA0212D2B2C3F3072394
:1013300083EA121343EA022383EAC2031BB283F057
:10134000320282EA0212D2B2C3F3072383EA1213F3
:1013500043EA022383EAC2031BB29AB24FF0FE08AB
:101360005FFA83FE0920C8210CF1010C84F8028089
:101370004FEA1228E070A17184F87EC1228084F8BF
:10138000128084F811E0049B186859689A68B3F8D1
:101390000CB00AF5CC7CACE807000AF5D47A8CF8DE
:1013A0000290ACF800B084F8B88184F8B7E117F87F
:1013B000011F3068FCF744FABA45F8D1039BC4F822
:1013C0006831FEF764BEDFF824A3B84FDFF820933E
:1013D000412026F0B7FDBAF9023087FB0320DB1766
:1013E000C3EBA00080B226F091FDBAF9003087FB74
:1013F0000320DB17C3EBA00080B226F087FDBAF90B
:10140000043087FB0320DB17C3EBA00080B226F07B
:101410007DFD99F80010D8F80000FCF711FA94F857
:1014200060A11AF0010700F0E183A14B1B68980648
:1014300072D5A04BA04F1B78990740F1C9863B7D20
:10144000042B8CBF032302234720039326F07AFD4D
:10145000386826F027FD786826F024FDB7F80EA03E
:10146000964AD8F80000A2FB0A3ACAF3471A514636
:10147000FCF7E6F93A8999F8001064208AEA010A33
:1014800000FB02F089F800A026F00CFD039B3F7DD5
:10149000D8F8000043EA8707FFB23946FCF7D0F9D5
:1014A00099F80030D8F800005F40394689F800709C
:1014B000FCF7C6F994F860A1BAF1000F2CD1804F67
:1014C0004F2026F03FFD386826F0ECFC786826F0C7
:1014D000E9FC504626F0E6FC0121D8F80000FCF7B4
:1014E000AFF9744B99F800201B78D8F8000003F08E
:1014F000010782F00102394689F80020FCF7A0F9C3
:1015000099F80030D8F800007B40194689F800307F
:10151000FCF796F994F860A16A4AC4F85CB10AF144
:101520000103DBB2A2FB0312D20802EB8202A3EB9F
:10153000420384F86031FEF78ABD634B6349186843
:10154000FCF746F900232370FEF729BE604F386888
:1015500000283EF469AD4FF0000ADFF898815D4C39
:10156000AB465546FCF768F9F8B1F5B94FF00109FB
:10157000AA463868FCF758F983B27E2B00F01A832C
:1015800098F80120002A49D194F84C11B1B11B2BD5
:1015900084F84C2100F0E8820D2B45D0386888F89B
:1015A0000190FCF749F90028E3D1AA4650460AAA5F
:1015B00049495D462BF072FFFEF736BD7D2B00F0EA
:1015C000AE8494F8502122B180F02003DBB284F87D
:1015D000501194F84B21062A10D8B4F84E113868EF
:1015E0001944A4F84E11A118013281F8543184F83D
:1015F0004B21FCF721F90028BBD1D6E7B4F84E21E6
:1016000088F8019013449BB21A0A52FA83F3FF2B15
:10161000A4F84E31386802D1304DA3E73868FCF7A2
:101620000BF90028A5D1C0E73868A4F84E21FCF7D3
:1016300003F900289DD1B8E794F8BC32C4F8B85239
:10164000012B40F2558494F8BD222549981801EBEE
:101650008001013202F001024E6A84F8BD22BEB15F
:10166000204F0B970DF14809123FA52349F8207D23
:10167000802284F8103115232946484684F8112128
:1016800084F81231B047002840F0B38394F8BC329C
:10169000154A013382FB0312A2EBE37202EB420212
:1016A0009B1A84F8BC32FEF702BD00BF676666660F
:1016B00074A50020CAA500203CAD00201F85EB5179
:1016C00068710020CDCCCCCC08A7002030A600202B
:1016D000D8A5002070290020BA2A0020C42A0020A2
:1016E000444D0408952A00205655555578A50020EC
:1016F000B4850020200000208F4A904B92F80BE028
:10170000029AD4F8381110681B888D4A401A4FF499
:101710007A71DFB201FB0EF11B0A977717758842C9
:101720004FF00007D37753759770177180F0CD8312
:10173000844985480B688968DFF828E2834F9EF862
:1017400000E097F8149080FB03C8DB1780FB010CC6
:10175000C817C3EBA80111770912C0EBAC00517791
:10176000F4214FEA202C7A4B82F820009176012058
:101770003021D07682F82210752078211EF0020FD9
:1017800082F821C083F81A9082F8230082F824108E
:1017900000F09883D7F800C06E4AD7F804E0DFF86D
:1017A000C8B1DFF8C88182FB0C014FEAEC7082FB04
:1017B0000EA2C0EBA1504FEAEE71C1EBA2520BFB9F
:1017C00000C10BFB02EB01EB41010BEB4B0B4900A2
:1017D0004FEA4B0B039288FB012A88FB0B284FEA48
:1017E000A8420692039AB7F80E803F8902EB820264
:1017F00002EB820207F5FA7707924FEAAA4ACA1764
:10180000BFB20597AAEB02073A464FFA87FA524F42
:1018100000EB800008EBC80807FB121200EB800009
:10182000069F4FEA8808CDF810800AEB800A4FEA3D
:10183000EB784948A7EB080100FB11B0039007982B
:10184000464FDFF81C81DDF814B083F815B049B2BB
:1018500001EB800106910499B9F1050F87FB01079F
:101860004FEADC7C4FEAE179C9EBA71983F809C09C
:10187000039FDFF8FCC0BDF81810CDF810904FEAB8
:10188000DE7E88FB02091FFA8AFA88FB070883F8C4
:101890000EE04FEAE770BCF800E0049FDFF8D4C028
:1018A00083F80AA04FEAE272C2EB6912C0EB68103B
:1018B0004FEA1A294FEA1B284FEA112B4FEA222A36
:1018C0001A73BCF800C083F80B90D97383F810B07A
:1018D0004FEA2029C7F307214FEA1E2B34BF3222DB
:1018E000332283F80DA0587483F8129083F8168081
:1018F000DF71197283F813E083F814B0DA7683F895
:101900001CC0C4F83451FEF721BBDFF86C90D9F845
:101910000000FBF781FF00283EF4A7ABD9F80000D8
:101920000121FBF775FF0222002387F8742088F855
:101930000030FEF79ABB00BFE4830020DC83002068
:10194000ACA600204CA50020676666663CAD002072
:10195000D8A600206BCA5F6B40420F00D34D6210C7
:101960001F85EB51CAA50020806967FF83DE1B43FA
:10197000D4A50020586D0020F85000205E2090472C
:10198000D8F8003002209847FF2025F0DBFF0378CD
:10199000FF2B00F01A8490F901304FEAE3795FFAE7
:1019A00089F9D8B22CF02EF948462CF02BF9D8F84A
:1019B00000305E209847D8F8003003209847FF2079
:1019C00025F0C0FF0378FF2B00F0FB83B0F908304F
:1019D000D8B2C3F307292CF015F948462CF012F9B8
:1019E000D34B1B78042B7DD0DFF880B3B4F82E11D5
:1019F0009BF80020DFF868A391FBF2F302FB1313BE
:101A00009BB2BAF80010A4F82E314FEA03191FFA5E
:101A100089F9642303FB01235200B3FBF2F349EA83
:101A20000329C3F303225E20D8F800301FFA89F996
:101A300049EA02099847D8F80030062098475FFA2B
:101A400089F02CF0DFF84FEA19202CF0DBF8B949C7
:101A5000B4F82E214B7ABAF800A00132012BA4F879
:101A60002E2100F05E864A7B0AEB8A031FFA83FA76
:101A7000002A40F0F683D8F800305E209847D8F866
:101A800000303A209847AC4BA3FB0A394FEA59196A
:101A90001FFA89FB5FFA8BF02CF0B4F84FEA1B2099
:101AA0002CF0B0F8D8F800305E209847D8F8003015
:101AB0003B209847642303FB19A39BB29F4805333F
:101AC00080FB0320DB17C3EBA000C0B22CF09AF818
:101AD00000202CF097F8DFF8989299F80630002B48
:101AE00040F08A833B689F0600F13A8294F82C31DB
:101AF000D8F80020FEF717BADFF878929FED908AA9
:101B00004FF0240A5E2090475046D8F8003098479E
:101B10008C4BF9EC016A9B8A07EE103AF8EEE66A04
:101B2000B8EEC77A0AF1010AC6EE877A5FFA8AFA36
:101B300067EE887AFDEEE77ACDED027ABDF908B05E
:101B40005FFA8BF02CF05EF8CBF307202CF05AF8FC
:101B5000BAF1270F02D0D8F80020D3E794F82C313F
:101B6000D8F80020FEF7DBB93868FBF765FE0028DF
:101B70007FF414AD386884F84A9188F80190FBF737
:101B80005BFE00287FF4F5AC0FE5FBF71BFB6E4B0B
:101B90001B68A0EB030B40F6B8339B4500F2B48101
:101BA0006A4B1A793A2A00F0CD84002388F8003075
:101BB000FEF75BBA386884F84AA184F84BA184F830
:101BC0004C9188F801A0FBF737FE00287FF4D1ACD8
:101BD000EBE494F8481194F849315D484A1CFEF74B
:101BE0000FBA013B84F86E31FEF76EBC594B1B886F
:101BF000DA0513D4D80600F1FD82990600F17C8540
:101C00005A0600F1A785180700F1A785D90700F14A
:101C1000DE8513F0020F0CBF04270C274E4B4F4AF2
:101C20001B78D27803F001030AB143F0020353207A
:101C3000039326F087F94A4A128802EB820202EBEC
:101C40008202900080B226F061F9002026F05EF951
:101C5000444A45491288D8F80000C2EBC21252002B
:101C600081FB023111444FEAE27ACAEB612A5FFA42
:101C70008AFA5146FBF7E4FD99F80020039BD8F857
:101C800000001F438AEA020A002189F800A0FBF73E
:101C9000D7FD3946D8F80000FBF7D2FD99F800309F
:101CA000D8F800007B40DBB2194689F80030FBF71A
:101CB000C7FD94F860A1FFF7FFBB013A84F86F21DC
:101CC000FEF72ABD0AF1FF3A84F877A1FFF776BB49
:101CD000013F84F87671FFF711B9013B84F8723146
:101CE000FFF71BB80024DFF8908027464FF0500A1A
:101CF00002E0DBB283F3118816F804B0601C594689
:101D0000304425F0CDFF002840F023810BF1010382
:101D10001C44EFF311838AF31288326E9442E8DB9D
:101D20000022DBB2326683F31188FEF7B6BA00BF39
:101D3000B85E0020E48300201F85EB51676666666D
:101D400000007A4480A50020DC4F0020C44F002012
:101D5000DCA50020C8A5002070820020386F00207C
:101D6000DC830020A460002003082080F283002090
:101D700064A50020B0A500206DDD03084FF0000A27
:101D80005E201F6884F82CA19047D8F80030DFF857
:101D900030931720984750462BF034FFBC4BA3FBE1
:101DA00007239B0BA9FB03125209C2EB0212A3EB00
:101DB0008203D8B22BF026FFD8F800305E20984777
:101DC000D8F8003018209847B24BA3FB07239B0993
:101DD000A9FB03125209C2EB0212A3EB8203D8B291
:101DE0002BF010FF50462BF00DFFD8F80020FEF727
:101DF0009FB80A9EBE4240F2AA843D46002141F2AD
:101E0000210015F8013B81EA03235A0013F4004F27
:101E100080EA020192B289B208BF11464A0080EA04
:101E2000020311F4004F99B293B218BF0B46590048
:101E300013F4004F80EA010289B292B208BF0A4649
:101E4000530012F4004F80EA03019BB289B208BF2D
:101E500019464B0011F4004F80EA03029BB292B284
:101E600008BF1A46530012F4004F80EA03019BB2E8
:101E700089B208BF19464B0011F4004F80EA0302F3
:101E80009BB292B208BF1A46530080EA030112F4D3
:101E9000004F9BB289B208BF1946B542B1D148463E
:101EA00006F03DFB7C490A9D7C486D1A152DA8BFA4
:101EB00015252A4631F0FAFA794A94F8BC321570A1
:101EC000FFF7E6BB2D22DA761BE5764B02991B78ED
:101ED0000968C4F83811013B012B3FF629AC1021E9
:101EE00002239170137123E42BF06EFEFEF790B87D
:101EF0006D4A02EB8302566AFFF7B1BB2BF054FE2A
:101F000001233B70FEF741B8684AB2F86231002104
:101F10000133A2F8623188F80010FEF7A6B83868DD
:101F200084F85091FBF788FC00287FF422ABFFF780
:101F30003CBBDFED5F7AB0EE677AFEF7FCBF01468F
:101F40008446074682460490804605900246FEF786
:101F5000F2BA41463A2025F0FFFD0743FFB2D5E62D
:101F6000DFF860A19AF80030980700F15782514FCE
:101F70004FF00009CB46D8F800305E209847D8F8DB
:101F800000300120984758462BF03CFE48462BF085
:101F900039FED8F800305E209847D8F80030092084
:101FA000984700202BF02EFE00202BF02BFE7B8A82
:101FB00097F81490B3F5967F0AD994F82C2102F083
:101FC0000F02072A04D842F20F79994528BF994693
:101FD000D8F80030DFF8F0B05E209847D8F800302D
:101FE000052098479BF80830002B00F09183A9F159
:101FF000200307EE903A9FED307AF8EEE77AF6EE9E
:10200000006A67EE877ABEEE007AF5EEC07AF1EEEE
:1020100010FA58BFB0EE667A77EE877AFDEEE77A6F
:10202000CDED027ABDF908905FFA89F02BF0EAFD58
:10203000C9F307202BF0E6FD9AF800200023920751
:102040000893099300F1CB8094F83031012B00F014
:10205000C680BBF90030DFED196A07EE103ABBF914
:10206000023007EE903AB8EEC77AF8EEE77A27EE3C
:10207000267A67EEA67ABDEEC77AFDEEE77A0AA861
:102080008DED0A7ACDED0B7A2BF0DEFD2EE500BF4B
:1020900073B2E745D34D6210802A00202CA20020A5
:1020A00041A20020B85E0020444D040870290020A1
:1020B000000000003CAD0020E4380E3F0050C34754
:1020C00089888888CAA50020E4830020C149C24BC2
:1020D0000093A1F13F07C14BC14A099101F8404C5F
:1020E0000AA8C049089706F0F1FA089F7B1C0893DC
:1020F0003C70089B2922591C08911A70089BEA22FF
:10210000591C08911A70089BC822591C08910AA8EA
:102110001A7030F03FFA00F101080AA94246089807
:1021200031F0C4F9089A02EB08030133089302F86E
:102130000840089B5A1C08921C70089B5A1C089265
:102140001C70089B5A1C08921C70089B5A1C089211
:102150001C70089B5A1C08921C70089B5A1C089201
:102160001C70089B5A1C08921C70089B5A1C0892F1
:102170001C70089B5A1C08921C70089B5A1C0892E1
:102180001C70089B5A1C08921C70089B5A1C0892D1
:102190001C70089B0122991812A808911A7050F817
:1021A000283DDB1B3B702BF0C7FD8F4B3470C3F811
:1021B000B052FDF770BFC4F83C5187F80080FDF7BE
:1021C000E4BE4FF00009484605E44846FFF7EABB85
:1021D0000123FFF739B9FBF71BFBFDF7EBBE97E8CF
:1021E0000C00012108A884F83011089209932BF003
:1021F0002BFD7BE4342711E5D8F80030DFF818A276
:10220000DFF810B25E209847D8F8003028209847B1
:10221000DAF800308BFB032BDB17C3EBAB0B5FFA59
:102220008BF02BF0EFFCCBF307202BF0EBFCD8F876
:1022300000305E209847D8F8003004209847B9F85D
:102240000830002B40F05B82DAF8083083F3100985
:102250005FFA89F02BF0D6FCC9F307202BF0D2FCF3
:1022600040E49BF800309AFBF3FA04E45F4AD2782A
:10227000002A0CBF4FF004084FF00508FEF765BFB9
:102280000123D9F800003B70FBF7CEFA0746D9F8D6
:102290000000FBF7C9FA7B067DF477AE8A2800F0D0
:1022A00085828E287DF471AE9AF80030002B7DF483
:1022B00088AE4F484F4B03602D2384F840310768A8
:1022C000FDF767BE434B0B93A3F140090022212188
:1022D000A3F13D0A03F8402C89F8021089F8012087
:1022E000CDF828A02FF034FD434B444A1B884449C5
:1022F00000280ABF11464FF003084FF004085A05A2
:1023000000F12182D80700F12B8203F002033D4A3D
:10231000002B1CBF4FF00308114642463A4831F0EB
:10232000C5F80AEB080312A8384A013340F8203DEB
:102330009B1A00220AF8082089F801302BF0FCFCD7
:10234000FDF753BF234A324B0B920DF14808A2F11F
:102350003D0048F8200D1988DFF8BC90A2F1400339
:1023600000204FF00A0E02F8400C082283F801E02A
:1023700040469A7006F0AFF8D9F800302549DA17D0
:1023800081FB0313C2EBA30399B2404606F0A3F806
:102390000EF074F9D9F808900A9B4FEA1942591CBB
:1023A0000A911A700A9B4FEA1922591C0A911A7055
:1023B0000A9B5A1C0A9283F800900A9B5A1C0A92A4
:1023C000187040462BF0B8FCFDF70CBF4FF0010829
:1023D000FEF7BCB930A6002046730020E07E04085A
:1023E000E87E0408F47E040870290020386F00207D
:1023F000E4A50020ACA60020C8A50020C47E0408E7
:10240000CC7E0408DC7E0408F3A50020F1A50020A2
:10241000DC830020676666664CA50020D24FD8F8A2
:102420000030DFF874935E209847D8F80030112010
:102430009847FA894FF4F36B0BFB02F289FB0239E0
:10244000D217C2EB69395FFA89F02BF0DBFBC9F3D5
:1024500007202BF0D7FBD8F800305E2098471920D2
:10246000D8F800309847FB89C04A0BFB03F382FB86
:102470000301DB17C3EB611382FB0321DA17C2EB05
:102480006112642101FB1233D8B22BF0BBFB002098
:102490002BF0B8FB9AF80030B7F8089099077FF551
:1024A00067AD5FFA89FB4FEA192964E5DFF8EC9222
:1024B0009FEDAF8AB9F90230AE4A0B9207EE903A1F
:1024C000F8EEE77A0DF1480867EE887AA2F140034A
:1024D000FDEEE77AA2F13D0148F8201D02F8400C1C
:1024E0000822CDED027A5A701E229A70BDF80810AB
:1024F000404605F0F0FFB9F9003007EE903AF8EEEB
:10250000E77A404667EE887AFDEEE77ACDED027A0B
:10251000BDF8081005F0DFFFB9F9043007EE903A76
:10252000F8EEE77A404667EE887AFDEEE77ACDED81
:10253000027ABDF8081005F0CEFF40462BF0FCFBF8
:10254000FDF74DBE99780393184614F0C9FF002893
:102550007FF42BAB8849894F894A8A4C0988DFF878
:1025600040929368F9611168B4F86221F863C7F882
:102570006CB0FB64F962D9F80000FA65F9F714FC55
:10258000834600287DF46CAD5146D9F80000FBF776
:102590003FF9039B94F86421DB780493642A4FF09D
:1025A000040387F8743040F01C8194F86531DFF83B
:1025B000F4A1072B08BF84F865B194F86521069251
:1025C00007EB021BDBF80410059108462FF0E2FF31
:1025D000DBF8083003935FFA80FB18462FF0DAFF30
:1025E000C3B20BEB0300069A0599059308308AF8ED
:1025F000070022F00F008AF80A0002F00F0203EB36
:10260000CB008AF80D208AF80E005A460AF10F0016
:1026100030F04CFF059B03990BF109001A460AF1B3
:102620000603184430F042FF9AF8073003F1010B1B
:10263000D3B1013B5FFA83FC0CF1080CDFF868E1D1
:10264000D4440AF10700002310F8011B59408B0005
:10265000CA0883EA410302F018024B404EFA02F224
:1026600053408445DBB2EFD1474A04980BF802305F
:1026700030F0F8FE94F865310022013384F86531BA
:1026800084F864219AF802305BB11AF80610D9F880
:102690000000FBF7D5F801369AF80230F6B2B342E3
:1026A000F3D894F864310322013384F8643187F855
:1026B000742088F80020FFF72AB92F4B334A1B8873
:1026C000927903EB830303EB83034FEA83081FFA3A
:1026D00088F8002A00F01581294B1B680FFA83FA4D
:1026E0000DF0CCFF40B2FDF72ABE114694461746C6
:1026F00092460492FDF71FBF2427FFF78FBA0DF013
:10270000BDFF2BF07FFA00202BF07CFAFFF7EAB92F
:102710005FFA89F02BF076FA4FEA19202BF072FA63
:102720008AE4D8F800305E209847D8F80030392085
:1027300098475FFA8AF02BF065FA4FEA1A202BF0DF
:1027400061FAFFF7C8B94FF003081149E5E5002128
:10275000FFF7A5BB1027FFF761BA2027FFF75EBA86
:102760000C494FF00408D8E53CAD00201F85EB5123
:1027700058A08B4130A60020DC83002020000020E0
:102780004CA50020702900207EBF002064A50020F9
:10279000D07E0408D47E040889B5F81478A50020FA
:1027A000F850002078BF00200007090E614B1B681D
:1027B0009F067DF5EAAB9AF80030002B7DF401AC62
:1027C0005D485E4B03602D2384F8403177E5082790
:1027D000FFF724BA5A4B8046B3F900A06420FDF7F6
:1027E000AEBD97F87530DFF868A1564905961A070F
:1027F00004BF0133DBB2072B28BF01234FEA031BC1
:1028000007EB0B02107C00228AF80A2011F800C0A6
:102810005FFA8BF203920AF10D02039E07EB0B01A4
:102820003043BCF1010F1070C96802F101000ED9EC
:10283000ACF10206F6B206F1020E9644024602F828
:10284000011B72454FEA1121F9D101363044BB44D6
:1028500021F0600201339BF81110DBB20A43082B10
:10286000027000F101024FD04FEA031B07EB0B008F
:10287000344E007C344916F800C0039E511A06F10C
:10288000100E01EB0C0606965FFA8EF60396069E76
:10289000132EC2DD059EDFF8BCE0C9B28A1DD2B29C
:1028A00042F040008AF8070002F1010BCAB14A1D4C
:1028B000D2B20832524403920EF1010C00221CF8ED
:1028C000010B5040820082EA4002C10842401F488A
:1028D00001F0180140FA01F14A4003996145D2B272
:1028E000EDD104980BF80E2087F8753030F0BAFD62
:1028F000C8E6114694461746924604929046FDF764
:102900001ABE4FF0FF33E9E60F49059E511AC2E7A0
:102910001146FDF710BE11469446FDF70CBE114658
:1029200094461746FDF707BE114694461746924651
:10293000FDF701BE74A50020E4A50020D8A6002064
:102940004CA50020444D040885BF00200007090E57
:1029500078BF00207EBF00202DE9F04F2DED068BC3
:10296000A94BAA4A1C7897B000F59C4120318146BA
:102970000B911160002C00F00387A54A1268904269
:1029800040F2EA80A34A07921668A349A34A069137
:10299000013C1C70A24B059206F480560993002E50
:1029A00040F0E8809F4B1B78022B01F0A781042B9D
:1029B00001F09681012B01F04A819B4B9945099BBF
:1029C0009B7800F2AD85002B40F0AE85974B0893C5
:1029D000079B1D6815F4805740F0A086DFF88092B1
:1029E000059BB3F90620069B5C8BA242B4BF002472
:1029F0000124DFF85882D8F80030DB0040F1C480B1
:102A0000089B1B7813F0010300F0C5800699498CE0
:102A1000914241F39082002C40F0C480844E96F89D
:102A20008C20002A40F0BE80824A8349106890F8CA
:102A30002D0000220A604A608A60804A002840F027
:102A4000B2801070002B40F0B3807D4B1A78002AC2
:102A500040F010810699059D488BB5F90070898B6F
:102A6000B5F902508742CCBF8026002646F04003CD
:102A70008F42A8BF33469B0843F080068542C8BFFB
:102A8000334643F040068D42B8BF3346059D9B0850
:102A9000B5F90460B5F9065043F080078642C8BF17
:102AA0003B4643F040078E42B8BF3B469B0843F08D
:102AB00080075F4E8542C8BF3B4643F0400796F80B
:102AC0008EE08D42B8BF3B469E4501F06E84A6F86D
:102AD000902086F892205B4986F88E300D78002D84
:102AE00001F0A7835F2B01F020846F2B00F0BA80E8
:102AF000089B1B78DF0700F1BD8096F89210002933
:102B000040F0B880B6F99030322B40F3B38096F89D
:102B10008E300120572B86F8920001F0BC87079A6F
:102B20001268540741F1BE825A2B41F0BB8296F8DD
:102B30009430002B42F0468196F8963083F00103E2
:102B400086F89630002B42F0DB810C202DF0CAFE77
:102B5000079B3D4D1B6890E02E4B07931E682F4B43
:102B60002D4A059306F480562D4B06920993002EAC
:102B70003FF418AF0021354806F0B3F900287FF480
:102B800011AF1FF055FE0DE76E023FF539AF089B00
:102B90001B7803F00103264E002286F88C20002CBF
:102BA0003FF442AF254A01211170002B3FF44DAF95
:102BB000E8067FF54AAF264B1B78D9063FF545AFAF
:102BC000002F7FF442AF2FF0C3F800287FF43DAF11
:102BD0001C4B1B78002B02F002811E4B9B78002CB3
:102BE00042F096813BB11C4A1C4B12681B689B1A31
:102BF000002BC2F26D8110200D4E2DF073FE0123CB
:102C000086F88D3021E700BF9CA4002034A300206B
:102C100098A40020247C00202495002074600020CB
:102C2000386F002096A30020404B4C00708200209B
:102C3000342C0020CCA5002004590020BC2E0020FC
:102C400053540020B4220020C8A50020EC580020D6
:102C5000CAA5002018A8002058AA0020F872002059
:102C6000AC500020B2F5FA7F04DB96F89220002ADF
:102C700001F08F84079B1B68854D590700F1D486AE
:102C8000844B0D930DF1500B1C460023CBF8043000
:102C90000A95149340F6330A192740F28336059DAE
:102CA00002E004344C4522D0A178E378994217FB26
:102CB0000160F6D294F801E00EF1040E17FB0361F7
:102CC00035F91E305345A8BF5346B3F5617FB8BFF1
:102CD0004FF461739842E4DA9942E2DB21782729C4
:102CE000DFD85846043406F0EDF84C45DCD16A4B89
:102CF0000A9D1B789BE8030088E80300002B40F046
:102D00007B86664B1B78002B00F0EC85644B0A93A6
:102D10006448012106F0E5F8002840F0EE82099BA6
:102D2000DB78002B40F0E982DFF894912B881EB20B
:102D300026F00106B7B2BB422F8001F00E805A4E3A
:102D40004FF002080E204FF0140B4FF0FF0A86F8E8
:102D5000008086F801B086F802A02DF0C3FD414640
:102D600050482F8806F0BDF8002841F0AE8227F0C9
:102D700002039BB2BB422B800AD04B4B0220142192
:102D8000FF2218700E2059709A702DF0ABFD2F881D
:102D9000464B474A197850680C93BE0708BF81F02C
:102DA0000201C1F340010B9204F02AFE24213D48A8
:102DB00006F097F830B9089A1378590744BF23F002
:102DC00004031370D9F8003013F00A0F1DD0052149
:102DD000344806F086F8002801F083802E887207B8
:102DE00041F13C822F48062106F07BF8002801F0D3
:102DF0006580730641F12A8207212A4806F071F89E
:102E0000002841F00380D9F800309F0600F13C858E
:102E1000B5F80080274F23480C2106F062F80028FF
:102E200000F0888248F4807343452B8009D01E4B04
:102E3000022214211A700E20FF2259709A702DF070
:102E400051FD1D4B1B78082B00F080820E2B00F0EB
:102E50007D82079B1E68700569D5184B1B79002B76
:102E600000F02D8214210F4806F03BF8002840F0B6
:102E70002B822AF0BBFF01202DF076FC002854D0D5
:102E8000DFF840A000264FF0CC0BA1461FE000BFAA
:102E9000C8A500205C500020487E0020FE53002082
:102EA000D0A50020EC5800206C33002020AA002080
:102EB00024AA0020F4830020A45A0020E4830020E8
:102EC00074A5002004C80020DEB2022E2CD80BFB13
:102ED00006F8731C5AF80840002CF5D1032290F92B
:102EE000023002940192C278E24951F82220009205
:102EF00018462246234601212DF09AF9034606EB97
:102F0000460000EB00100E9353B121460AEB8000FF
:102F1000CC2231F05EFC0E9B4AF808300136F6B246
:102F200020F046FE0028D0D14C46079B1E68089B27
:102F300093F800A0D04B1AF0010A00F05A82012247
:102F40001A700A9B05991B68B1F906105A89CB487B
:102F50004FF0010E914280F800E080F23082C84BC1
:102F60004FF07E521A60C74A069B0598B3F8188046
:102F7000B0F900E092F90430107892F801C0002B0B
:102F8000AEEB080314BF01224FF0FF32002BB8BF95
:102F90005B42B3F5FA7FA8BF4FF4FA73984280F210
:102FA000AF821B1A07EE903AF8EEE77AF045C7EDCC
:102FB000007A03DDF1EE677AC7ED007A059BB3F97D
:102FC00002E0AEEB0803002BB8BF5B42B3F5FA7F1B
:102FD000A8BF4FF4FA73984280F2EE811B1A07EEF5
:102FE000903AF8EEE77AF045C7ED017A03DDF1EEAD
:102FF000677AC7ED017A059BB3F90400A0EB0803DB
:10300000002BB8BF5B42B3F5FA7FA8BF4FF4FA7349
:103010006345CCBFA3EB0C03002302FB03F307EED5
:10302000903AF8EEE77A4045C7ED027ABCBFF1EE80
:10303000677AC7ED027A16F4805600F09A81B1F5EE
:10304000FA6F914BA8BF4FF4FA61B1F57A7F1A7805
:10305000B8BF4FF47A71A1F57A71002A41F0068168
:103060008A4ADFF840E282FB0130CB17C3EB6013E2
:10307000581C6FF0630C3EF910003EF913E00CFB96
:103080000313A0EB0E0003FB00F382FB0312DB171C
:10309000C3EB62139E440FFA8EFE07EE90EAB8EE81
:1030A000E78A87ED038A002E40F0AC832B885A060E
:1030B00040F1FA807649774A91ED018AD2ED019A82
:1030C00092ED026A91ED034A92ED030A91ED029AA4
:1030D00092ED007AD1ED005AD7ED011A97ED002A52
:1030E0006D4A6E4938EE445A79EEC63A77EE007A68
:1030F00065EE233A75EEC96A75EE890A37EE401A15
:1031000066EEA76AB0EE633AA0EE813A13F00303CD
:10311000B0EE665A78EE044A79EE867AA0EE815ACD
:10312000F0EE638AA4EEA73AD4EEA78AA4EEE75A9B
:1031300033EE263AF0EE687AF0EE674AF6EE008A51
:1031400035EE88AAE0EEC14A28EEC33A35EE635A5E
:1031500077EE293A77EEE67AAAEE233A25EE285A58
:1031600076EE403A34EE49AAE0EE817A74EEA64A51
:10317000AAEE235A34EE094A37EE697A64EEA84A79
:1031800063EE036AE4EE074A75EEC85A36EE006A4B
:1031900067EEA87AB0EE667A95EE057AE5EE056AF6
:1031A000E5EE867AB1EE648AF0EE665AF0EE476A92
:1031B000B1EE674AE8EE246A63EE270A67EEA43AA6
:1031C000E4EE275AB1EE450AB0EE606AB0EE631A3B
:1031D000A4EE277A23EE244AE7EEA76AA5EE246A36
:1031E000A0EE031AE8EE245AB0EE448A31EEA19A1A
:1031F000E0EE240AA5EE278A66EEA16A72EE028A44
:10320000E5EE033A61EE211A26EE096AA4EEA47AED
:10321000A0EE274A0CBFD7ED022ADFED212A82ED6E
:10322000005AA2EE256AE0EEA86AE2EE081A73EEF2
:10323000A33A27EE227A34EE044AF0EE005AE3EE87
:10324000A26AA4EE226AA1EEA57AC7ED016AC1EDD9
:10325000376A81ED366A87ED006A81ED387A82ED52
:10326000013AC2ED027AC2ED034AEBB987ED027A68
:103270001AE000BF1872040871820020F42E0020AA
:103280006C2E0020F0A70020603400201F85EB5139
:103290006C1B0020DC00002014010020342C0020D6
:1032A0000000000054D40020BAF1000F40F02B8140
:1032B0002EF0A2FF17B0BDEC068BBDE8F08F089B87
:1032C0001B78D9077FF5D5AD4FF40F702EF008F9B4
:1032D00000283FF42AAE0DF069FD4FF40F702EF078
:1032E000A9F800283FF421AE0DF060FD4FF40F70F7
:1032F0002EF0A0F80028EED117E6DFF88C93D9F86D
:10330000003099077FF512AD2F88FA073FF52FADF2
:1033100047F001039F422B803FF429ADC44B0222AA
:1033200014211A700E20FF2259709A702DF0DAFACB
:103330002F881CE528F480739BB243452B807FF4D3
:1033400076ADBC4B1B78082B7FF480AD2A8822F029
:1033500040039BB29A422B803FF47BADB44B0222D8
:1033600014211A700E20FF2259709A702DF0BAFAAB
:103370006FE5069B5A8B9142C0F2EC84B1F5FA6F6F
:10338000D4BFC2EB0101C2F5FA614FF47A7303FBBB
:1033900001F1A9480378C2F5FA62B1FBF2F1002B02
:1033A0003FF45EAE4378A54A01FB03F182FB0123A3
:1033B000C917C1EB631153E6DFEDA17A13E6B1F54E
:1033C000FA6F80F2C084187A8B1A03FB00F3C2F5FF
:1033D000FA6293FBF2F3C3F1640307EE903AF8EE5E
:1033E000E77A9FED987A984B67EE877AC3ED007A7B
:1033F000B9E51B780793002B7FF4A3AD934A1268BD
:10340000002A3FF49EAD924A089212F8030CDFF8AE
:103410007CB21146A2F103092EF070FC9BF80080EB
:10342000089A002800F0B285079BB8F1000F59D127
:1034300009F1080199F805002EF060FC002841F020
:10344000AD84844999F80A002EF058FC002800F059
:10345000B285B8F1020F41F09D847F4999F80F00C1
:103460002EF04CFC002841F091847C4999F814001E
:103470002EF044FC002800F0B285B8F1040F41F0B2
:103480008184774999F819002EF038FC002841F022
:103490007584744999F81E002EF030FC002800F065
:1034A000B285B8F1060F41F065846F4999F82300A1
:1034B0002EF024FC002841F059846C4999F828002A
:1034C0002EF01CFC002800F0B285B8F1080F41F086
:1034D0004984674999F82D002EF010FC00283FF42C
:1034E00030AD09231A4602EB82029144614A99F8F1
:1034F000010099F802108BF800301070517020E52F
:10350000DFED4F7A52E50C9B19780B9B01F001011E
:10351000186804F075FA17B0BDEC068BBDE8F08FA3
:1035200013B9099A01239370534B099A1D7892F8A5
:10353000214008931B202EF019FC012C05F00108F6
:10354000814600F00B8705F00205099A4B4E92F870
:103550002030DFF83CA14A4F0A959346052B00F234
:103560006387DFE813F0C000B6000600FE0000012C
:10357000F300012C04BF05238BF82030B8F1000FB5
:1035800012D0069B3088B3F918100022134661F35D
:103590000F0260F31F4261F30F03059861F31F43AD
:1035A0000360032342600A93364DDBF814102A6847
:1035B000914280F02E8647F230510322CBF81C1046
:1035C0008BF82020022003F077FA1FF031F92968E8
:1035D000DBF81C200A440421CBF818208BF82010BB
:1035E000012C40F08C872A68DBF81810914280F09B
:1035F0001B879AF8000020B92EF0B8FB002840F095
:1036000013873A6822F002023A602A6873886421BC
:1036100001FB03234FF480600022CBF810308BF8BD
:1036200020208BF8032003F017FA9BF8203095E751
:103630006C330020A45A0020603400201F85EB5119
:10364000000000000AD7233C6C2E0020748200206A
:103650003A33002044330020493300204E33002009
:1036600053330020583300205D33002062330020A4
:10367000673300207882002070820020944D002063
:10368000C4A5002058AA002074A5002096000020A0
:10369000B42200202EF070FB012807D1834D7288E0
:1036A0002B68642101FB0233CBF81030B9F1000F15
:1036B00002D0B379002B4BD1012C00F0B5867B4DA5
:1036C000DBF810102A689142C0F0268701238BF89E
:1036D0002030012C3AD0F379012B46D010F064FE53
:1036E0009BF820303AE7B8F1000FD3D10A9D4FF490
:1036F0008060B9F1000F00F04E8303F0C5F9099A1C
:1037000000231361002D3FF463A928462DF0EAF849
:10371000079B1D6815F480573FF460A91D2164487C
:1037200005F0DFFB00287FF459A9624B03F1500933
:1037300003E00433994500F07D861A78262AF8D1F3
:103740009978DA789142F4D2FFF74AB9574D5CE79D
:1037500010F02AFE03224FF47A738BF82020CBF866
:103760001C30524D2EE7514D3AE710F01DFE03225A
:1037700040F6B8338BF82020CBF81C304B4D21E7B6
:103780004D4F3B78002B01F0FB814C4BDFF848811B
:10379000DFF848B1DFF848A1069345465E4605903C
:1037A00099460EE019F804109847032C28DC88B9D4
:1037B0003B782AF8020F01349C4205F1040580F29F
:1037C0006D81072CE1B23046DBF80430EADD984722
:1037D00000B2EDE738F824206B88801A4FF47A7134
:1037E0009B1A01FB00F040F6CA0290FBF3F008447C
:1037F000904240F2EE23A8BF10469842B8BF184648
:1038000000B2D5E71D212A4805F06BFB002840F0E7
:10381000E4850D9B03E00433A3423FF447AC1978E1
:103820002629F8D19878DA789042F4D2099BDB788F
:10383000002B7FF43BAC1E4805F053FBDFED207AF4
:10384000002801F0B48138EE678A1E4A1E49FDEE59
:10385000C87ACDED057ABDF914301B0382FB030253
:10386000DB17C3EBA212C8F57A731BB203FB02F39A
:1038700043F30F33434407EE903AF8EEE77A01231F
:10388000C7ED037A0B7011E4104B1B789E0704D52B
:103890000F4E337D042B00F24A86B5F8008018F0F5
:1038A000300F40F0D2830B4FFFF7B5BA58AA002073
:1038B000EC5800205C50002020510020249500206E
:1038C00000007A44D34D6210E82E0020CAA50020E3
:1038D0003CAD0020F48300204051002020A30020B4
:1038E000322C0020DFF8A8B1DFF8A891614E98468D
:1038F0000BF15A074FF0010A59461BF8010C2EF044
:10390000FDF9F8B19BF804009BF802309BF803E046
:1039100000EB400106EB8101013BD1F8A02003EB55
:1039200043034B4493420DD096F8CC2081F89CE0A1
:103930000AFA00F022EA0000C1F8A030C1F8A48021
:1039400086F8CC000BF1060BBB45D5D14A4B0A9348
:1039500019464A4A4A4B09681B78D2F80080DFF8BA
:1039600038A10C910B934FF0FF394FF0000BDAF8B0
:103970000430002B37D01F78002F34D0DAF808201D
:10398000A8EB0202002A11DB3A4E012196F8CC2066
:1039900001FA0BF122EA010286F8CC20394A08F537
:1039A000FA704FF0FF31CAF8080011600B9AD2B1DB
:1039B0009AF8002059780432D2B2002940F0C1822E
:1039C00006990598098B30F9122001F1C80082424E
:1039D00040F36685274E9A7896F8CC3043FA0BF37D
:1039E000DB0740F1F9850BF1010BBBF1040F0AF184
:1039F0000C0ABCD1FFF78CB9234B03E00433A3427C
:103A00003FF47FA919782329F8D19878DA78904281
:103A1000F4D21E4805F065FA00283FF472A914207C
:103A20002CF060FFFFF76DB9124E96F896305BB13F
:103A3000089B1B78DA0707D5059BB3F90620069B80
:103A40005B8B9A4200F3B7851121104805F049FAC3
:103A5000002800F05E8296F89A302BB996F89430E0
:103A600013B93223A6F89830012386F89A30FFF76D
:103A700007B900BF342C0020D0A5002058AA002090
:103A80002C6F0020601B00205C500020EC580020B0
:103A900051320020784D0408D02C0020DDF814901D
:103AA000BE4A0792BE49126842F2010AA1FB091BF5
:103AB00012EA0A0A4FEA9B1B00F02882B94DBA4865
:103AC000BA4CBB492D780078257008701DB1B849F3
:103AD0000D7885F00105B74E0F2186F82410002BD4
:103AE00000F0C783069CB44BB4F826C0B4F824E0B9
:103AF000069C10931846248B0078B04B129496F8CD
:103B000025400994AE4C0F9005940446A3FB000396
:103B10005B0803EB4303E31ADBB2CDF834C002F4D5
:103B200080520C9397F80080DFF8D8C2A44C0E9115
:103B30000BF5967306F12800CDF844901392DDF84A
:103B400024900A930996002108957646089B002B3D
:103B500000F00283099B33F911201FFA82FEB6455B
:103B60004FEA410303D30D9DAE4540F239835CF823
:103B70002120934580F0F982E25EBAF1000F40F017
:103B80000E8301314145E25200F10600DEDB0E9A60
:103B9000099E8C4B86F824200F2A49460CBF01222F
:103BA0000022DDF8449086F825101A7000F0688332
:103BB000854B7D497E4ADFF850B209931C460420AC
:103BC00001230B70137002F077FFDBF80030A1685F
:103BD0006268E3605B1A934284BF002384F821305B
:103BE000079B3C781E68002C01F00280069A774DF6
:103BF000B2F824E0178B724916F48056284640F03C
:103C0000768332460EE0437803EB830303EB8303B2
:103C100003F2EE239BB20132944221F8023B00F101
:103C200002000ED015F81230002B00F0DD82022BBE
:103C3000E9D001320B8821F8023B944200F10200E6
:103C4000F0D1109A137801331370FEF7A8BE594EC5
:103C5000D6F88830A9EB0303002BFEF6AEAE5C4A23
:103C60005C4B527C069933F812308A7DDFED5A6A3C
:103C70009FED5A6AC97D9BB207EE102A07EE903A73
:103C8000B8EEC77AF8EEE77A27EE267A67EE867AFC
:103C90000B9AC6F88820C7EE876A40F2FF32FCEE26
:103CA000E67ACDED087ABDF82030934228BF13465E
:103CB00009B1D31A9BB24A484A4D01784A4C35F8AB
:103CC0001160226825F81130921B13440131474DD1
:103CD000236001F00F021B0902702B80FEF76DBEFE
:103CE000F9F770FA424B434A1B68C31A93427EF7B6
:103CF00064AE3E4B00221A80FEF75FBE069A05991D
:103D0000537DD27D013B31F913301AB1C3F53B63CA
:103D100008331BB2A3F57A7307EE903A9FED367A1B
:103D2000324AF8EEE77A40F2FF3167EE877AFCEE2E
:103D3000E77ACDED087ABDF820308B4228BF0B46DC
:103D40001380FEF73ABE1B7AC3F1640307EE903A84
:103D5000FFF745BB3146FFF71CBB0221274805F0A2
:103D6000C0F800283FF403A82E80BB073FF510A839
:103D700047F00203BB422B803FF40AA8204B0222EB
:103D800014211A700E20FF2259709A702CF0AAFD8F
:103D90002F88FEF7FDBF02F05FFEB0E4247C002018
:103DA000D34D6210FCA200205C1E00202C6F00206E
:103DB0005D1E0020342C002013500020ABAAAAAABC
:103DC00074600020F4580020386F002074510020E7
:103DD000F8A9002018AA00200000C8420000804472
:103DE00097A300209CA3002098A30020A46000209B
:103DF0006029002060E316006F12833FEC5800201A
:103E00006C3300201450002058AA0020B84AB2F9A0
:103E10000030002BB8BF5B42B3F5E17FBEF6F3AFD5
:103E2000B2F90230002BB8BF5B42B3F5E17FBEF6BA
:103E3000EAAFB04B93ED057AD3ED077AD3ED096A7B
:103E400093ED030A77EEA67A30EE070AF7EE000A42
:103E5000B0EE007AE7EEC70A30EE000A04F08EFDFD
:103E6000B6EE008A20EE488A9FEDA30A38EE000ADB
:103E7000FDEEC07A17EE903A2033402B40F2A98332
:103E80009FED9E0A9E4EDFED9D7A86ED000ABDEE07
:103E9000C87AC6ED017A17EE103A2033402BC6EDF2
:103EA000027A00F25486B0EE480A04F0EDFC0A20D3
:103EB00086ED030A2CF016FDFEF7A5BF26F04003A1
:103EC0009BB2B3422B803EF497AF8E4B022214215B
:103ED0001A700E20FF2259709A702CF003FDFEF725
:103EE0008BBF2B8823F00406B6B2B3422E803EF47B
:103EF00079AF844B022214211A700E20FF225970D0
:103F00009A702CF0EFFC2E88FEF76CBF7E490D787E
:103F1000DCE596F89430002B3EF4B2AE089B1B789B
:103F200013F001037EF4ACAE012286F8943086F8DB
:103F30009520FEF7A5BE754E012286F88C20FEF76F
:103F400031BE012900F06285B9F1FF3F6F4E0BD001
:103F50001B780C2B08D06E4B6E4A03EB87076E4B19
:103F6000C3F800907B6C136096F8CC20012303FA11
:103F70000BF30BF1010B1343BBF1040F86F8CC30AC
:103F80000AF10C0A7FF4F3ACFEF7C2BE511D99F89A
:103F900005002DF0B3FE00283FF453AAB8F1010F3D
:103FA00040F0FC8609F10D0199F80A002DF0A6FEFB
:103FB000002840F0EF86594999F80F002DF09EFE39
:103FC00000283FF452AAB8F1030F40F0DF865449AD
:103FD00099F814002DF092FE002840F0D386514944
:103FE00099F819002DF08AFE00283FF452AAB8F182
:103FF000050F40F0C3864C4999F81E002DF07EFE57
:10400000002840F0B786494999F823002DF076FE44
:1040100000283FF452AAB8F1070F40F0A7864449A0
:1040200099F828002DF06AFE002840F09B8641494F
:1040300099F82D002DF062FE00283EF482AFB8F111
:10404000090F3EF47EAFFFF74CBA102002F004FDDA
:10405000202002F001FD384BB5F80080374F0022D8
:104060001A703749374A384E384800230B603849B0
:1040700033604FF0000E036053609361C2F800E0BC
:10408000C2F808E0C2F814E0C2F81CE0C1F800E091
:104090004B60C1F808E0C1F814E08B61C1F81CE086
:1040A000FEF7B9BE5D2B00F09C825B2B00F06C85A7
:1040B0005E2B00F0E285562B00F0E385972B00F095
:1040C0007886A72B00F0CF85224D2A88900740F0F4
:1040D0009B85A3F1B702072A00F2AD82DFE812F058
:1040E0008F02AB02AB02AB02A402AB029D029602AE
:1040F00078A50020EC000020DB0FC93F0000000085
:104100006C1B00206C3300202C6F0020342C00200E
:10411000784D0408706D0020601B0020493300209A
:104120004E33002053330020583300205D330020ED
:10413000623300206733002074710020F483002074
:104140006072002010720020902E0020502F00205E
:1041500038720020C8A50020002E3FD05CF8212036
:1041600093454FEA4103FFF407ADBB4ABA4DD25C19
:1041700005EB030E002A00F09C80022A47D19EF82E
:10418000012002EB820202EB820202F2EE2292B2E4
:10419000032933DD12B2BAF1000F3FF4F2AC0C9DEB
:1041A00020F81520B9F1000F03D10F9D022D7FF6E5
:1041B000E8ACB0F800904288B0F804E04A44964475
:1041C000A64A0FFA8EFE82FB0E52A54DA2EBEE72AE
:1041D00025F803E012B24FF00109D2E432464B0059
:1041E0000A9D4CF82150C8E4D3B2022B04D9032B0A
:1041F0007FF41FAD73460EE53B460CE5012505FA3D
:1042000001FE0E9D25EA0E0512B20E95B5E4E25AA6
:10421000BEE7944A1278002A7FF4CDA9B8F1000FC6
:104220003FF4C9A9012C40F0FF809BF82030FFF734
:1042300095B929468C4804F054FE002800F091807E
:1042400086F893501EF024FFFEF752BC46F0400360
:10425000B3422B807FF439AEFEF7CEBD46F00403A7
:104260009E422B807FF445AEFEF7BCBD5B78FFF726
:104270009AB87E4B7E4A109201221A707D4B0593AC
:104280001B21794804F02DFE00287FF491AC7A4B75
:10429000DFF808B209931946DBF80030CA688B6072
:1042A0009B1AC82B00F27484079B1E6806F4805684
:1042B000C7E4CAB2022A40F2A683032AA7D1129AFF
:1042C000139D002D08BF324662E727F001039BB221
:1042D000BB422B803FF449AD0E2086F8008086F863
:1042E00001B086F802A02CF0FDFA2F883DE50022EF
:1042F0000FE0437803EB830303EB830303F2EE2326
:104300009BB20132A24221F8023B00F102003FF4CD
:1043100098AC15F812301BB1022BEAD00B88F0E7ED
:10432000D3B2032BFAD83B46EBE7B2F5FA7FFEF6A1
:10433000A1AC96F89230002B7EF49CAC089B1B78C5
:10434000012213EA020486F8922000F0C8831EF0CE
:104350006FFA079B494D1B68FEF78FBC0025FFF7DE
:10436000F4B8089B464A1B781060DA077EF5C5ABA7
:10437000444B1B78002B3EF47DAC099BDB78002B73
:104380007EF478AC96F893300133DBB2032B86F8D9
:1043900093307EF66FAC3C4B5B7813B9002C7EF407
:1043A00069AC1EF045FAFEF7A3BB384A38491068DD
:1043B000B6F99020C56981FB05018911ED17681ACE
:1043C00000F5FF407F3082423EF785AB491B0A442F
:1043D00012B2A6F89020FEF77EBB099BDB78002B7B
:1043E0007FF417AADFED2B7A294938EE678AC8F5E2
:1043F000FA63FDEEC87A1BB2CDED057ABDF9142043
:10440000120381FB0201D217C2EBA11203FB02F3DC
:1044100043F30F33434407EE903AB8EEE78A0D9B1F
:1044200087ED038AFFF7FBB90A9D002D3EF4D0AA61
:10443000FFF76BB9184A069BD488059A1B8BB2F913
:104440000620191B8A4240F3B38023449A42B4BF2A
:1044500000240124FEF7CDBA74510020565555555D
:10446000A42C0020AC2E0020EC580020F458002092
:104470001350002074600020386F0020C8A5002071
:10448000FC7200202C6F002018A80020B0A700208C
:10449000D34D621000007A447C4D002058AA0020C1
:1044A000C8398A42C74E65DA9A7896F8CC3043FA12
:1044B0000BF3D8073FF597AA524201200E922CF039
:1044C00037FB7B1E0E9A162B00F29683DFE813F063
:1044D000BF01A6018A01EC01D8011902340164026E
:1044E0004A027B025F019403EC0199021902340134
:1044F000640246029502ED001F010601D500AB469D
:104500000999DBF80020CB690A9D13448B61002DCB
:104510003EF45EAAFFF7F9B80FF046FF032140F61C
:10452000B8328BF82010CBF81C20FFF74BB80A20CC
:104530002DF01CFCB5F800808146002800F0EC82CC
:1045400018F0100F00F0A3839E4E96F8D490B9F1A6
:10455000000F7FF4A8A99C4F0D202CF0C3F9012374
:1045600086F8D430B5F80080B9F1000F7FF479AD4A
:10457000FEF751BC96F8CC30012202FA0BF223EA86
:10458000020308F5FA7286F8CC30CAF80820FFF763
:104590002ABA089B1B780121DB0786F8921000F1EC
:1045A000DA821EF075FD079B884D1B68FEF765BB20
:1045B0000124FEF71EBA0021854804F092FC002871
:1045C0007FF442AA322386F89600A6F89830FFF7C7
:1045D0003BBA04F059F955E4002A0CBF012002202F
:1045E0006CE77C4B002201207B497C4C0B602270E5
:1045F0002CF09EFA079B754D1B68FEF73EBB012011
:104600001FF0A4FA079B1B68FEF737BB02201FF0C0
:104610009DFA079B1B68FEF730BB03201FF096FA3C
:10462000079B1B68FEF729BB00201FF08FFA079B32
:104630001B68FEF722BB9E2B00F013849D2B00F01D
:104640000884AE2B00F0FD83AD2B00F0F383EF2B3D
:1046500000F0ED83FD2B00F0DA83FB2B00F04284A9
:10466000FE2B00F03C84F72B00F02F847B2B00F016
:10467000B083079B1B68FEF700BBD6F8D000584BF1
:1046800090F836909B789144B9F1640FA8BF4FF031
:10469000640929EAE97980F83690002B40F010840B
:1046A0000FF018F8DAF8043052E4D6F8D0004C4B8A
:1046B00090F802909144B9F1C80FA8BF4FF0C80913
:1046C00029EAE97980F802909B78002BE8D0142041
:1046D00049462DF093FBD6F8D000E1E7D6F8D0009C
:1046E0003F4B90F837909B789144B9F1FE0FA8BFEB
:1046F0004FF0FE0929EAE97980F83790002BCFD0F6
:10470000162049462DF07AFBD6F8D000C8E70C9960
:10471000334B91F801909144B9F5967FA8BF4FF4BF
:10472000967929EAE97981F801909B78002B40F08D
:10473000FF83D6F8D000B3E7D6F8D000284B90F826
:10474000049099789144B9F1C80FA8BF4FF0C809F7
:1047500029EAE97980F80490002940F0FA83102FC3
:104760009ED090F801909144B9F1C80FA8BF4FF0C6
:10477000C80929EAE97980F801909B78002B8FD04D
:10478000132049462DF03AFBD6F8D00088E7D6F83A
:10479000D000134B90F808909B789144B9F1C80F62
:1047A000A8BF4FF0C80929EAE97980F80890002BE2
:1047B0003FF476AF0B2049462DF020FBD6F8D00011
:1047C0006EE700BF342C0020F4830020C8A5002031
:1047D000EC58002016550020CCA500204073002086
:1047E000806D00200C99C54B91F804900E93914474
:1047F000B9F1640FA8BF4FF0640929EAE97981F89B
:1048000004902DF015FB0E9B9B78002B91D003207C
:1048100049462DF0F3FAD6F8D00041E70C99B74B92
:1048200091F802909144B9F1640FA8BF4FF0640968
:1048300029EAE97981F802909B78002B3FF479AF5F
:10484000022049462DF0DAFAD6F8D00028E70C9974
:10485000AA4B91F800909144B9F1FA0FA8BF4FF01C
:10486000FA0929EAE97981F800909B78002B3FF456
:1048700060AF012049462DF0C1FAD6F8D0000FE70D
:104880000C999E4B91F807909B78914489F3080905
:1048900081F80790002B3FF44CAF052049462DF0DE
:1048A000ADFAD6F8D000FBE60C98944B90F8069041
:1048B00099789144B9F1640FA8BF4FF0640929EACF
:1048C000E97980F80690002940F03A830D2F3FF4F3
:1048D00030AF0C989B7890F805909144B9F1640F33
:1048E000A8BF4FF0640929EAE97980F80590002B08
:1048F0003FF41FAF0E2049462DF080FAD6F8D000C5
:10490000CEE6D6F8D0007D4B90F80390997891448C
:10491000B9F1C80FA8BF4FF0C80929EAE97980F8B2
:104920000390002940F0E1820F2F3FF4B9AE90F8D8
:1049300000909144B9F1C80FA8BF4FF0C80929EA07
:10494000E97980F800909B78002B3FF4A9AE122003
:1049500049462DF053FAD6F8D000A1E6D6F8D0009B
:10496000664BE4E7D6F8D000644B90F806909B784D
:104970009144B9F1C80FA8BF4FF0C80929EAE979F5
:1049800080F80690002B3FF48BAE092049462DF0AD
:1049900035FAD6F8D00083E6D6F8D000574B90F819
:1049A000059099789144B9F1C80FA8BF4FF0C80994
:1049B00029EAE97980F80590002940F0D682112F84
:1049C0007FF476AE6CE6D6F8D0004C4B90F80790AA
:1049D0009B789144B9F1C80FA8BF4FF0C80929EAE4
:1049E000E97980F80790002B3FF45AAE0A20494637
:1049F0002DF004FAD6F8D00052E6D6F8D0003F4B9E
:104A0000AFE63E4B65E7129AFFF7C2BB059993F8F4
:104A1000029031F91220B2F5617F4FF4966191FB5B
:104A2000F9F1C0F29F8040F633099145A8BF914645
:104A30000C2FA9F5617999FBF1F95FFA89F900F07A
:104A40007881182F40F099804A46C82AA8BFC8220A
:104A50002B4ED6F8D01091F817E0D0B270453FF445
:104A600077AAB2EB0E02254BC87548BF0732D210A9
:104A70009978531CDBB239B913B118462CF058F8A9
:104A8000DAF80430FFF764BA494618200E932DF087
:104A9000B5F90E9BF0E71B4B1B491A684FF47A736C
:104AA000B3FBF2F3C3EB431203EB8202079B1B68D9
:104AB000D2001E06A1F8A8207EF5DEA8134A1278BF
:104AC00095077EF5D9A8124A127D042A7EF6D4A84D
:104AD0001CF092FA079B0F4D1B68FEF7CEB80F2013
:104AE0002BF000FFB6F8903086F89240FA3BA6F81B
:104AF0009030079B074D1B68FEF7BFB8806D002004
:104B0000342C0020147C002024740020CAA500202E
:104B10003CAD0020C8A5002018F0100F40F0FE802A
:104B20000B202DF023F9002840F0C980D14F18F058
:104B3000200F40F03781D04E96F8D430002B3FF450
:104B40000BADB9F1000F7FF48CAAFEF764B9B0EE9B
:104B5000670AFFF7ACB9C949079B0A601B68C84DD3
:104B6000FEF78BB80C2F00F0FA80182F03D14FF00E
:104B700000094A466CE74FF00009BF4EFFF7E8B95D
:104B8000C04A0692FEF78CBFBF4B012202202BE5E4
:104B9000BE4A079B1E68136823F004031360099A3A
:104BA000012306F4805682F82130FFF74AB838EE28
:104BB000678AB74BB7491870FDEEC87AC8F5FA6333
:104BC000CDED057ABDF91420120381FB0201D21745
:104BD000C2EBA1121BB203FB02F343F30F334344B6
:104BE00007EE903AF8EEE77AC7ED037AFEF75EBA81
:104BF00006F48056FFF725B8D6F8D0000EF06AFD0F
:104C00004FF0FF39FFF7B0B90022BB2B149200F030
:104C1000FC80B72B00F0F680BE2B00F0F080BD2B9F
:104C20007FF409AD13464FF6FE729B49C8898C8903
:104C3000034422448A81CB8127F054FF03F05AF9C0
:104C400027F038FFF7F722FB01202BF071FFB6F8B1
:104C50009020079BFA3A00211B68A6F8902086F85E
:104C60009210FEF70AB88D49079B0A781B68844D9D
:104C700042F004020A70FEF700B8894B02220320BA
:104C8000B2E4F7F79BFC96F88E30FFF717BA1020C6
:104C900001F0FAFE202001F0DFFE8249754F081F67
:104CA00014F0C6F8804B02221A70734E96F8D43076
:104CB000002B00F03981B5F80080FFF7D2B97B4BAB
:104CC0006C4F5B8997ED007A07EE903AF8EEE77A41
:104CD000B0EEC77AB4EEE77AF1EE10FA7FF527AFBF
:104CE00097ED017AB0EEC77AF4EEC77AF1EE10FADA
:104CF0007FF71DAF18F0200F7FF41DAF202001F0CB
:104D0000C3FE96E80C006A490A60084641F8043F71
:104D100014F08EF8644B01221A70C6E7102001F0DF
:104D20009BFE614BB5F8008083F800904FF00109BD
:104D3000F6E64E465F4A5278B2423FF41EAF5E4BF3
:104D40000E9330461EF002FF0E9B9B781BB1494626
:104D50000C202DF053F8731CDBB2474E8CE6002676
:104D6000B146E7E708231A46FEF7BDBB07231A46FC
:104D7000FEF7B9BB06231A46FEF7B5BB05231A4654
:104D8000FEF7B1BB04231A46FEF7ADBB03231A4658
:104D9000FEF7A9BB02231A46FEF7A5BB01231A465C
:104DA000FEF7A1BB202001F057FE3F4B00221A70F6
:104DB0007BE7424A079B324D1B684FF4C871118054
:104DC000FDF75BBF86F8941086F895002C4DFEF732
:104DD0002CBE4FF4FA6102201EF0E2FD49E4002CE3
:104DE0003DF409AF244E96F88D30002B3DF42DAEE6
:104DF0002BF05CFD002386F88D30FDF726BE1346B0
:104E0000022212E74FF6FE730FE702230DE700219F
:104E100001201EF0C5FDB6F89020079B963A0021B0
:104E20001B68A6F8902086F89210FDF726BF002197
:104E30000846EEE7FF21002021F029FE96F88E308B
:104E400005E40121002021F022FE96F88E30FFF7C4
:104E5000FBBB0021FF2021F01AFE96F88E30FFF7F1
:104E6000F0BB0021012021F012FE96F88E30FFF7F2
:104E7000E5BB00BFF4830020342C0020FC7200202E
:104E8000C8A500202495002064550020C4A500205A
:104E9000E82E0020D34D6210F8A70020CAA50020FC
:104EA000B25500206C710020747100200472002043
:104EB0004429002040730020806D00206ED4002023
:104EC000494617202CF09AFF33E400210420A0E784
:104ED0002B4E1DF0ADFC86F88D40FDF7B6BD0021D0
:104EE000032096E70021022093E70F2049460F9305
:104EF0000E922CF083FFD6F8D0000F9B0E9A13E58C
:104F00000B202BF0EFFC079B1E4D1B68FDF7B5BE79
:104F1000002B3FF467AF1C491C4A09684FF47A70B4
:104F200000FB031313605DE74FF00109FFF714BBAB
:104F3000152049462CF062FFD6F8D000FFF7B0BB31
:104F400049460D200F930E922CF058FF0F9B0E9A9E
:104F5000BCE4102049460F930E922CF04FFFD6F878
:104F6000D0000F9B0E9AFFF7FABB112049460F9312
:104F70000E922CF043FFD6F8D0000F9B0E9A1EE540
:104F8000342C0020C8A5002058AA0020F872002068
:104F90002DE9F047C74C636820469847002800F089
:104FA000C380C54B1B780122042B84F83C2000F001
:104FB000BD80B4F91610B4F91820B4F91A30216381
:104FC0006263A363BD4B1B88002B69D0BC4DD4ED3D
:104FD0000C7AD5ED004A95ED050A95ED015A95ED4F
:104FE000067AD5ED035A95ED026AF8EEE76AD5ED3B
:104FF000047AA4EEA60AA5EE267A67EEC07AA5EE9C
:10500000C07AE6EE267A85ED057AC5ED067A2EF0B1
:1050100023FCD4ED0D6AD5ED094A95ED0E0A95ED08
:105020000A5A95ED0F7AD5ED0D7AD5ED0C5A95ED1E
:105030000B6A2063F8EEE66AA4EEA60AA5EE267ACD
:1050400067EEC07AA5EEC07AE6EE267A85ED0E7A96
:10505000C5ED0F7A2EF000FCD4ED0E6AD5ED124AA4
:1050600095ED170A95ED135A95ED187AD5ED167A48
:10507000D5ED155A95ED146A6063F8EEE66AA6EE72
:10508000A40AA6EE857A67EEC07AA0EE657AE6EE0F
:10509000867A85ED177AC5ED187A2EF0DDFBA063D0
:1050A000884FA17F884817F09FFC3B88002B40F079
:1050B0008480864ED6F8E450854B1B685B0743D44A
:1050C000B5F90070216B636BA06B824A824E92ED42
:1050D000026AD2ED006AD2ED015AC91B2163B5F90B
:1050E0000270DB1B6363B5F904703568C01B07EE03
:1050F000900AB8EEE75A07EE901AB8EEE77A07EE94
:10510000903AF8EEE77A36EE056A36EE877A77EE71
:10511000A57A0135A06382ED026A82ED007AC2EDC4
:10512000017A3560BDE8F087BDE8F0876B4BB4F9D4
:105130001600B4F91810B4F91A20188020635980A9
:1051400061639A80A2633DE7B6F89820322A00F0A6
:105150008880002A66D196F89530002BB0D0604840
:10516000D6F800215F4980FB0273D217C2EB2312ED
:105170002A80D6F8042180FB0273D217C2EB2312D7
:105180006A80D6F80831A78A80FB0302DB17C3EBDD
:105190002213DB1BAB800023CB6086F8953027F011
:1051A000A1FC02F0A7FE27F085FCF7F76FF80120BD
:1051B0002BF0BEFCD6F8E45082E7444E226BD6F8C2
:1051C000E450B3F5C87F4FF0000323632B80398888
:1051D00018BFD6F8E800B7F8008008BF0020B1F586
:1051E000C87F18BFD6F8EC30616B02440B44002036
:1051F000B8F5C87F6063C6F8E820C6F8EC30688070
:1052000052D0D4F838E0D6F8F010A0637144B8F169
:10521000010FA880C6F8F01068D008F1FF38A7F891
:10522000008049E7D6F80001236B00210344C6F84B
:10523000003121632980D6F80401636B6163034464
:10524000C6F804316980A36BD6F80801A163034452
:10525000012AC6F80831A98075D0013AA6F898202D
:1052600079E72B8820491F48276BA6F8F4300023E4
:10527000B5F802E0B5F804C0C0684B608B602363EA
:10528000C6F800712B80616BC6F8041163636B80F4
:10529000A16BC6F80811A363A6F8F6E0A6F8F8C05B
:1052A000C6F8FC00AB80D8E7A36BC6F8F030A0636B
:1052B000A880B2E780A50020E18D002028A400206E
:1052C0002CA400206ED40020B0A50020342C002097
:1052D000247C00205847002054470020E48D002003
:1052E0001F85EB51F8A70020342D0020DFF88CC07B
:1052F000DFF884E0C8328CFB02A9C833D217C2EBB6
:10530000E9128CFB03A9DB17C3EBE913C8316B80EF
:105310002A808CFB013CA28ACB17C3EBEC139B1AAF
:10532000AB80CEF80C0027F0DDFB02F0E3FD27F0A8
:10533000C1FBF6F7ABFF40462BF0FAFBB7F8008055
:10534000D6F8E45069E70B2086F89A1086F8942086
:105350002BF0C8FAD6F8E450074BB6F8F420B6F8AC
:10536000F670B6F8F800D6F8FC102A806F80A88096
:10537000B6F89820D96070E7F8A700201F85EB5198
:105380002DE9F0478C4B1B78DB07074644D58B4B48
:105390008B4D1C788B4E012C59D01CD3022C07D17D
:1053A00089498A4A09881288914201D901241C70CE
:1053B000EB7AE3B12B89D3B1854B1B78BBB10BF0F2
:1053C0005DF9002800F09B802B7B83422CBF0121DC
:1053D000002131700CE07C497E4A098810886A7B84
:1053E000801A8842E2DAEB7A0024002BE2D131788D
:1053F0002A79632A06D8022C774E00F0BA803378D7
:10540000002B5DD1754AAB7A8C4238BF0C461470C4
:10541000002B4CD1BDE8F0876B4B694D19885B8838
:10542000E878CB1A83EAE3728142A2EBE3721DD3E0
:105430002B788B421AD3614B1C78E01E012861D96E
:105440006749097802294FD0012C5E4EA5D15F4AE9
:105450005D491288687B0988121A914239DD5D4ADC
:1054600012888A42A4D200241C70A1E7B1EB400F3D
:10547000E1DC524B1C78E11E012940F29480022AA3
:10548000DEDC57494F4E0878DFF84481DFF844C12D
:10549000DFF838E100210324022834701C7088F8FA
:1054A0000010ACF80010AEF8001081D11FE0012C04
:1054B00071D0022C0BD10720BDE8F0472BF012BAB7
:1054C0007068381A474B984258DD72709AE7BDE809
:1054D000F08702241C706BE7022AD2DD404909786C
:1054E00002294FF0040464D13949364E09783E4808
:1054F000022ACCBF00220122C28081804BE7022118
:10550000317075E7022A9BDC95F800C091FBFCFC2A
:105510000CF1010CBCF1080FDFF8B4A0304EA878F4
:1055200095F801E096F800802A4CDFF8A090254E0F
:10553000A8BF4FF0080C8AF800C01FFA8CFA10FBC5
:105540000AF01EFB0AFE80B2DFF88CA02080A9F8CA
:1055500000E000244FF0640EB8F1020F34701C70AC
:10556000CAF804408AF801E07FF439AF0FFA8CF1F1
:10557000BDE73078A0B9012377603370C2F16402CF
:105580001A4B00FB02F083FB0023C017A0EBA350D3
:105590006430707036E70820BDE8F0472BF0A2B900
:1055A0007368F81A8EE7032C96D10D490978022901
:1055B0009AD0044EFCE600BF7082002058340020D0
:1055C00064A5002068340020DC8300205C340020C7
:1055D000F28300205A34002060340020B85E00209E
:1055E000E18D00207F969800E48D00206BCA5F6BF0
:1055F0000C4B1B78DB0700D570470B490B68002B61
:10560000FAD04FF47A7202FB03F39842F4D3074BBB
:105610001B781BB9064B9A681B69136000230B604B
:10562000704700BF70820020207300201473002098
:105630000073002008B50EF025FAF4F77FFF00BFD5
:10564000024A034B1278197813F0F6BC4029002067
:10565000412900209F4B1B7803B170472DE9F0438F
:105660009D4D2B688BB013B90BB0BDE8F0839B4EFA
:105670009B4A3378044601A8D75C22F099F87368F6
:1056800003F5C333A0339C4205D9032F68D8DFE864
:1056900007F0485C3F10934B1B78DB07E4D42B6882
:1056A000002BE1D01B681B68002BDDD020469847FB
:1056B000DAE704AF384622F07BF897E8070007AB3B
:1056C00003C39DF810101A80002974D108A813F0A4
:1056D0006DFC0DF11E0013F081FC38460A2207A96B
:1056E0002FF04EF87F4B1A78071C18BF012702F0E5
:1056F00001027D49337808787460013393FBF0F13F
:1057000000FB11333370002AC9D0002FC7D1ABE79B
:10571000DFF8D08198F8002012F0010251D0002764
:10572000E7E79DF80430DFF8BC8143B398F8003018
:10573000D9075CD56C4A337811787460013393FBD8
:10574000F1F201FB123333708EE704A813F046FC2C
:105750000746002840D1634B1A7802F00102C8E7DF
:10576000604A614933780978107874600133C00762
:1057700093FBF1F201FB1233337090D574E798F884
:105780000030DA07D6D404A813F010FC002840F04B
:10579000848055493378087898F800207460013384
:1057A00002F0010293FBF0F100FB11333370002A89
:1057B0003FF475AF58E70DF11D0107A813F01AFC6F
:1057C00087E707A813F0FEFB00284AD198F80020CD
:1057D000002702F001028CE707A821F0E9FF9DF8FD
:1057E0001E009DF8103083422ED10027B3E704A994
:1057F0000DF1030013F0FEFB0028CAD007A821F02A
:10580000D7FF9DF81C009DF803309DF81D108342C2
:1058100003D19DF810308B42BBD02B684BB11A7965
:10582000824206D35A798A4203D31B68DB6803B1EC
:1058300098472D4A337811787460013393FBF1F265
:1058400001FB123333702AE72B68002B83D09A793F
:10585000824280D31B681B69002B3FF47CAF9847C2
:1058600079E727202CF082FA07460028AED01F4B9C
:10587000DB88002BAAD127202CF01CFA9DF81C30C5
:105880008146E8B1002BA1D1012013F0BFFB98F8AD
:1058900000204F4602F001022BE707A821F088FF05
:1058A000BDF82000BDF8103083423FF472AF2B6882
:1058B000002BBED01B689B69002BBAD09847B8E775
:1058C000002B83D013F0A2FB98F8002002F0010215
:1058D0000FE700BFFE53002074820020402D0020FF
:1058E000DD46002070820020E14600207882002002
:1058F0002DE9F04F2DED028BA0F10A0389B00C4683
:10590000ED2B00F24987DFE813F0590147074707FD
:105910004707470747074707470747074707470717
:105920004707470747074707470747074707470707
:1059300047074707470747074707E0024707470763
:1059400047076A01470747074707780147079D024E
:105950004707850247074D024707460247072102CE
:1059600047070D024707470747070802870547070C
:105970007405470747076D0547074505470747076C
:105980004707CE054707470747074707AF054707BC
:10599000390147078803E6014707470747074707D5
:1059A0004707470747070A054707DD044707AA04D3
:1059B0004707570447074404470747074707470770
:1059C0002104BA032C063403290165034A06330671
:1059D00022064707EA059B06470747074707470789
:1059E0008F06470747076D064707470747075E06C5
:1059F000CC06B8060507470747074707AC031E0351
:105A00004707FE0247074707470747074707470774
:105A10004707470747074707470747074707470716
:105A2000470721044707470747074707470747072F
:105A30004707470747074707470747074707EE0056
:105A400047074707470747074707470747074707E6
:105A500047074707470747074707470747074707D6
:105A600047074707470747074707470736054707D9
:105A700047074707470747074707470747074707B6
:105A800047074707470747074707470747074707A6
:105A90004707470747074707470747074707470796
:105AA0004707470747074707470747074707470786
:105AB0004707470747074707470747074707470776
:105AC0004707470747074707470747074707470766
:105AD000470747074707DC01B20147074707470762
:105AE0004707470784010B68DFF824C3591C9CF85B
:105AF000002021601A709CF800304BB3AF4EB04DBF
:105B0000B048B1490023226816F8017F02F1010E66
:105B1000C4F800E01770226815F8017F02F1010E49
:105B2000C4F800E01770226810F8017F02F1010E3E
:105B3000C4F800E01770226811F8017F02F1010E2D
:105B4000C4F800E017709CF8002001339A42DADCB8
:105B5000012009B0BDEC028BBDE8F08F9B4E33787D
:105B6000002BF5D09A4F002537F8021F204602F08F
:105B7000D6FC33780135AB42F6DCE9E7934E337857
:105B8000002BE5D0934F0025B846236817F8152061
:105B9000591C21601A7098F8011001EB810101EB8A
:105BA000810101F2EE2189B2204602F0B8FC33787F
:105BB0000135AB4208F10208E7DCC9E7864D28460B
:105BC0002CF0E8FC0028C3DD2B460544226813F8BE
:105BD000011B501C9D4220601170F7D1B8E77F4D2A
:105BE0000846298802F09BFCA988204602F097FC11
:105BF0002989204602F093FCAAE70B68784A581CD2
:105C000011782060197023685278591C21601A702D
:105C10009EE705A802F062FB002899D0BDF8141099
:105C2000204602F07CFC23689DF81620591C216058
:105C30001A7023689DF81720591C21601A70236878
:105C40009DF81820591C21601A7023689DF81920AE
:105C5000591C21601A7023689DF81A20591C216074
:105C60001A702046BDF81C1002F059FC70E75D4B1D
:105C700003F1700522681978501C206011702268A9
:105C80005978501C2060117022689978501C20604F
:105C900011702268D978501C20601170226819791F
:105CA000501C2060117022685979501C20601170BE
:105CB000226899790733501C9D4220601170D9D118
:105CC00046E7494D0846E98902F029FCA9892046A2
:105CD00002F025FC3CE70B68444D591C0122216071
:105CE0001A702368AA78591C21601A7028F07CFC6D
:105CF00023683F4A3F495E1C26601870B1F90010C6
:105D0000B2F9000002F02CFE23685A1C22601870C1
:105D10002988204602F003FC1AE70846002102F019
:105D2000E7FB15E7344D354E05F1300795F90210C4
:105D3000334B93F906208A4203F1080300F02F85C4
:105D40009E42F6D10835BD42F0D101E72D4B03F15B
:105D50005A0522685979501C206011702268197800
:105D6000501C2060117022685978501C20601170FE
:105D700022689978501C206011702268D978501CD4
:105D800020601170226819790633501C9D422060F2
:105D90001170DED1DCE60B681B4A591C527D216074
:105DA0001A70D5E6194D05F1800655F8041F2046F6
:105DB00002F09EFBAE42F8D1CAE600BF7F6F002022
:105DC0008F6F0020AF6F00209F6F002020A3002066
:105DD00072600020745100205A6D0020BC460020E3
:105DE000A45A002064310020F8A70020806D002014
:105DF000C8A70020CAA7002050950020A481002039
:105E0000748100205032002024950020D45E0020B0
:105E10007D6F0020B74D05F14006B5F88010204693
:105E200002F07DFB236895F88220591C21601A70CE
:105E3000236895F883200435591CB54221601A70F7
:105E4000EBD185E6AC4D0B682A7A591C21601A709B
:105E5000A98B204602F063FB298B204602F05FFBF2
:105E6000698B204602F05BFB2368EA7C591C2160A9
:105E70001A70A98C204602F052FBE98C204602F0F1
:105E80004EFB2368AA7F591C21601A70236895F87D
:105E90002020591C21601A70698C204602F03FFBBB
:105EA0002368EA7A591C21601A70E968204602F0DA
:105EB0001FFB23682A7C591C21601A70236895F8FF
:105EC0002120591C21601A7042E68C4D05F15006C4
:105ED00028782AF037FF2368027A591C21601A704B
:105EE00023686A78591C21601A702368AA78591CA3
:105EF00021601A702368EA780435591CAE4221608B
:105F00001A70E5D124E60B687D4F591C3A78216060
:105F10001A703B78002B3FF41BAE0025EEB23046E2
:105F200021F010FD23684278591C216030461A7018
:105F300021F008FD0189204602F0F1FA3B78013595
:105F4000AB42EBDC04E60A686E4B501C197820600B
:105F5000117022685978501C20601170226899785D
:105F6000501C206011702268DB78511C2160137076
:105F7000EEE5654D654E9FED668ADFF8CC81DFED7D
:105F8000658A05F120070EE0FCEEE77ACDED017A97
:105F9000BDF804102046043502F0C1FAAF4206F104
:105FA00018063FF4D5AD717C0029F3D05A4BD5EDDE
:105FB000007A1B78012BE7D1584B1B68DB0440F1BA
:105FC000A984F5EE407AF1EE10FA40F0DC8440F25C
:105FD000DC51DFE7524B0A681B78524D511C03F02D
:105FE00002032160137023682A7D591C21601A70F6
:105FF0002968204602F07CFA6968204602F078FAA7
:106000002989204602F08BFAE989204602F087FAB6
:10601000298A204602F083FA9AE50B68424D012650
:106020009A190A601E7018F0EFF8002840F08A8470
:106030003E4B2268511C21601070226841F2B4105E
:10604000511C185C216041F278111070595820469B
:10605000890A02F04DFAA96A2046490802F048FA76
:1060600076E5334D0846298A02F059FA698A2046B6
:1060700002F055FAA98A204602F051FA68E52D4B44
:106080009B8AB3F5006F00F25A84B3F5806F00F27B
:106090007784B3F5007F34BF01270227264D05F131
:1060A0000C0655F8041B91FBF7F1204689B202F06B
:1060B00036FAB542F5D1214D214F05F10C06B5EC6C
:1060C000010AD7ED077A80EE270A2DF0C5FB81B2D1
:1060D000204602F024FAB542F1D11A4D05F10C0622
:1060E00055F8041B204689B202F019FAAE42F7D1E6
:1060F0002EE500BFD85E0020249500205C500020D3
:10610000C5820020646F00202C590020647D00208F
:106110000000404200E08244487E0020247C0020B1
:10612000CAA500203CAD002068CA002054AD002064
:10613000247E002080A50020B0A50020187C00202F
:1061400024740020B04D0020DB9B91410025814646
:10615000DFF80C83DFF80CB30495039505950695DD
:1061600001214FF6FF7A05E001350B2D00F0358354
:1061700018F9011F4F1C4AFA05F3F5D0DE07F3D5D5
:10618000BBF800302B41D807EED505A802F09AFEE7
:10619000EAE70B68A44AA549D078A54A5D1C2560AA
:1061A000187023684979581C206019702368D278C8
:1061B000591C21601A70CBE42046002102F0AFF98F
:1061C0002046002102F0ABF92046002102F0A7F999
:1061D0002368984D00265A1C22601E7023682A6886
:1061E000591C92F82C2021601A7023682A68591CC7
:1061F00092F8362021601A7023682A68591C92F898
:10620000372021601A7023685A1C22601E70236890
:106210005A1C22601E7023685A1C22601E702B6854
:106220002046598F02F07BF92B682046198F02F027
:1062300076F923682A68591C92F82E2021601A707A
:1062400023685A1C22601E702B682046598E02F06B
:1062500066F92B682046998E02F061F978E4764E53
:106260000B687279734D591C21601A702B68204697
:10627000198C02F054F92B682046D98B02F04FF9A3
:106280007189204602F04BF9B189204602F047F9A6
:106290002B682046598C02F042F92B682046998CD5
:1062A00002F03DF9F189204602F039F9318A2046A1
:1062B00002F035F92A68236892F82620591C2160DB
:1062C0001A7045E45C4EF378002B00F02C830B68C9
:1062D0000822591C21601A70236801229918216034
:1062E0001A702368554D591C2A7921601A70236849
:1062F000AA78591C21601A702988204602F00FF9EB
:10630000E989204602F00BF92368F279591C2160D3
:106310001A702368EA78591C21601A7018E412F088
:106320007FFEFF28054600F0258308A8002300F81B
:106330000C3D12F047FE2268414B511C2160157044
:1063400022681978501C2060117022685978501CFE
:106350002060117022689978501C206011702268AA
:106360009DF81410501C206011702046998802F08E
:10637000D6F8FFF7EDBB0B68324A591C1278216042
:1063800005A81A7001F0AAFF23685A1C2260187031
:10639000FFF7DEBB0B682C4A2C4D11782C4A581C99
:1063A000206019701168204602F0A2F82368294A7B
:1063B000591C127A21601A702988204602F0AFF821
:1063C000A988204602F0ABF82989204602F0A7F8F8
:1063D0002046002102F0A3F82046002102F09FF899
:1063E000FFF7B6BB084608221A4902F053F8FFF738
:1063F000AFBB0B68184A194990785D1C256018706E
:1064000023685278581C20601A7023680A79591C36
:1064100021601A70FFF79CBB0B680122991821605C
:106420001A70FFF795BB00BFF8A7002090A70020C7
:1064300008A80020CCA50020007C0020247E00209D
:106440007882002096A30020A45A0020BC46002099
:106450006C5600202495002018A800205029002008
:10646000504E0408C8A500200B68994D591C2A7984
:1064700021601A7023686A79591C21601A70298872
:10648000204602F04CF82368AA79591C21601A7042
:106490006988204602F043F82368EA79591C216094
:1064A0001A70FFF755BB02F051FD2368894D002893
:1064B00003F101010CBF0222032221601A70298816
:1064C000204602F015F8A968204602F011F802F003
:1064D00015FD0146204602F00BF8FFF739BB7E4D53
:1064E0000B682A68591C127821601A702B68226880
:1064F0009978531C2360002311702A6821681A447C
:1065000001335279481C032B20600A70F5D12368AF
:106510002A68591C127A21601A7023682A68591C4B
:10652000D27821601A7023682A68591C1279216078
:106530001A702B682046598901F0F1FF2A682368F8
:10654000527A591C21601A702A68FFF75CBB2046FA
:10655000002101F0CDFF2046002101F0E0FFFFF710
:10656000F7BA084610225D4901F094FFFFF7F0BA30
:106570005B4D0846298801F0D2FF6988204601F06A
:10658000CEFFB5F90430574AD91782FB0323C1EB7C
:10659000A301204689B201F0C2FFFFF7D9BA524BDE
:1065A0000846198801F0BBFF504B2046198801F0BE
:1065B000B6FF4F4B22681B78511C03F0010321608A
:1065C0001370FFF7C5BA4B4D0846298801F0A7FFA5
:1065D0006988204601F0A3FFA988204601F09FFFAB
:1065E000FFF7B6BA444D05F16006A988204601F0D0
:1065F00096FFE988204601F092FF2989204601F0A4
:106600008EFF2368AA7A591C21601A702368EA7ADF
:10661000591C21601A7055F80C1B204601F068FFC8
:10662000AE42E2D1FFF794BA344952232268501C9B
:106630002060137011F8013F002BF7D1FFF788BAE3
:106640002F4800232268056803EB4301561C6D5C4C
:1066500026601570026825680A446E1C5278266010
:106660002A70026825680A4401339278691C0A2B53
:1066700021602A70E6D1FFF76BBA0B68214A2249E4
:106680001078224A5D1C2560187023688978581C90
:106690002060197023689278591C21601A70FFF7E6
:1066A00057BA0A681A4B13491878551C25601070A0
:1066B00022685878551C2560107022689B78501C01
:1066C000206013702046C98801F029FFFFF740BA07
:1066D000944D0020E81D0020D0A500201C5900206A
:1066E00078A5002067666666D4A50020586D002056
:1066F000727100207C4D0020A4300020204E040840
:10670000CCA50020007C0020F8A7002008A80020CD
:10671000F0A70020DFF838E30027FEB2714600231F
:106720002268501C206016702268501C2060137074
:10673000226811F8010F0133551C062B25601070DB
:10674000EED10137062F0EF1060EE6D1B549002332
:106750002268501C206017702268501C2060137043
:10676000226811F8010F0133551C0B2B25601070A6
:10677000EED12368AC4A581C0721206019702368A9
:106780000021581C20601970236892F8F020591CD1
:1067900021601A70FFF7DCB90020FFF7DAB923682F
:1067A0005A1C226019702988204601F0B8FE23681F
:1067B000EA78591C21601A7023682A79591C2160D3
:1067C0001A702368AA79591C21601A7023686A79A3
:1067D000591C21601A70FFF7B5BADFF878A20025BE
:1067E0004FF0A8080135C5F1200208FA02F2A5F120
:1067F00020032AFA05F6164328FA03F31E43282D30
:1068000006F001024FF000030BD01343EAD0E8B2C8
:106810002BF0ACFA0028E5D0294605A802F052FB7F
:10682000E0E7824B1B78DA0700F194800025804E68
:106830002F4602E00135282D0DD02946304602F0C2
:1068400050FB0028F6D0294605A802F04AFB002894
:106850005BD10137EEE7774B774DB3F85010204608
:1068600001F05DFE0021204601F059FE734B1968CE
:106870004B0103F02002C1F340031343C1F3800234
:1068800043EA4203C1F3C00243EA8203C1F3401268
:1068900043EAC20301F010011943204601F03FFE14
:1068A00003A90422204601F0F5FD23682978644AF3
:1068B000581C2060197011886429A8BF64212046E3
:1068C00001F02DFEB9F1960F49D00021204601F0CC
:1068D00026FE2168B7F1190348BFA7F11203A3F3FD
:1068E000C4034A1C226020461A460B7004A901F01A
:1068F000D1FD2368534A581C11212060197020468D
:10690000116801F0F5FDFFF723B9394603A802F03D
:10691000D9FA9EE7F4EEC87AF1EE10FA59DA4FF49C
:106920007A71FFF737BB0B68B178474A581C206073
:10693000197023681278591C21601A70D1E4082755
:10694000FFF7ACBB95F82420404B002A38D13046E5
:10695000FFF76FBB059B43F00103059366E72368D0
:106960000322591C21601A7023686A78591C21601F
:106970001A70AEE723685A1C22601870FFF7E8B857
:106980000427FFF78BBBF4EEC87AF1EE10FA3FF55F
:106990001EABF4EEE87AFDEEE77AF1EE10FA17EEB0
:1069A000901A2FD86FF4F973303903FB01F140F2DC
:1069B000E73391FBF3F101F2DB5189B2FFF7EABA59
:1069C0005978022918D003290CBF04203046FFF75C
:1069D00030BBFDEEE77A40F2E73217EE903A303BFB
:1069E00002FB03F388FB0312D917C1EB622101F20A
:1069F000E93189B2FFF7CEBA042A34BF022003205E
:106A0000FFF717BB40F2F313A1F5836103FB01F11C
:106A100040F2E73391FBF3F101F2DD5189B2FFF768
:106A2000B9BA00BFBB5F0020D85E00207082002092
:106A30001CAD00206C1E00204073002074A50020B7
:106A40006A2F0020C4A50020ECA7002054AD002030
:106A5000975F002090E33FF438B5094D2B8823EA77
:106A60000000834228800AD0064B1421FF220E200A
:106A700002241C7059709A7029F034FF288838BDA0
:106A8000C8A500206C33002038B5094D2B88184369
:106A9000834228800AD0074B1421FF220E200224B3
:106AA0001C7059709A7029F01DFF288838BD00BFEE
:106AB000C8A500206C330020024A136818431060F8
:106AC000704700BFC4A50020684B694870B55822C4
:106AD000012500211D702DF07CFE664A6649674C39
:106AE000674800230B60136009F04AFF2946052020
:106AF00009F096FF6579291C4FF0070018BF0121A6
:106B000009F08EFFA679311C4FF0080018BF012153
:106B100009F086FFA37A002B7DD05A4C002D40F05F
:106B20008780311C18BF0121092009F079FF2168F5
:106B3000554EC1F340510E2009F072FF3168CA076B
:106B400000F186804E4D11F0020173D1003118BF63
:106B50000121032009F064FF4C4A4D4B128E93FB38
:106B6000F2F301210420C5F8143109F059FF494B13
:106B70000620197809F054FF01210A2009F050FF7E
:106B800021680B20C1F3C01109F04AFF21680C20D5
:106B9000C1F3802109F044FF21684B0508D53E4B25
:106BA0001B7A083B012B9CBF4FF4FA63C5F8803277
:106BB000C1F300410D2009F033FF21680E20C1F31D
:106BC000405109F02DFF21680F20C1F3804109F0E9
:106BD00027FF21681020C1F3C06109F021FF0121C6
:106BE000112009F01DFF0121122009F019FF0121D8
:106BF000132009F015FF294B1968B3F8464029B155
:106C000011F0ACFF014608B9C4F3C0011420BDE87F
:106C1000704009F005BFE37A1A4C002B7FF47EAF79
:106C2000216811F480213FF47FAF002D3FF479AF4C
:106C3000012179E70121022009F0F2FE184B3168A9
:106C4000DB6A0A2BB8BF0A2301F00201AB677DE7BC
:106C5000144B0B4D1B680A2B4FF00101B8BF0A23E0
:106C600008466B6409F0DCFE31686CE7D83400201C
:106C700080340020DC3400207C34002064A5002017
:106C80006C1E0020247C002074A50020509500205C
:106C900040420F00AC500020249500208872002054
:106CA00080A50020147C002010B5084B03F10C01D6
:106CB00093F900205C78845402449C78D470DC788A
:106CC000947104338B42F3D110BD00BF5C4E0408B5
:106CD000002870B51EDB0928044620DD012303EBE4
:106CE00083035B00B0FBF3F2092AF8D87BB10E4EA8
:106CF000B4FBF3F00928CCBF57223022A6FB03E5F2
:106D0000024403FB1044EB0801F8012BF0D10023EF
:106D10000B7070BD2D230B7040420131DBE730302A
:106D200001F8010BF3E700BFCDCCCCCC884230B4E6
:106D30004FF001042ED301FB04F4B0FBF4F58D42B7
:106D4000F9D284B1AAB901E0B0FBF4F5092DCCBFAA
:106D5000572230222A4404FB150003F8012BB4FB10
:106D6000F1F4002CF0D100221A7030BC7047B0FB57
:106D7000F4F5092DCCBF372230222A4404FB15003C
:106D800003F8012BB4FBF1F4002CF0D100221A70AF
:106D900030BC70470546002AEBD1D7E72DE9F04714
:106DA00014461D46064600234FF47A7220462946B3
:106DB0002CF0BAF8DFF848814B4A4C4F88FB003181
:106DC0000144C31782FB002EC3EB611188FB01282D
:106DD00087FB00278644464AC3EBEE2EC1EB011C1D
:106DE00082FB0E29A0EB8C0C0744424A86F806C0B1
:106DF000C3EB27474FEAEE7C08EB010ACCEBA90C6A
:106E000082FB07824FEAE1780CEB4C0CC8EB6A1866
:106E1000AEEBCC0EC8EB0818DFF8E8C086F804E04B
:106E2000A1EB880171718CFB0010F917C1EBE21224
:106E300040F2B55101FB1272C3EBE050B2F5896F1D
:106E40004FEA80073FDA40F2DA239A4243DCB2F598
:106E5000B77FB4BF4FF0000C4FF0010C4FEA4C0865
:106E6000254B08EB0C0103EBC1031FFA8CFE588C79
:106E7000224908EB0C0301EBC30116310B2301E09F
:106E800031F8020D82421BDA013BF9D11A4BC4449E
:106E900003EBCC0C0123BCF80C00B37007F2B27703
:106EA0000132121ABE44F270A6F800E020462946CC
:106EB0004FF47A7200232CF037F83281BDE8F08766
:106EC0000133DBB2E9E74FF0030EF44640F296508F
:106ED0004FF00608CCE74FF0020EF44640F229408E
:106EE0004FF00408C4E700BFC5B3A29107452EC206
:106EF000ABAAAA2A73B06D165C4E0408684E04084B
:106F000089888888792D031103685A1C02601970DA
:106F100070472DE9F047089C2578002B804689466C
:106F20000CBF4FF0200A4FF0300A661C35B3002A20
:106F300029DD334601E0024698B113F8011B501ECB
:106F40000029F8D1971E60B13D46013D51464046AB
:106F5000C8476B1C002BF8DC257827EAE770013066
:106F600055B1041B29464046C847301916F8015B45
:106F7000002DF7D1BDE8F087BDE8F087002A04DCDA
:106F80002846BDE8F0870020EBE7571EDCE7836862
:106F90004268D0ED037A00EB83010133934281ED27
:106FA000040A836004BF0023836000EB830393ED36
:106FB000047A036870EE277A9A42C0ED037A77EE7E
:106FC000C77AC0ED037A0CDA013307EE103AF8EE17
:106FD000C76AB7EE007A87EEA60A036030EE070AAA
:106FE000704707EE102AB8EEC77A87EE870A704717
:106FF00090ED057A90ED004AD0ED066AD0ED014A99
:10700000D0ED047A90ED035AD0ED025AA4EE007A46
:10701000B0EE406AB0EE470AB0EE667AA6EE247A89
